:0200000480007A
:10000000970500009385C547732510FC6B10B5005C
:10001000EF00C046130510006B00050017650100D6
:10002000130545A617660100130686B73306A640DA
:1000300093050000EF00505317150000130585C30A
:10004000EF00903EEF009048EF0080006F00103FFF
:1000500037350180130101F3130585192322910C13
:100060002326110C2324810C2320210D232E310B58
:10007000232C410B232A510B2328610B93040102EB
:10008000EF00C0641387040093070000930640024A
:100090002320F7009387170013074700E39AD7FE42
:1000A0001304000013071000B73901801309400240
:1000B00083A70400930504001385491C6386870009
:1000C000EF00C06013070000130414009384440081
:1000D000E31024FF63140718373501801305C51F8B
:1000E000EF00C05EEF00401F373501801305C520CB
:1000F000EF00C05DEF0000253735018013050522B4
:10010000EF00C05CEF004030373501801305052358
:10011000370400FFEF00805B93040000373B018051
:10012000B73A0180373A0180B73901801309440199
:10013000232094009305040013054B24EF0000597D
:100140009385040013850A25EF0040589385040029
:1001500013054A26EF0080571385492713044400EE
:10016000EF00C05693841400E31424FD373501805A
:100170001305C528EF008055B75701809387070204
:100180002326F10037690180B7050080B757018049
:1001900013074000938707061306C100938545287F
:1001A00013050001130909A92328F100232CE100FC
:1001B000232EE100232A2101EF00406F3735018013
:1001C0001305C52AEF0080508327C1019304000066
:1001D000373A0180B739018063860704832781019C
:1001E0001304000063860702B38797021385892EE4
:1001F000B387870093972700B307F90083A507000B
:1002000013041400EF00804C83278101E36EF4FC9B
:1002100013050A1CEF00804F8327C101938414004B
:10022000E3EEF4FA373501801305052FEF00004E99
:100230008320C10C0324810C8324410C0329010C6D
:100240008329C10B032A810B832A410B032B010B4A
:10025000130500001301010D678000003735018090
:100260001305451DEF0080466FF01FE79307000060
:100270006388070037150080130505C76F00D01A83
:100280006780000083A7450003A70500131525001C
:10029000B386A7003307A70083A7850003270700BD
:1002A00083A606003385A700B307D7002320F500F7
:1002B00067800000F32730CC3767018093962700D2
:1002C000130787AF3307D7002320F70093B7170032
:1002D0006B8007006780000037350180130101FF44
:1002E0001305C52F2326110023248100EF00003EB3
:1002F000930740006B800700732700CC37540180C0
:100300001304040A93172700B307F40023A0E7009F
:10031000930710006B80070003250400EF00C04224
:1003200003254400EF00404203258400EF00C04154
:100330000325C400032481008320C10013010101AF
:100340006F008040130101FF232611002324810048
:10035000930740006B800700F32700CC13B72700FA
:100360006B20070013071000637AF70613B73700F6
:100370006B2007003764018013072000130484B04A
:100380006388E70493972700B307F4001307D000AE
:1003900023A0E7006B3000006B30000093071000D3
:1003A0006B80070003250400EF00003A032544009A
:1003B000EF00803903258400EF0000390325C400D5
:1003C000032481008320C100130101016F00C037A5
:1003D0009307C0002324F4006FF0DFFB13C717005E
:1003E0006B20070037640180130484B06398070012
:1003F0009307A0002320F4006FF0DFF99307B0000B
:100400002322F4006FF01FF9130101FFB7070080EA
:100410002326110023248100130740009387472BD4
:100420006B10F700F32730CC37640180130484AFDE
:10043000139727003307E4002320F70093B7170032
:100440006B80070003250400EF0000300325440003
:10045000EF00802F03258400EF00002F0325C40048
:10046000032481008320C100130101016F00C02D0E
:10047000EF004058130500006B000500732500FCD9
:100480006B000500975101009381C1391701007F6E
:10049000130141B793050040732610CCB385C50204
:1004A0003301B140F32630CC63860600130500000B
:1004B0006B0005006780000063060520130101F54D
:1004C0002324810A232E31092326110A2322910A8B
:1004D0002320210B232C4109232A510923286109B8
:1004E00023267109930905000345050013841900AB
:1004F0006306051CB7340000B73A0180138A050073
:100500001309500293849480938ACA3063042505AA
:10051000EF00806F03450400130B140013040B005D
:10052000E31605FE330534418320C10A0324810A02
:100530008324410A0329010A8329C109032A810965
:10054000832A4109032B0109832BC1081301010BE5
:1005500067800000130B04001306D0009306100000
:1005600003470B0013050B00130B1B00930707FE3B
:1005700093F7F70F6368F600B397F600B3F79700A9
:10058000E39007FE9307A002630AF7001306A0009A
:1005900093050104EF00902C032B010483470B000B
:1005A0001307E00213051B00638EE70C938747FBDC
:1005B00093F7F70F1307E0026364F702939727009E
:1005C000B387570183A707006780070003471B0015
:1005D00093078006630AF708130B0500130515003F
:1005E0002300210533058540635AA00893070400C2
:1005F000130711043306A40083C60700938717006E
:1006000013071700A30FD7FEE398C7FE13051500C5
:1006100093070108B387A70093060A001306010495
:100620009305001013050100238007FCEF00103133
:1006300013040100B30BA100635AA000034504009A
:1006400013041400EF00405CE39A8BFE03451B008B
:1006500013042B00E31C05EA6FF0DFEC03471B00DB
:100660009307C006E31AF7F613053B0023002105A4
:1006700033058540130B2B00E34AA0F61305100049
:100680006FF01FF903471B009307A002631AF700DE
:1006900083472B0013053B00130B2B006FF01FF15A
:1006A0001306A00093050104EF00501B032B010467
:1006B00083470B0013051B006FF05FEF130510005D
:1006C0006FF09FE61305F0FF67800000130101FC47
:1006D000130341022322B10293050300232E1100CC
:1006E0002324C1022326D1022328E102232AF10276
:1006F000232C0103232E110323266100EFF0DFDBFF
:100700008320C1011301010467800000130101FF70
:10071000232481002326110013040500034505004E
:10072000630C05001304140013041400EF00C04D03
:100730000345F4FFE31A05FE8320C1000324810072
:100740001301010167800000130101FF23229100C2
:100750002326110023248100232021019307F00088
:100760009304050063FCA704373901809306000059
:10077000130400021309893C1304C4FFB3D7840097
:1007800093F7F7003307F9006394070063880600C6
:1007900003450700EF00404793061000E31E04FCEA
:1007A000032481008320C100832441000329010028
:1007B0001305A000130101016F000045B737018048
:1007C0009387873CB384A70003C50400EF00C043B0
:1007D000032481008320C1008324410003290100F8
:1007E0001305A000130101016F000042130101FE77
:1007F000232E1100232C8100232A9100232821017C
:1008000023263101F32700FC6B800700F32650CC30
:10081000F32930CC732700CC732600FCB767018026
:1008200093962600938787B1B387D70083A40700E8
:1008300003A4040183A6C40033A98900930704001C
:100840003309D9003384360363D4F9009387090050
:100850003304F40083A684003304C402B307E9021E
:100860003304D4003304F40033098900635E2401A7
:1008700083A7040083A54400130504001304140097
:10088000E7800700E31689FE93B919006B80090021
:100890008320C10103248101832441010329010133
:1008A0008329C1001301010267800000130101FCCC
:1008B000232E1102232C8102232A910223282103B3
:1008C00023263103F32620FC732810FC732400FC3C
:1008D000F32750CC1307F0016344F70CB30804036B
:1008E0001307100063D4A8003347150363C8E60C50
:1008F00063D8E70A9386F6FF3343E50293080300C3
:100900006396F6003365E502B3086500B3C4880258
:1009100033E9880263CA040B9306100033C704034B
:10092000630607009306070033E70403B7690180F5
:10093000938989B1232EE1001307C1002326B1005A
:100940002328C100232CD1003303F30293972700FF
:10095000B387F90023A0E700232A6100634C9006C7
:100960006300090433848402232A81006B00090098
:10097000F32750CC732520CC93972700B389F90037
:1009800083A7090083A6870003A7070083A5470064
:100990003305D500E7000700930710006B800700C0
:1009A0008320C1030324810383244103032901031A
:1009B0008329C10213010104678000001387060028
:1009C000E3CAE7F26FF0DFFD1307000093061000A3
:1009D0006FF0DFF5138704006354980013070800D5
:1009E000B70700809387C77E6B10F700EFF01FE01A
:1009F0006FF01FF7F32750CC3707FF00B387E700EE
:100A000093978700732700B023A0E700732710B0E7
:100A100023A2E700732720B023A4E700732730B098
:100A200023A6E700732740B023A8E700732750B040
:100A300023AAE700732760B023ACE700732770B0E8
:100A400023AEE700732780B023A0E702732790B09E
:100A500023A2E7027327A0B023A4E7027327B0B054
:100A600023A6E7027327C0B023A8E7027327D0B0FC
:100A700023AAE7027327E0B023ACE7027327F0B0A4
:100A800023AEE702732700B123A0E704732710B158
:100A900023A2E704732720B123A4E704732730B10E
:100AA00023A6E704732740B123A8E704732750B1B6
:100AB00023AAE704732760B123ACE704732770B15E
:100AC00023AEE704732780B123A0E706732790B114
:100AD00023A2E7067327A0B123A4E7067327B0B1CA
:100AE00023A6E7067327C0B123A8E7067327D0B172
:100AF00023AAE7067327E0B123ACE7067327F0B11A
:100B000023AEE706732700B823A0E708732710B8C1
:100B100023A2E708732720B823A4E708732730B877
:100B200023A6E708732740B823A8E708732750B81F
:100B300023AAE708732760B823ACE708732770B8C7
:100B400023AEE708732780B823A0E70A732790B87D
:100B500023A2E70A7327A0B823A4E70A7327B0B833
:100B600023A6E70A7327C0B823A8E70A7327D0B8DB
:100B700023AAE70A7327E0B823ACE70A7327F0B883
:100B800023AEE70A732700B923A0E70C732710B937
:100B900023A2E70C732720B923A4E70C732730B9ED
:100BA00023A6E70C732740B923A8E70C732750B995
:100BB00023AAE70C732760B923ACE70C732770B93D
:100BC00023AEE70C732780B923A0E70E732790B9F3
:100BD00023A2E70E7327A0B923A4E70E7327B0B9A9
:100BE00023A6E70E7327C0B923A8E70E7327D0B951
:100BF00023AAE70E7327E0B923ACE70E7327F0B9F9
:100C000023AEE70E67800000974201009382824A7C
:100C100083A20200732320CC131303013363A300C8
:100C200023A0620067800000930505009306000082
:100C300013060000130500006F004052130101FF6E
:100C400093050000232481002326110013040500CE
:100C5000EF00805AB767018003A507A78327C50364
:100C600063840700E780070013050400EFF05F804E
:100C7000130101FF23248100B757018037540180FD
:100C80001304C4019387C701B387874023229100CF
:100C90002326110093D42740638004029387C7FF63
:100CA00033848700832704009384F4FF1304C4FF74
:100CB000E7800700E39804FE8320C100032481003D
:100CC000832441001301010167800000130101FF2B
:100CD00023248100232021013754018037590180CA
:100CE00093078401130989013309F9402326110070
:100CF000232291001359294063000902130484013F
:100D00009304000083270400938414001304440018
:100D1000E7800700E31899FE3754018037590180B6
:100D2000930784011309C9013309F9401359294074
:100D30006300090213048401930400008327040064
:100D40009384140013044400E7800700E31899FE1D
:100D50008320C10003248100832441000329010072
:100D600013010101678000001303F0001307050061
:100D7000637EC3029377F7006390070A63920508C6
:100D8000937606FF1376F600B386E6002320B700BD
:100D90002322B7002324B7002326B7001307070137
:100DA000E366D7FE6314060067800000B306C34005
:100DB0009396260097020000B38656006780C6000F
:100DC0002307B700A306B7002306B700A305B700A3
:100DD0002305B700A304B7002304B700A303B7009B
:100DE0002303B700A302B7002302B700A301B70093
:100DF0002301B700A300B7002300B70067800000FD
:100E000093F5F50F93968500B3E5D500939605010C
:100E1000B3E5D5006FF0DFF6939627009702000048
:100E2000B386560093820000E78006FA93800200A2
:100E3000938707FF3307F7403306F600E378C3F6DE
:100E40006FF0DFF3130101FF23261100232481003B
:100E500093071000638EF60A93074002938F0600F3
:100E600063E8D70A37330180938705001303D33D26
:100E700003C70700138E0700938717003308E300AA
:100E80008348080093F88800E39408FE1308D00212
:100E9000630807151308B002630C0709B702008046
:100EA0001308070093C2F2FF13040000638E0608C4
:100EB000130700016386E614B3F3F20393080000FE
:100EC00013030000130E9000130F9001B3DEF20322
:100ED000130708FD6378EE001307F8FB6360EF0A61
:100EE000130798FC6354D70A63C608089308F0FFF9
:100EF00063EA6E0063826E0C930810003303F30301
:100F0000330367009387170003C8F7FF6FF05FFC98
:100F1000EF00C0408320C1000324810093076001DB
:100F20002320F50013050000130101016780000074
:100F3000B702008003C8070093C2F2FF93072E0098
:100F400013040000E39606F6130700036314E80A8F
:100F500003C70700930680051377F70D631ED70AB2
:100F600003C81700930F0001938727009306000121
:100F70006FF09FF49308F0FF6FF0DFF81307F8F9B4
:100F80006366EF00130798FAE340D7F663CA0802D6
:100F9000630404003303604063060600639A080696
:100FA0002320B6008320C100032481001305030021
:100FB0001301010167800000E3C6E3F46FF0DFF383
:100FC000130720022320E50013830200E30C06FC34
:100FD0009385F7FF138302002320B6006FF09FFC78
:100FE00003C80700B702008093072E001304100007
:100FF0006FF0DFEB930FA0009306A0006FF0DFEB24
:10100000130700036300E802930F00016FF0DFEAAB
:10101000930203006FF0DFFB930F800093068000C4
:101020006FF09FE903C70700930880051377F70D5A
:10103000E30817F3930F00016FF01FE86FF09FE0D4
:101040003767018093070500032547A7930606002D
:1010500013860500938507006FF0DFDE3767018098
:1010600093070500032547A793060600138605008E
:10107000938507006FF01FDD130101F8232C810613
:10108000232E1106232A9106930706001304050058
:10109000634E060813860600930607001307802098
:1010A000231AE1002324B100232CB1006384070438
:1010B0009387F7FF9304F0FF930581002328F10045
:1010C000232EF100231B9100EF00002663569500AC
:1010D0009307B0082320F4008327810023800700B2
:1010E0008320C107032481078324410713010108DA
:1010F000678000009304F0FF93058100232801001E
:10110000232E0100231B9100EF000022635695005F
:101110009307B0082320F4008320C107032481072C
:101120008324410713010108678000009307B0087A
:101130002320F5001305F0FF6FF01FFE37670180D5
:1011400093070500032547A71387060093060600AB
:1011500013860500938507006FF01FF2B7670180C3
:1011600003A707A783278714638C070403A74700F7
:101170001308F001634EE806131827006306050202
:10118000338307012324C30883A88718130610009C
:101190003316E600B3E8C80023A417192324D3109C
:1011A000930620006304D5021307170023A2E7006B
:1011B000B387070123A4B700130500006780000070
:1011C0009307C7142324F7146FF05FFA83A6C71898
:1011D0001307170023A2E70033E6C60023A6C718AB
:1011E000B387070123A4B700130500006780000040
:1011F0001305F0FF67800000130101FDB767018050
:10120000232C410103AA07A723202103232611022F
:1012100003298A142324810223229102232E3101DF
:10122000232A5101232861012326710123248101EE
:1012300063000904130B0500938B0500930A10004B
:101240009309F0FF832449001384F4FF63420402EE
:1012500093942400B304990063840B0483A744107F
:10126000638077051304F4FF9384C4FFE31634FF0F
:101270008320C10203248102832441020329010245
:101280008329C101032A8101832A4101032B010122
:10129000832BC100032C8100130101036780000030
:1012A0008327490083A644009387F7FF638E870452
:1012B00023A20400E38806FA8327891833978A005B
:1012C000032C4900B377F70063920702E78006001A
:1012D0000327490083278A1463148701E304F9F87C
:1012E000E38807F8138907006FF0DFF58327C91833
:1012F00083A544083377F700631C070013050B0030
:10130000E78006006FF0DFFC232289006FF09FFA70
:1013100013850500E78006006FF09FFBB76701802B
:1013200003A547A767800000130101E12326111ED2
:10133000232A511D2328611D2320A11D138B050085
:10134000130D06002326D1002324811E2322911E83
:101350002320211F232E311D232C411D2326711DE7
:101360002324811D2322911D232EB11B930A0500E6
:10137000EF50D02783270500138507002320F104B1
:10138000EF7000718357CB002328010E232A010E32
:10139000232C010E232E010E93F70708232EA10202
:1013A0006388070083270B01639407006F10C05BFD
:1013B000B737018093874752232AF10083470D00F6
:1013C000930BC110B73901802322710F2326010E20
:1013D0002324010E23280100232C010023220104D1
:1013E000232C0102232401042326010423220100CB
:1013F00093880B009389096A6380072213040D0008
:10140000930650026382D73C8347140013041400F0
:10141000E39A07FEB304A4416300A4218326C10E0E
:101420008327810E23A0A801B38696009387170017
:1014300023A298002326D10E2324F10E93067000D8
:101440009388880063CAF638032741008347040065
:10145000330797002322E1006380071C83441400B4
:10146000A303010C130414001303F0FF130A00007C
:1014700013090000130CA005930C9000930DA0021B
:1014800013041400938704FE6364FC0403274101E2
:1014900093972700B387E70083A7070067800700BB
:1014A000130A0000938704FD8344040093162A0066
:1014B000338A4601131A1A00338A4701938704FDC1
:1014C00013041400E3F2FCFE938704FEE370FCFCBB
:1014D0006384041423069114A303010C130C10005D
:1014E000930C1000130DC114930D000013030000A2
:1014F00023260102232A010223280102937F2900C7
:1015000063840F00130C2C00137F49088327C10E3E
:1015100063160F0033088A41E34000738346710C61
:10152000638A06028326810E1306710C23A0C8006D
:1015300093871700130610009386160023A2C80095
:101540002326F10E2324D10E130670009388880001
:101550006340D660638C0F028326810E1306810CD4
:1015600023A0C80093872700130620009386160047
:1015700023A2C8002326F10E2324D10E13067000E7
:10158000938888006354D6006F00107B9306000890
:10159000E302DF4E33039341E34A605A9376091026
:1015A000E39E06380327810EB387970123A0A80185
:1015B0001307170023A298012326F10E2324E10E1E
:1015C0009306700063C0E66E938888001379490023
:1015D00063060900B3048A416346906E63548A012E
:1015E000130A0C0003274100330747012322E100BF
:1015F000E39C07602324010E63880D0093850D0092
:1016000013850A00EF20D01293880B00130D0400FD
:1016100083470D00E39407DE8327C10E6384070030
:101620006F1090398357CB0093F70704638407004A
:101630006F20803F8320C11E0324811E03254100AB
:101640008324411E0329011E8329C11D032A811DF4
:10165000832A411D032B011D832BC11C032C811CDC
:10166000832C411C032D011C832DC11B1301011F61
:101670006780000013850A00232E110123246100D6
:10168000EF50C07683274500138507002326F10419
:10169000EF7000409307050013850A00938407004C
:1016A0002324F104EF5080748327850003238100F5
:1016B0008328C101232CF102638404006F10C0153C
:1016C000834404006FF0DFDB8344040013690902E4
:1016D0006FF01FDB13690901937709026388076CB8
:1016E0008327C1009387770093F787FF03A74700FD
:1016F00083AD0700938787002326F100930C070032
:101700006340076E1307F0FF130C0900E30CE300BE
:1017100033E79D01137CF9F7E3160700E31A030092
:1017200013090C0013030000930C0000130D011BA0
:10173000138C0C0063D46C00130C03008347710CF2
:1017400023260102232A010223280102930D00000F
:10175000E38607DA130C1C006FF05FDA13690901E6
:1017600093770902638C07608327C1001387770092
:10177000137787FF832D0700832C4700930787008B
:101780002326F100137CF9BF13070000A303010C0B
:101790009306F0FF630AD366B3E69D011379FCF765
:1017A000E3980648E31E0312E31E07F6937C1C0031
:1017B000130D011BE38E0CF693070003A307F11A28
:1017C000130DF11A6FF0DFF6B304A441E318A4C5BA
:1017D000834704006FF05FC81306410E93050B00AA
:1017E00013850A00EF70003EE31E05E293880B00AC
:1017F0006FF09FC593778900638407006F1080079F
:101800008327C1001305010B232E11019387770055
:1018100093F787FF83A5070003A6470093878700F8
:10182000232461002326F100EF10C1218327010B3F
:101830008328C101032381002328F10E8327410B54
:10184000232AF10E8327810B232CF10E8327C10B52
:10185000232EF10E1305010F232E11012324610005
:10186000EF5000522326A10C930720000323810090
:101870008328C1016314F5006F10C05E9307100048
:101880006314F5006F109000930710066394F40042
:101890006F204012930710046394F4006F10D04639
:1018A00093FCF4FD9307F0FF232C91076314F300DE
:1018B0006F109015930770046394FC006F208017DD
:1018C000032EC10F23242107832E010F032F410F65
:1018D000832F810F9367091063540E006F20002A35
:1018E000232E010613890700930D0000930760045F
:1018F0006394FC006F10D02193075004232411033C
:101900006384FC006F10D029930C1300130C010B9F
:101910001308C10D93860C009307010D1307C10C2A
:101920001306200093050C0013850A002322610290
:101930002328D10B2320D103232AE10B232EE101FD
:10194000232CF10B2328F101232EC10B2324C101E9
:10195000EF40C016032E8100832F0101032FC10128
:10196000832E01020323410283288102330895015B
:10197000130D0500930C010A93850C0013050C0050
:10198000232E010123281101232461002328D10BD8
:10199000232AE10B232CF10B232EC10B2320010A58
:1019A0002322010A2324010A2326010AEFD09043AF
:1019B0000328C10103238100832801019307080044
:1019C000630205028327C10D63FE070113060003AE
:1019D00093861700232ED10C2380C7008327C10DC7
:1019E000E3E807FF0327C10CB387A7412328F100D1
:1019F0002328E10203278107930770046314F7008B
:101A00006F10500203278107930760046314F700E7
:101A10006F105027832701030327810793051004C4
:101A20009387F7FF2326F10C93F6F40F13060000BB
:101A30006318B7009386F60093F6F60F13061000AE
:101A4000230AD10C9306B00263DA070003270103CF
:101A5000930710009306D002B387E740A30AD10C86
:101A60009306900063C4F6006F2000231308310E24
:101A7000130508001306A000130E3006B3E6C702D4
:101A800093050500138307001305F5FF93860603EE
:101A9000A38FD5FEB3C7C702E3426EFE9387070349
:101AA00013F6F70FA30FC5FE9387E5FF63E4070165
:101AB0006F2040339306610D6F00800003C607005E
:101AC0002380C6009387170093861600E39807FFCC
:101AD0009307510EB387B7401307610DB307F700A3
:101AE0009306410DB387D7402322F1040327010158
:101AF0008326410493071000B30CD70063C4E700AA
:101B00006F20801C8327C103B38CFC0083278106D0
:101B100013CCFCFF135CFC4113F9F7BF13690910E8
:101B200033FC8C0123260102232A0102232801020F
:101B30008327C107639407006F1000769307D002D4
:101B4000A303F10C13030000130C1C006FF01F9B88
:101B50001306410E93050B0013850A002320610232
:101B6000232EE1012324F101EF70C005E318050ADB
:101B70008327C10E03230102032FC101832F81009C
:101B800093880B006FF01F9D0326810E0327010130
:101B90009306100023A0A801938717009304160052
:101BA000938C8800E3DCE6329306100023A2D80071
:101BB0002326F10E2324910E93067000E3C6963E71
:101BC0000327C1038326010493841400B387E7002D
:101BD00023A0DC0023A2EC002326F10E2324910E87
:101BE00093067000938C8C00E3C2963E8326010F0F
:101BF000138814009305010A2328D10A8326410F74
:101C00001305010B232EF100232AD10A8326810F0D
:101C1000232401012320010A232CD10A8326C10F8A
:101C20002322010A2324010A232ED10A2326010A92
:101C3000EFD0501B832701010328810093888C007B
:101C40009386F7FF130608008327C101E30C052ADA
:101C500013071D00B387D70023A0EC0023A2DC00EC
:101C60002326F10E2324010F13077000E34A0777A0
:101C700013870C0113862400938C08009308070037
:101C8000832641041307410D23A0EC00B387F6001F
:101C900023A2DC002326F10E2324C10E13077000BB
:101CA000E356C7921306410E93050B0013850A00F5
:101CB000EF605071631405768327C10E93880B0083
:101CC0006FF0DF90930600010327810E63C4960036
:101CD0006F10D002B7360180938E06691309000198
:101CE000930C70006F00C000938404FF635A990442
:101CF000938707011307170023A0D80123A2280107
:101D00002326F10E2324E10E93888800E3DEECFC09
:101D10001306410E93050B0013850A002324D101FD
:101D2000EF60506A631C056E938404FF8327C10E25
:101D30000327810E832E810093880B00E34A99FAD2
:101D4000B38797001307170023A0D80123A2980098
:101D50002326F10E2324E10E93067000E3D0E688DB
:101D60001306410E93050B0013850A00EF60906582
:101D70006316056A8327C10E6FF05F868326C10054
:101D80009377090113874600E39E072C9377090494
:101D9000639407006F10C02D8327C100930C0000CF
:101DA0002326E10083DD07006FF0DF9D8326C1005D
:101DB0009377090113874600E39C0728937709046A
:101DC000639407006F1000278327C1002326E100DA
:101DD000839D070093DCFD4113870C00E3540792B9
:101DE0003337B001B3079041B38CE7401307D002FB
:101DF000A303E10C9306F0FFB30DB041130C0900EF
:101E000013071000E31AD39893061000630CD71041
:101E1000930620006302D72E130D011B1396DC01DD
:101E200093F67D0093DD3D0093860603B36DB60106
:101E300093DC3C00A30FDDFE33E69D0193050D000E
:101E4000130DFDFFE31C06FC93771C006380072E37
:101E500093070003638CF62C9385E5FFA30FFDFE2B
:101E60009307011BB38CB74013090C00138D0500B9
:101E70006FF01F8C8327C100A303010C03AD070083
:101E800093864700E3060D309307F0FF6314F300D9
:101E90006F108010130603009305000013050D005A
:101EA000232ED1002326110123246100EF5000715D
:101EB000032381008328C1008326C101930D0500FF
:101EC000631405006F104056B30CA5418347710C95
:101ED00013CCFCFF135CFC412326D1002326010216
:101EE000232A01022328010233FC8C01930D0000F8
:101EF00013030000E39007866FF04FE00327C10053
:101F0000A303010C130C10008327070013074700DD
:101F10002326E1002306F114930C1000130DC114C5
:101F20006FF08FDCE3940C4E13079000E360B74F23
:101F3000938D0D03A307B11B13090C00930C100024
:101F4000130DF11A6FF0CFFE8344040013694900AA
:101F50006FF00FD39307B00283440400A303F10C86
:101F60006FF00FD283440400136909086FF04FD15A
:101F700083440400930614006394B4016F10D0618D
:101F8000938704FD138406001303000063ECFCCE6A
:101F90008344040093162300338366001313130055
:101FA0003303F300938704FD13041400E3F2FCFEF3
:101FB0006FF04FCD8327C1008344040003AA0700BC
:101FC000938747002326F100635C0ACA330A404125
:101FD000136949006FF0CFCA8344040013691900E4
:101FE0006FF00FCA8347710C83440400639A07C8DB
:101FF00093070002A303F10C6FF08FC8136C090163
:1020000093770C02638A07768327C10013877700D2
:10201000137787FF93078700832D0700832C4700E2
:102020002326F100130710006FF04FF68327C1003D
:102030003787FFFF1347078383AD07002314E10CA5
:1020400093874700373701802326F1009307074F16
:10205000930C0000136C2900232CF10013072000BF
:10206000930480076FF08FF28344040013698900A2
:102070006FF00FC1834404009307C006E386F40C9D
:10208000136909016FF0CFBF8344040093078006F2
:10209000E384F408136909046FF08FBE8326C1003E
:1020A0009377090203A70600938646002326D100F2
:1020B0006398077493770901E39A07629377090499
:1020C000638407006F10C00813790920E3000962D8
:1020D00083274100130D04002300F7006FF04FD356
:1020E000930610006314D7006F109013930620001E
:1020F000130C0900E312D7D2130D011B83278101B2
:1021000093F6FD0093DD4D00B386D70003C60600AD
:102110009396CC01B3EDB60193DC4C00A30FCDFE3A
:10212000B3E69D01130DFDFFE39A06FC9307011B27
:10213000B38CA74113090C006FF08FDF9306500694
:10214000E3D496A48326010F9305010A1305010B1E
:102150002328D10A8326410F232EF10023241101C5
:10216000232AD10A8326810F2320010A2322010A70
:10217000232CD10A8326C10F2324010A2326010A16
:10218000232ED10AEFD00046832881008327C10186
:10219000631C053C0327810EB736018093860652E7
:1021A00023A0D80093871700930610001307170089
:1021B00023A2D8002326F10E2324E10E93067000FB
:1021C00093888800E3C4E6420327C10C83260101FB
:1021D0006350D762032701048326C10393888800D4
:1021E00023ACE8FE0327810EB387D70023AED8FEC9
:1021F000130717002326F10E2324E10E9306700027
:1022000063C4E672032701019304F7FF635090BC97
:10221000930600010327810EE3DA963E930C00013A
:10222000130D70006F00C000938404FFE3D09C3E48
:10223000938707011307170023A0380123A29801F1
:102240002326F10E2324E10E93888800E35EEDFC43
:102250001306410E93050B0013850A00EF609016DC
:10226000631E051A8327C10E0327810E93880B0076
:102270006FF09FFB33088A41635E00B113060001D3
:102280008326810E635C0607130E0001930E700017
:102290006F00C000130808FF63520E079387070101
:1022A0009386160023A0380123A2C8012326F10E2D
:1022B0002324D10E93888800E3DEDEFC1306410E52
:1022C00093050B0013850A00232E010123246100CE
:1022D000EF60500F631405140328C101130E0001B1
:1022E0008327C10E130808FF8326810E0323810074
:1022F00093880B00930E7000E3420EFBB387070137
:102300009386160023A0380123A208012326F10E8C
:102310002324D10E1306700093888800635CD6A630
:102320001306410E93050B0013850A002324610058
:10233000EF6050096314050E032381008327C10E4B
:1023400093880B0033039341635A60A41306000182
:102350008326810E6358660613080001130E700071
:102360006F00C000130303FF635E680493870701D7
:102370009386160023A0380123A208012326F10E1C
:102380002324D10E93888800E35EDEFC1306410E01
:1023900093050B0013850A0023246100EF6090026F
:1023A000631E050603238100130800018327C10E65
:1023B000130303FF8326810E93880B00130E700016
:1023C000E34668FAB38767009386160023A03801B6
:1023D00023A268002326F10E2324D10E13067000D9
:1023E00093888800635CD69A1306410E93050B0010
:1023F00013850A00EF60007D631205028327C10E7A
:1024000093880B006FF08F991306410E93050B0014
:1024100013850A00EF60007B630E059C63840DA0AA
:1024200093850D0013850A00EF1090306FF08F9F99
:10243000130C09006FF05F9D373701801306000110
:102440008326810E930E0769130E0001930270001C
:10245000634806016F004008130808FF635E0E071B
:10246000938707019386160023A0D80123A2C801F1
:102470002326F10E2324D10E93888800E3DED2FCBC
:102480001306410E93050B0013850A002324D10384
:102490002322010323206102232EE1012324F101E1
:1024A000EF604072E31C05F603284102130E0001A1
:1024B0008327C10E130808FF8326810E832E810215
:1024C00003230102032FC101832F810093880B0096
:1024D00093027000E3460EF9B38707019386160056
:1024E00023A0D80123A208012326F10E2324D10E14
:1024F00013067000938888006344D6006FF00F8243
:102500001306410E93050B0013850A002320610278
:10251000232EE1012324F101EF60C06AE31005F0EE
:102520008327C10E03230102032FC101832F8100E2
:1025300093880B006FE09FFE1306410E93050B007E
:1025400013850A00232E61002324E101EF608067D8
:10255000E31605EC8327C10E0323C101032F81007D
:1025600093880B006FF08F828325C10C635CB07879
:1025700003270103832601019304070063C6E632A3
:10258000635690028326810EB387970023A0A8018B
:102590009386160023A298002326F10E2324D10E41
:1025A0001306700093888800E340D63693C6F4FF84
:1025B0000327010393D6F641B3F4D400B304974044
:1025C0006348903E0327010393760940B304ED006E
:1025D000639406448325C10C0327010163C6E5000B
:1025E00093761900E3860634832601040327C1038A
:1025F0001306700023A0D8008326810EB387E7005E
:1026000023A2E800938616002326F10E2324D10E80
:1026100093888800E34CD64C832601013307DD0004
:102620003386B64033079740930C06006354C700C7
:10263000930C0700635690030327810EB38797011D
:1026400023A098001307170023A298012326F10E58
:102650002324E10E9306700093888800E3CCE65EA5
:1026600013C7FCFF1357F74133F7EC00B304E64000
:10267000634490006FE09FF5930600010327810EED
:1026800063D69678930C0001130D70006F00C000A4
:10269000938404FF63DC9C7693870701130717007C
:1026A00023A0380123A298012326F10E2324E10E52
:1026B00093888800E35EEDFC1306410E93050B0042
:1026C00013850A00EF600050E31A05D48327C10E7A
:1026D0000327810E93880B006FF09FFB9375190001
:1026E000639405CC23A2D8002326F10E2324910E57
:1026F000130770006346974E13062600938808015F
:102700006FF00FD8635ED0D6130700016344D70083
:102710006F100068130D70006F000001938606FFB4
:10272000E350D70C138814009387070123A03C01C2
:1027300023A2EC002326F10E2324010F93040800AA
:10274000938C8C00E35C0DFD1306410E93050B008A
:1027500013850A002324D100EF60C046E31005CCA6
:102760008327C10E8324810E83268100938C0B0066
:10277000130700016FF09FFA8326C10093770C01C5
:1027800013874600639C070A93770C04E3840708C9
:102790008327C100930C00002326E10083DD07009E
:1027A000130710006FE09FFE1306410E93050B0008
:1027B00013850A00EF600041E31205C68327C10EAE
:1027C0008324810E938C0B006FF08FBF1306410E94
:1027D00093050B0013850A00EF60C03EE31005C4AB
:1027E0008327C10E8324810E938C0B006FF00FC0E2
:1027F00013771900631407006FE05FDD6FF09F9D92
:1028000083264100130D040093D7F6412320D700FF
:102810002322F7006FE0DFDF832781038344040076
:10282000639407006FE0DFC583C707006394070068
:102830006FE01FC5136909406FE09FC42326E100C4
:1028400083AD0600930C0000130710006FE01FF427
:1028500083AD06002326E10093DCFD4113870C00C5
:102860006FE01FEA83AD0600930C00002326E10011
:102870006FE05FF10327C1008327070013074700BC
:102880002326E10083A5070003A6470083A687004F
:1028900083A7C7002328B10E232AC10E232CD10EF3
:1028A000232EF10E6FE01FFB93840600E34C90CCC7
:1028B0006FF0DFCF130C09006FF08FF4B737018092
:1028C0009387074F232CF100937709026386072C27
:1028D0008327C10013877700137787FF832D0700B5
:1028E000832C4700930787002326F10013771900F4
:1028F000630E070033E79D01630A07001307000317
:102900002304E10CA304910C13692900137CF9BF83
:10291000130720006FE09FE7834414001369092028
:10292000130414006FE0DFB51306410E93050B008E
:1029300013850A00EF600029E31205AE8327C10E5C
:1029400093880B006FF01F8C8344140013690902F5
:10295000130414006FE0DFB2B7370180938747504C
:10296000232CF1006FF05FF69305000413850A0035
:10297000EF4040492320AB002328AB00631405003F
:102980006F10C04393070004232AFB006FE05FA28F
:1029900093076000930C030063E867783737018082
:1029A000138C0C002326D100130D87516FE0DFB389
:1029B000130600018326810E635A966E930C000164
:1029C000130870006F00C000938404FF63D09C6EF6
:1029D000938707019386160023A0380123A298014C
:1029E0002326F10E2324D10E93888800E35ED8FCC1
:1029F0001306410E93050B0013850A00EF60801C3F
:102A0000E31E05A08327C10E8326810E93880B0049
:102A1000130870006FF05FFB03270101130E7000B5
:102A2000130800013307ED002324E10003274103CD
:102A3000630E070A0327C102631E070A03278103E7
:102A40001307F7FF232CE102032741031307F7FFC6
:102A5000232AE1028326C104032781049388880086
:102A600023ACD8FE8326810EB387E70023AEE8FEB1
:102A7000938616002326F10E2324D10E634EDE1218
:102A8000032781038346070003278100938C0600F8
:102A9000330697406354D600930C060063589003A6
:102AA0008326810EB387970123A098009386160092
:102AB00023A298012326F10E2324D10E634CDE3687
:102AC00003278103938888008346070013C6FCFF11
:102AD0001356F641B3FCCC00B38C9641634490038B
:102AE000B384D40003274103E31607F40327C1028C
:102AF000630007720327C1021307F7FF2326E102D1
:102B00006FF05FF58326810E634898016F00C00562
:102B1000938C0CFF635A98059387070193861600E0
:102B200023A0380123A208012326F10E2324D10E6D
:102B300093888800E35EDEFC1306410E93050B00CC
:102B400013850A00EF600008E31A058C13080001E2
:102B5000938C0CFF8327C10E8326810E93880B0074
:102B6000130E7000E34A98FBB38797019386160013
:102B700023A0380123A298012326F10E2324D10E8D
:102B80006346DE720327810393888800834607002B
:102B9000B384D4006FF01FF58326C1009377090139
:102BA000138746006386072283AD0600930C00005E
:102BB0002326E1006FF09FD31306410E93050B000F
:102BC00013850A00EF600000E31A05848327C10E15
:102BD00093880B0013080001130E70006FF05FEA7A
:102BE0001306410E93050B0013850A00EF50907DEC
:102BF000E31605820326810E8327C10E9308411137
:102C000013061600938C0B006FF08F8713790C401E
:102C100023280100130D011B6F0040031306A000C1
:102C20009306000013850D0093850C00232E1101DF
:102C300023246100EFB04010032381008328C101E9
:102C400063880C4A930D0500938C05001306A000C1
:102C50009306000013850D0093850C00232E1101AF
:102C600023246100EFB08050832701011305050381
:102C7000A30FADFE938717002328F10003238100E3
:102C80008328C101130DFDFFE30A09F8032781031F
:102C900083460700E394D7F81307F00FE380E7F8C3
:102CA00063960C009307900063F2B7C983278104F1
:102CB0008325C104232E1101330DFD401386070027
:102CC00013050D0023246100EF5050658327810315
:102CD0001306A0009306000003CE170013850D0015
:102CE00093850C00333EC001B387C701232CF1024A
:102CF000EFB08004032381008328C1012328010051
:102D00006FF05FF48326810E37360180130606527A
:102D100023A0C8009387170013061000938616009F
:102D200023A2C8002326F10E2324D10E130670001F
:102D300093888800634CD6066392051C0327010123
:102D400093761900B3E6E600639406006FE01F88EF
:102D5000832601040327C1031306700023A0D800B3
:102D60008326810EB387E70023A2E800938616002E
:102D70002326F10E2324D10E6342D6469388880081
:102D8000032701019386160023A0A801B387E7005B
:102D900023A2E8002326F10E2324D10E130770008E
:102DA0006344D7006FE05F826FE0DFEF1306410EF0
:102DB00093050B0013850A00EF50D060631005E601
:102DC0008325C10C8327C10E93880B006FF0DFF6BB
:102DD00093770904638007288327C100930C0000C0
:102DE0002326E10083DD07006FF05FB01306410E7C
:102DF00093050B0013850A00EF50D05C631005E2C9
:102E00008327C10E93880B006FF00FBC23A03801FD
:102E100023A29800B3879700130717002326F10E0B
:102E20002324E10E9306700063C4E6006FE0CFF93F
:102E30006FE05FE71306410E93050B0013850A0050
:102E4000EF505058631C05DC8327810393880B00E7
:102E50001308000183C60700130E70008327C10EFC
:102E60006FF0DFC68327010F9305010A1305010BDD
:102E70002328F10A8327410F232411012320010A6B
:102E8000232AF10A8327810F2322010A2324010A1E
:102E9000232CF10A8327C10F2326010A232EF10ACE
:102EA000EFC0D01B83288100634C05428347710C1F
:102EB000130770046354972437370180130D474E6E
:102EC00023260102232A0102232801021379F9F79C
:102ED000130C3000930D0000930C3000130300001E
:102EE000638407006FE01F876FE04FE18327410095
:102EF000130D04002320F7006FE08FF183260104F7
:102F00000327C1031306700023A0D8008326810E77
:102F1000B387E70023A2E800938616002326F10E6C
:102F20002324D10E93888800634AD62AE3DA05E485
:102F3000130600FFB304B040E3D6C528930C00018C
:102F4000130870006F00C000938404FFE3DC9C262C
:102F5000938707019386160023A0380123A29801C6
:102F60002326F10E2324D10E93888800E35ED8FC3B
:102F70001306410E93050B0013850A00EF50904491
:102F8000631E05C88327C10E8326810E93880B001C
:102F9000130870006FF05FFB13050D00232411016F
:102FA0002326D100EF50D02E8347710C134CF5FF30
:102FB000135CFC4123260102232A0102232801027B
:102FC00083288100930C0500337C8501930D00005C
:102FD00013030000638407006FE0CFF76FE00FD2A8
:102FE0001386140013878C00B387D70023A2DC005C
:102FF00023A03C012326F10E2324C10E930670006A
:10300000E3C0C6BE1306160093088700930C0700A2
:103010006FE01FC793770C20638407188327C100D4
:10302000930C00002326E10083CD07001307100056
:103030006FE0CFF593770920638807148327C100D9
:103040002326E100838D070093DCFD4113870C00EC
:103050006FE00FEB93770920638E07108327C10081
:10306000930C00002326E10083CD07006FF01F883A
:10307000937709206386070E8327C100930C000015
:103080002326E10083CD07006FE0CFEF8327C10F38
:1030900063C007148347710C13077004635297428F
:1030A00037370180130DC74E6FF09FE1B38797004C
:1030B0009386160023A0380123A298002326F10E40
:1030C0002324D10E1306700093888800635CD6CE4B
:1030D0001306410E93050B0013850A00EF50902E46
:1030E000631E05B28327C10E93880B006FF08FCD4E
:1030F00093079000E3E8B7B56FF04F83373701804F
:10310000130D074E6FF0DFDB1306410E93050B0026
:1031100013850A00EF50102B631205B08327C10EF0
:1031200093880B006FF08FC8930C60006FF01F87BF
:10313000832601013307DD003386B6403303974011
:10314000930C0600635EC3D0930C03006FF04FD165
:1031500083274100130D04002310F7006FE04FCBCD
:103160008327C100930C00002326E10083AD0700F4
:103170006FE04FE18327C100930C00002326E1009C
:1031800083AD07006FF08FF68327C1002326E1008F
:1031900083AD070093DCFD4113870C006FE04FD631
:1031A0008327C100930C00002326E10083AD0700B4
:1031B000130710006FE08FDD1306410E93050B001F
:1031C00013850A00EF5010208357CB006FE0CFC566
:1031D0009307D002A303F10C6FF01FEC1306410E0E
:1031E00093050B0013850A00EF50D01D631805A24C
:1031F0008325C10C8327C10E8326810E93880B0083
:10320000E3D005B86FF0DFD2130360006FE04FEB3F
:1032100003270101B306ED0063FE96BA938406000E
:103220006FF04FBB032701039307D0FF6344F70000
:10323000635AE3009384E4FF93F7F4FD232CF10633
:103240006FE04FFD83270101032701036340F72847
:1032500083278106930C070093F717006386070006
:103260008327C103B30CF7008327810693F7074038
:103270006386070083270103E340F00613CCFCFFBD
:10328000135CFC4133FC8C0193047006232601027D
:10329000232A01026FE0DF898347710C13030000CA
:1032A000638407006FE00FCB6FE04FA51306410E5C
:1032B00093050B0013850A00EF50D010631005969C
:1032C0008327810393880B001308000183C607003E
:1032D000130E70008327C10EB384D4006FF09F805B
:1032E0009307D002A303F10C6FF09FBC1306410EAD
:1032F00093050B0013850A00EF50D00C6310059264
:103300008325C10C8327C10E93880B006FF0CFB0CB
:10331000130C010B930603001308C10D9307010D55
:103320001307C10C1306300093050C0013850A0027
:1033300023241103232261022328D10B2320D1034C
:10334000232AE10B232EE101232CF10B2328F10189
:10335000232EC10B2324C101EF204076032E8100D0
:10336000832F0101032FC101832E01020323410298
:1033700083288102130D05009307600433086D0054
:10338000639CFC6883460D0093070003E388F614F2
:10339000930C010A8327C10C3308F8006FE0CFDDDE
:1033A000130C010B9307010D930603001308C10DC5
:1033B0001307C10C1306200093050C0013850A00A7
:1033C000232261022328D10B2320D103232AE10BDE
:1033D000232EE101232CF10B2328F101232EC10B15
:1033E0002324C101EF20806D93077004032E810018
:1033F000832F0101032FC101832E01020323410208
:1034000083288102130D0500E398FCF683278106CB
:1034100093F71700639C075E130770048327C10DA1
:10342000232CE1066FE00FDC8347710C2326D100CB
:1034300023260102232A010223280102130C030080
:10344000930C030013030000638407006FE08FB048
:103450006FE0CF8A1306410E93050B0013850A0017
:10346000EF504076630405006FE05FFB8324C10CDE
:10347000032701018327C10E93880B003306974071
:103480006FF00F9E832781060327010393F7170030
:10349000B3E76700E354E00C6398076C832C0103E7
:1034A000930460068327810693F7074063980762B9
:1034B00013CCFCFF135CFC4133FC8C016FF01FDD6F
:1034C00037370180130D874E6FF09F9F83270101CF
:1034D0000327C10393047006B38CE700832701031D
:1034E000E342F0FCB38CFC40938C1C0013CCFCFF3B
:1034F000135CFC4133FC8C016FF05FD9B73601805F
:10350000938E06696FE0DF83930700032304F10CB9
:103510009307800513672900A304F10C2324E10617
:1035200093073006930D0000130DC11463CE67445A
:10353000032EC10F93FCF4FD232C9107232E0106CB
:10354000832E010F032F410F832F810F1369291041
:1035500063420E3C930710066388F46293071004DD
:103560006384F4006FE08FB8130C010B13050C009B
:1035700023261103232461022328D10B232AE10BE4
:10358000232CF10B232EC10BEFF0406E1306C10C60
:10359000EF50C025138605009305050013050C00A8
:1035A000EFF0404A93070109938507002324F100B7
:1035B0008327010B930C010A130601082328F10845
:1035C0008327410B13850C002326C106232AF1080B
:1035D0008327810B2320010823220108232CF108D3
:1035E0008327C10B23240108232EF108B707FC3FD2
:1035F0002326F108EFC0403B0328010A032E410AAD
:10360000832E810A032FC10A93850C0013050C0039
:103610002328010B23220103232AC10B2320C103EA
:10362000232CD10B232ED101232EE10B2328E101E2
:103630002320010A2322010A2324010A2326010A46
:10364000EFB0507A032F0101832EC101032E010236
:1036500003284102032381028328C1026316050067
:10366000930710002326F10CB7370180938747504A
:103670002322F1069306F3FF93070D006F00400924
:1036800093850C0013050C002320C106232EF105A1
:10369000232C5104232A71042328F104232A110323
:1036A000232861022328710A23267102232A510A42
:1036B00023245102232CF10B2322F103232EC10AD0
:1036C0002320C1022320010A2322010A2324010A04
:1036D0002326010AEFB010718326C101032F0102D6
:1036E000832E4102032E81020328C102032301031A
:1036F0008328410383270105832341058322810514
:10370000832FC105032601069386F6FF630E05107D
:103710000326810093850C00232AF10213050C0077
:10372000B70703402328D10423281103232661026D
:10373000232EF1082326E10B2320010B2322C10BAA
:103740002324D10B23280108232A0108232C010854
:10375000EFC08025832E010B032E410B0328810B24
:103760000326C10B13050C002324D1032322C1031C
:1037700023200103232EC100EFE0107D93050500F7
:103780002328A10013050C00EFF0C0160326C10189
:10379000832E8102032E4102232EC1080326010B32
:1037A00003280102832581002320C1080326410B41
:1037B00013850C002328D1092322C1080326810B7D
:1037C000232AC109232C01092324C1080326C10B84
:1037D0002326C1080326C106EFD0804A03274106ED
:1037E00083270101832601058323010A3306F7009D
:1037F00083450600832741038322410A832F810AE0
:103800000326C10A232AF1062380B7002328D10604
:103810001307F0FF232ED1000323C10283280103E5
:1038200093871700E39EE6E4B706FE3F93850C00FE
:1038300013050C002320F102232E11012324610023
:103840002328710A23287102232A510A23265102B0
:10385000232CF10B2324F103232EC10A2322C102BE
:103860002320010A2322010A2324010A2326D10A44
:10387000EFB0106A032381008328C101832701026E
:103880006344A00A832301038322C102832F8102A0
:1038900003264102B706FE3F93850C0013050C007A
:1038A0002328710A232A510A232CF10B232EC10A43
:1038B0002320010A2322010A2324010A2326D10AF4
:1038C000EFB05052032381008328C10183270102F6
:1038D0006318050003270101937617006396060419
:1038E000032701071306000393061700B386D700CA
:1038F000635407006FE00F8F93871700A38FC7FEF5
:10390000E39CD7FE6FE00F8E23242107930D000068
:1039100013890200B707008033CEC7019307D00296
:10392000232EF1066FF01FC303274107938607007C
:10393000232EE10C0327410603C6F7FF8345F7005A
:103940006310B60213050003A38FA6FE8326C10DE4
:103950001386F6FF232EC10C03C6F6FFE386C5FED1
:10396000930516001305900393F5F50F6306A60063
:10397000A38FB6FE6FE00F87032741068345A7009C
:10398000A38FB6FE6FE00F869305130013850A0020
:103990002328110123246100EF30C0460323810056
:1039A00083280101130D050063040542930D0500F2
:1039B0006FF01FB8930700032304F10C93078007EF
:1039C0006FF05FB5B38797009386160023A0380188
:1039D00023A298002326F10E2324D10E1306700093
:1039E000635ED6B81306410E93050B0013850A00DB
:1039F000EF50401D630405006FE05FA28327C10EF6
:103A00008326810E93880B006FF08FB793077004A5
:103A100033086D00232CF106930C010A6FD0DFF5FB
:103A2000130C09006FE0CFD09307F0FF2322F100C1
:103A30006FD05FC06314030013031000032EC10F87
:103A4000832E010F032F410F832F810F93620910E3
:103A5000E34C0EEA130C010B930603001308C10D8F
:103A60009307010D1307C10C1306200093050C00EA
:103A700013850A0023265102232411032322610205
:103A80002328D10B2320D103232AE10B232EE1018C
:103A9000232CF10B2328F101232EC10B2324C10178
:103AA000EF20C0018322C10223242107032E8100BD
:103AB000832F0101032FC101832E01020323410241
:103AC00083288102130D050013890200930D000065
:103AD000232E01066FF09F939304700683278103C2
:103AE0009306F00F2326010283C70700232A010251
:103AF0006388D7040327010363D4E704B307F740BF
:103B0000032781032328F10283471700638E0700F0
:103B10000326410313071700232CE10213061600A6
:103B2000232AC1026FF0DFFC0327C1028327810330
:103B30001307170083C707002326E1026FF05FFB1E
:103B40000327C10283274103B387E70003278104CA
:103B5000B387E702B38C970113CCFCFF135CFC41E5
:103B600033FC8C016FD0DFFC8327C1039304600614
:103B7000B30CF700B38C6C006FF0DF92930D000074
:103B8000138907006FF01FD9130C010B13050C00EC
:103B900023261103232461022328D10B232AE10BBE
:103BA000232CF10B232EC10BEFF0400C1306C10C9C
:103BB000EF40D043138605009305050013050C0064
:103BC000EFE0506893070109938507002324F10073
:103BD0008327010B930C010A130601082328F1081F
:103BE0008327410B13850C002326C106232AF108E5
:103BF0008327810B2320010823220108232CF108AD
:103C00008327C10B23240108232EF108B707FC3FAB
:103C10002326F108EFB050590328010A032E410A68
:103C2000832E810A032FC10A93850C0013050C0013
:103C30002328010B23220103232AC10B2320C103C4
:103C4000232CD10B232ED101232EE10B2328E101BC
:103C50002320010A2322010A2324010A2326010A20
:103C6000EFB05018032F0101832EC101032E010272
:103C700003284102032381028328C1026316050041
:103C8000930710002326F10CB73701809387074F65
:103C90002322F1066FF01F9E9306610D6318060044
:103CA00093060003230BD10C9306710D1307011B20
:103CB000938707033386E6402380F6009307D60DEB
:103CC0002322F1046FD09FE28327810693F7170028
:103CD000639407006FD09FE36FD0DFE2930C010A7B
:103CE00093850C0013050C002326010323241103E4
:103CF000232261022328D10B2320D103232AE10BA5
:103D0000232EE101232CF10B2328F101232EC10BDB
:103D10002324C1012320010A2322010A2324010AAA
:103D20002326010AEFB0100C032E8100832F01011E
:103D3000032FC101832E0102032341028328810244
:103D40000328C102630805E493071000B3876740A6
:103D50002326F10C3308F8006FD01FC2639A0700C6
:103D6000130C100093046006930C10006FF00FD238
:103D70008327C10393046006938C1700B38C6C00F7
:103D800013CCFCFF135CFC4133FC8C016FF00FD0B3
:103D9000138708006FF04FA58327C10003A3070016
:103DA00093874700635403001303F0FF8344140018
:103DB0002326F100138406006FD08FEC9307C00018
:103DC00023A0FA009307F0FF2322F1006FD09F8613
:103DD0008357CB0013E70704930707002316EB0074
:103DE0006FD09F84930720002322F1046FD01FD04F
:103DF000130101FE23263101B7590180232C8100D4
:103E0000232A91002328210123244101232E11007C
:103E1000138A0500130905009389094EEF305007F6
:103E200003A78900B71700001384F7FE8324470017
:103E30003304444193F4C4FF330494001354C40086
:103E40001304F4FF1314C400634EF4009305000040
:103E500013050900EF40502483A78900B38797001A
:103E60006308F50213050900EF30D0028320C10179
:103E70000324810183244101032901018329C10015
:103E8000032A81001305000013010102678000006E
:103E9000B305804013050900EF4010209307F0FFA1
:103EA000630AF504B7670180938707AD03A707008E
:103EB00083A68900B384844093E4140033048740CC
:103EC0001305090023A2960023A08700EF30807C11
:103ED0008320C101032481018324410103290101BD
:103EE0008329C100032A8100130510001301010278
:103EF000678000009305000013050900EF40D0190A
:103F000003A789009306F000B307E540E3DCF6F46D
:103F1000B766018083A686A793E717002322F700E0
:103F20003305D540B766018023A8A6AC6FF09FF398
:103F3000638A0512130101FF2324810023229100CB
:103F4000138405009304050023261100EF3040740C
:103F50000328C4FF130784FFB75501809377E8FF58
:103F60003306F7009385054E8326460003A585009A
:103F700093F6C6FF630AC51A2322D60013781800E9
:103F80003305D6006310080A032384FF0328450085
:103F90003755018033076740832887001305854E16
:103FA000B3876700137818006380A8140323C70041
:103FB00023A66800232413016304081E93E6170058
:103FC0002322D7002320F6009306F01F63E8F60AA9
:103FD00093F687FF9386860003A54500B386D50038
:103FE00003A6060013D8570093071000B3970701E4
:103FF000B3E7A700138586FF2326A7002324C70065
:1040000023A2F50023A0E6002326E6000324810076
:104010008320C100138504008324410013010101A2
:104020006F3040670325450013751500631E0502B8
:1040300037550180B387D7001305854E8326860048
:1040400093E817003308F7006388A6160326C60016
:1040500023A6C6002324D600232217012320F8001C
:104060006FF09FF66780000093E61700232ED4FEC2
:104070002320F6009306F01FE3FCF6F493D6970096
:1040800013064000636CD60E93D667001388960320
:104090001386860313183800338805018326080029
:1040A000130888FF6308D81203A646001376C6FFDC
:1040B00063F6C70083A68600E318D8FE03A8C600EF
:1040C000232607012324D700032481008320C10075
:1040D0002324E800138504008324410023A6E6007E
:1040E000130101016F30005B631608148325C600BD
:1040F00003268600B387F600032481002326B6003A
:1041000023A4C50093E617008320C1002322D70013
:10411000138504003307F700832441002320F700B0
:10412000130101016F30005713781800B387D700CF
:1041300063100802032584FF3307A7408326C700C6
:1041400003268700B387A7002326D60023A4C60032
:10415000B766018013E6170083A6C6A72322C7000F
:1041600023A4E500E3E4D7EAB767018083A587A825
:1041700013850400EFF0DFC76FF05FE9130640011D
:104180006374D602130640056364D60693D6C7004F
:104190001388F6061386E606131838006FF0DFEF73
:1041A000B387D7006FF09FE91388C6051386B6055D
:1041B000131838006FF05FEE23AAE50023A8E5008E
:1041C0002326A7002324A700232217012320F80079
:1041D0006FF0DFE303A54500135626409307100058
:1041E0003396C7003366A60023A2C5006FF05FEDCB
:1041F00013064015636CD60093D6F7001388860724
:1042000013867607131838006FF01FE91306405520
:10421000636CD60093D627011388D6071386C6078A
:10422000131838006FF05FE71308803F1306E007AC
:104230006FF09FE693E617002322D7002320F600B5
:104240006FF0DFDC93064500930700001305A5011E
:104250003788FFFF6F00C001939717002390E60097
:10426000939707019386260093D70701630ED50223
:1042700003D70600137617006304060093E71700C0
:104280001357170013F62700B3650701E30606FC72
:10429000939717002390B600939707019386260003
:1042A00093D70701E316D5FC6780000093068501CC
:1042B00013070000130525006F00C0011317170036
:1042C0002390F600131707019386E6FF13570701A3
:1042D0006304D50483D706001396070113560641DD
:1042E000939717006354060013671700939707010D
:1042F00093D707011376270093E51700E30006FC28
:10430000131717002390B600131707019386E6FFD3
:1043100013570701E310D5FC67800000130101FE6D
:10432000370E0100231D0100231E01009385850126
:104330009307C10113088100130EFEFF03D7050088
:104340009387E7FF9385E5FF63180702239F07FE26
:10435000E39607FF130646009306E10103D7070023
:104360009387270013062600231FE6FEE398D7FE57
:1043700013010102678000003307A70283D82700DA
:1043800003D30700B376C701B3861601135707019D
:1043900093D80601330767003307170193580701C5
:1043A0002391D7002390E700239F17FFE39807F995
:1043B0006FF05FFA130725018357050013052500E9
:1043C00063980700E31AE5FE13050000678000000C
:1043D0001305100067800000130101FF23229100E4
:1043E00083542501232481002326110093C7F4FF61
:1043F000139717011304050063160700EFF09FFBE6
:1044000063180500B787FFFFB3C4F40023199400B5
:104410008320C10003248100832441001301010192
:1044200067800000130101FF23248100035425014C
:10443000232611009347F4FF13971701631A07000F
:10444000EFF05FF793070500130500006394070082
:104450001355F4008320C1000324810013010101DE
:104460006780000083572501130101FD2324810289
:1044700093D7F70023229102232611022320210340
:10448000232E3101B307F0402390F5008357250117
:10449000378700001307F7FFB377F7002391F50084
:1044A00093040500130405016382E7049387650004
:1044B000239205001305E5FF035704001304E4FFEE
:1044C00093872700239FE7FEE31885FE239C0500C2
:1044D0008320C102032481028324410203290102B3
:1044E0008329C101130101036780000003572501DF
:1044F0001389450033F7E700631CF7022326B10058
:10450000EFF05FEB8325C10063040502938765002C
:10451000239205001385C4FF035704001304E4FF2E
:1045200093872700239FE7FEE31885FE6FF05FFA6D
:104530009389A50113092900231F09FEE39C29FF84
:104540008320C10203248102832441020329010242
:104550008329C101130101036780000083572501EE
:10456000130101FB2324810493C7F7FF2322910445
:1045700023261104139717019304050013840500E3
:1045800063160700EFF01FE3631205088357240149
:1045900093C7F7FF1397170163040706930581007C
:1045A00013850400EFF01FEC93054102130504008E
:1045B000EFF05FEB8355810003554102630CB504B6
:1045C0009307A100130761021306010283D60700B7
:1045D00093872700639A060883560700130727006E
:1045E00063940608E394C7FE130500008320C1040A
:1045F0000324810483244104130101056780000022
:1046000013050400EFF01FDBE30A05F81305E0FFD4
:104610006FF0DFFD133515000356A10083566102CC
:104620003305A0401307A10093076102137525000D
:104630001305F5FF9305C103938727001307270090
:10464000631ED600E382B7FA0356070083D607003D
:104650001307270093872700E306D6FEE3E8C6F892
:104660003305A0406FF09FF813051000E38005F8B4
:104670001305F0FF6FF09FF7130101FF23261100D0
:10468000EFF05FD38320C100133515001301010142
:1046900067800000130101FE232C8100232A910072
:1046A000232E1100232821012326310193840500A4
:1046B0001304050063C4050A9307F0001386050080
:1046C00013054500930684019305F00063D4970217
:1046D0009307050003D7270093872700239FE7FE52
:1046E000E39AD7FE231C0400130606FFE3C2C5FEAF
:1046F00093F4F4009307700063D8970213078401C2
:104700009305240093070000835607001307E7FF73
:1047100013968600B3E7C7002311F70093D78600EE
:10472000E314B7FE938484FF638A04009384F4FF48
:1047300013050400EFF09FB7E39A04FE1305000091
:104740008320C10103248101832441010329010144
:104750008329C1001301010267800000930710FF45
:104760003309B04063DCF51293058501930900001D
:10477000930645001306F000035784019387050054
:10478000B3E9E90003D7E7FF9387E7FF2391E70049
:10479000E39AD7FE23120400130909FFE34E26FD16
:1047A000930700FF130710FFB3879740130900001A
:1047B00063C4E40A3309F9009307700063D6270540
:1047C0009399090193D90941834784019305A40171
:1047D000B3E9F9009399090193D9090193070000FE
:1047E00003D60600938626001357860033E7E700BA
:1047F0009317860093970701239FE6FE93D707013F
:10480000E390B6FE130989FF630C09068357840100
:104810001309F9FF1305040093F71700B3E93701F3
:10482000EFF05FA2E31409FE9397090193D70741C4
:104830006390070413950901135505018320C101F5
:104840000324810183244101032901018329C1003B
:10485000130101026780000013F907FF33092041AB
:104860003309F90093077000E3D027FB6FF05FF581
:104870009309100013950901135505016FF01FFCF2
:1048800013850900639809001315050113550501E7
:104890006FF01FEB130510006FF01FFF930790FFE1
:1048A00093090000E3D4F5F6930644006FF0DFF1BE
:1048B00083574500130101FF232291002326110095
:1048C000232481002320210193040500639C070C0D
:1048D00003576500130400009317070193D707419E
:1048E00063C4070A9306A5011306000A63180702AA
:1048F000938764006F00800003D707009387270029
:10490000239EE7FEE39AF6FE239C040013040401B1
:10491000630CC40603D76400E30C07FC937707F02D
:104920006390070413858401938524009307000096
:1049300013070500835607001307E7FF1396860049
:10494000B3E7C7002311F70093D78600E394E5FE91
:1049500003D7640013048400937707F0E38807FC0F
:104960001309000A6F00400113041400EFF01F94B4
:10497000634C890003D764001317070113570741DD
:1049800013850400E35207FE8320C10013050400D1
:104990000324810083244100032901001301010144
:1049A0006780000013F707F013040000631007048A
:1049B0001309F0F66F0040011304F4FFEFF09F8835
:1049C000E30424FD83D7440013850400E39607FE27
:1049D0008320C100130504000324810083244100C7
:1049E00003290100130101016780000093064500BF
:1049F0009305A501130700006F00800083D7060010
:104A000013D687003367C700939787002390E6008B
:104A1000139707019386260013570701E390B6FE0C
:104A200083D74400130480FF6FF09FF8130101FE49
:104A3000232C8100232A91002328210123263101E0
:104A40002324410123225101138906009384070086
:104A5000232E11001304050093890500130A060094
:104A6000930A0700EFF0DFE4930700093309A94038
:104A700063DCA716B78700009387E7FF63DA271F79
:104A800063840A1C03A5440083A70400630AF50697
:104A90001387A4019387440313072700231F07FEEE
:104AA000E31CF7FE93078003630CF53263D0A7166F
:104AB00093070004630CF52E930710076318F53471
:104AC000B78700409387F7FF1307A00023AAF400DD
:104AD000B787FFFF23A4E400239CF40023A6E4008F
:104AE0009307A000378700009387870093971700EC
:104AF000B387F4002395E70023A0A4006358201B8C
:104B000083A5840083D744011308F0081396150089
:104B10003306C40003570600B376F700634AA802C1
:104B20001308B0006346B80293070600930584019A
:104B300003D727006304070093E6160023910700BC
:104B400093872700E396F5FE0357060083D74401B9
:104B500093C7F7FFB3F7E7002310F60083D764018C
:104B600033F7D700630007046384D71A138624033E
:104B7000930684019384C401130700008357060041
:104B800083D506009386E6FF1306E6FFB387B700DA
:104B9000B387E70013D707012391F60013771700B7
:104BA000E31E96FC6358201983574400639E071246
:104BB000B7870000231C04009387E7FF63C8270919
:104BC000231124018320C101032481018324410195
:104BD000032901018329C100032A8100832A41009E
:104BE00013010102678000006354090E930700F768
:104BF000635CF908930724001304A401938727003A
:104C0000239F07FEE39C87FE6FF0DFFB9307800185
:104C10006308F51693075003631AF51E3717000053
:104C2000B7070004930660009387F77F1307078098
:104C300023AAF40023A4D400239CE40023A6D400D8
:104C4000930760006FF05FEA231C0400B787FFFF43
:104C500093C7F7FF2311F400930744001304840162
:104C60002390070093872700E31CF4FE6FF09FF565
:104C7000930724001304A40193872700239F07FEB2
:104C8000E39C87FE6FF01FF49305090013050400F1
:104C9000EFF05FA06304050093091000638C0A0C19
:104CA00003A5440083A70400E314F5DE930700097D
:104CB0006304F50A835784011305040093F7170072
:104CC000B3E9F900EFF00FD803A544006FF05FE3FC
:104CD000E3800AEE03A5440083A70400E31AF5DA93
:104CE000E34020E36FF09FFC13050400EFF08FD545
:104CF000B787000013091900231C04009387E7FFFE
:104D0000E3C627F5E35E09EA231104006FF09FEB89
:104D10006394090C83A7C40003D7840193971700F9
:104D2000B307F40083D70700B3F7E700E39007E485
:104D3000E34C20E7930700096306F5001305040020
:104D4000EFF0CFD683574400E39007FA231C04000A
:104D5000E34C09FA6FF0DFE603A6840083D7440131
:104D6000131616003306C40003570600B3F6E70017
:104D70006FF01FDE231C0400231104006FF09FE47A
:104D8000B70780009387F70F1307400023AAF400AA
:104D90009307001023A4E400239CF40023A6E4005E
:104DA00093074000130700106FF01FD493077000A3
:104DB00023A4F400B70701809387F7FF23AAF40028
:104DC00093071000239CF4009307600023A6F400CF
:104DD000130710006FF05FD1E30A0AD86FF09FDC71
:104DE000B70780009387F70F1307600023AAF4002A
:104DF0009307001023A4E400239CF40023A6E400FE
:104E000093076000130700106FF01FCE9307C000D8
:104E100023A4F400B70701809387F7FF23AAF400C7
:104E200093071000239CF4009307B00023A6F4001E
:104E3000130710006FF05FCB130101FD23229102D5
:104E4000232E310193840500835925002326110266
:104E50002324810223202103232C4101130906006E
:104E6000232A510123286101232671012324810172
:104E7000232291012320A101130A0500EFF05FA373
:104E800003D424009307050013850400B389F94077
:104E9000930A4903EFF0DFA13304A4401307E904A8
:104EA00093870A0093872700239F07FEE39CE7FE72
:104EB000634A3409930B4A00138B44009389F9FF2A
:104EC000930CAA01138C240013070B0093870B008B
:104ED00003D6070083560700938727001307270090
:104EE000631AD60AE39697FF13068A011387840193
:104EF0009306000083570700835506001307E7FF5A
:104F0000B387D740B387B74093D607012311F70083
:104F100093F616001306E6FFE31EECFC130D1000DB
:104F200013850A00EFF08FB88357C9041304F4FF08
:104F300013850400336DFD002316A905EFF00FB7AC
:104F4000E31434F993060400032481028320C10290
:104F50008329C101032A8101832A4101032B010115
:104F6000832BC100032C8100832C4100032D010001
:104F700093070900138504000329010283244102D9
:104F8000130700001306000093050000130101033E
:104F90006FF0DFA9130D0000E3E4C6F86FF0DFF453
:104FA0000357050083572500630607003787000075
:104FB000B3E7E7002399F50003572500B787000002
:104FC0009387F7FF6304F702930765009385050154
:104FD0001305850103D70700938727009385E5FF15
:104FE0002391E500E398A7FE678000009307650022
:104FF0001305A50103D7070093872700631A07024B
:10500000E39AA7FE1387250193870500938727005E
:10501000239F07FEE31CF7FE83D725013787000097
:105020001307F7FFB3E7E7002399F5006780000057
:10503000138705019387050093872700239F07FEA9
:10504000E31CF7FEB7C7FF7F23A8F50067800000C9
:10505000130101F723286107035B2501B7870000CF
:105060009387F7FF232C410733FA6701131A0A01CC
:10507000232481082322910823202109232E31078C
:1050800023261108232A5107232671072324810789
:1050900023229107135A0A0193040500138905007E
:1050A00013040600938906006312FA10EFF08FB024
:1050B000631A0528835A2901B3775A016382472B63
:1050C00013850400EFF04FDB630E052EB73501802A
:1050D0009385856D13050900EFF04FC8630605360B
:1050E000835A2901B78700009387F7FFB3FA570166
:1050F000939A0A0193DA0A016394FA2C13050900C2
:10510000EFF08FD76310053283D72401B3F7FA008D
:105110006398570B13850400EFF00FD66318050052
:1051200013050900EFF04FD5630C05081385040043
:10513000EFF04FAF9304050013050900EFF08FAEB9
:10514000B384A440B33490009394F40023199400E2
:10515000130724019307040093872700239F07FE6A
:10516000E31CF7FE83572401378700001307F7FF7E
:10517000B3E7E7002319F4008320C1080324810862
:1051800083244108032901088329C107032A8107D1
:10519000832A4107032B0107832BC106032C8106B9
:1051A000832C4106130101096780000083DA250181
:1051B00033F757011317070113570701630AF70461
:1051C000138504009305C100EFF0CFA91305090072
:1051D00093058102EFF00FA98354E1000359A10266
:1051E000639C040493070101930641026388D7205E
:1051F00003D7070093872700E30A07FE1305C100C2
:10520000EFF00FEB0357A102B304A0406F000003BF
:1052100013850500EFF00F9AE30605EC130749012B
:10522000835709001309290013042400231FF4FEE7
:10523000E318E9FE6FF05FF413070900930A090011
:105240009307C10293060104631207026382F61CEE
:1052500003D7070093872700E30A07FE130581029F
:10526000EFF00FE50357A102B30AA940835781026B
:10527000138C8903239BE902239AF9021387E9041B
:1052800093070C002390070093872700E31CF7FE89
:10529000138AC904930B000013094102930C010106
:1052A000130B6104035509001309E9FF6318050C8A
:1052B00003D7C90493070A00B3EBEB0003D7E7FF5A
:1052C0009387E7FF2391E700E39A87FF239C090276
:1052D000E31A99FD1387490393078102930521047B
:1052E000035607009387270013072700239FC7FE55
:1052F000E398F5FEB7C6FFFFB384540193862600FA
:1053000093850B001305810293870900130700049E
:10531000B386D40013060000EFF04FF1035781026B
:105320008357C1009305040013058102B387E7404A
:10533000B337F000B307F0402314F102EFF05FC67B
:105340006FF09FE31387440183D704009384240004
:1053500013042400231FF4FEE398E4FE6FF0DFE162
:1053600013050900EFF00F85E31A05EA1385040021
:10537000EFF08FB0E30805D66FF05FD51306410458
:1053800093058102EFE09FF993050A0013060000E0
:105390001307C10503D80500835707009385E5FF70
:1053A0001307E7FFB3870701B387C70013D60701C9
:1053B0002391F50013761600E31E67FD6FF05FEF93
:1053C00003DB2401B78700009387F7FF33FB6701F6
:1053D000131B0B01135B0B01E314FBDE13850400AD
:1053E000EFF08FA9E31405D48357290193C7F7FF82
:1053F00013971701E31607DC6FF09FD29307440160
:1054000013042400231F04FEE39C87FE6FF0DFD605
:105410009307440113042400231F04FEE31CF4FE3D
:105420006FF09FD5B73501809385856D1385040096
:10543000EFF0CF92630A050083D72401B3F7FA0097
:10544000E38E57F96FF05FFA130704019307040026
:1054500093872700239F07FEE39CE7FEB7C7FF7FE4
:105460002328F4006FF05FD183572501130101F564
:105470002324810A93C7F7FF2322910A2320210BBB
:10548000232E31092326110A232C4109232A5109ED
:1054900023286109232671092324810923229109E4
:1054A0002320A109232EB107139717011309050023
:1054B0009389050013040600938406006316070011
:1054C000EFE05FEF6318053883D7290193C7F7FF33
:1054D00013971701630E0708373A018093058A6D09
:1054E00013050900EFF08F8763040510035A2901A3
:1054F00003D72901B78700009387F7FF33FA4701E5
:10550000B3FAE700631AFA0813050900EFF0CF9623
:105510006308051063984A0113850900EFF0CF95E1
:105520006310050E9307440113042400231F04FE97
:10553000E31CF4FE8320C10A0324810A8324410A68
:105540000329010A8329C109032A8109832A410900
:10555000032B0109832BC108032C8108832C4108EC
:10556000032D0108832DC1071301010B6780000083
:1055700013850900EFE01FE4E30005F613874901F6
:1055800083D709009389290013042400231FF4FE04
:10559000E398E9FE6FF01FFA6386FA081305090025
:1055A0009305C101EFE01FEC93058103138509000A
:1055B000EFE05FEB835BA1030359E10163920B0C06
:1055C0009307C103930D0105638EFD3403D70700D4
:1055D00093872700E30A07FE13058103EFF04FAD21
:1055E000B307A0400356E1012326F1006F00C00974
:1055F00093058A6D13850900EFE05FF6E31805EE69
:10560000130704019307040093872700239F07FED5
:10561000E39CE7FEB7C7FF7F2328F4006FF09FF1FC
:10562000E39E4AF713850900EFF00F85E30805F6BE
:1056300013050900EFE01FDF93040500138509003F
:10564000EFE05FDEB387A440B337F0009397F70035
:105650002319F400130724019307040093872700FC
:10566000239F07FEE39CE7FE835724013787000052
:105670001307F7FFB3E7E7002319F4006FF09FEB80
:105680002326710113060900232421019307010237
:1056900093064103631206026380F62A03D70700CC
:1056A00093872700E30A07FE1305C101EFF04FA01F
:1056B000B307A9402324F10003278103138D84033A
:1056C00093070D0023AAE4021389E40493872700BB
:1056D000239F07FEE31CF9FE13058103EFE09FB64D
:1056E000035C2102370A0100930D0105931A0C0196
:1056F000B38A8A41130BA103130AFAFF930CE10644
:10570000930961058357C1030357E103930B0A0013
:1057100093970701B387E70063E8FA00B3D78703DD
:10572000939B070193DB0B01130641059305C10110
:1057300013850B00EFE09FBE1307C103930781059C
:1057400083D5070003560700938727001307270018
:105750006390C512E39697FF930700009305C10677
:1057600013860D000357060003D805001306E6FF55
:105770003307F74033070741935707012311E6002A
:1057800093F717009385E5FFE31E66FD23107D0167
:105790009307C10303D7270093872700239FE7FEC2
:1057A000E39AB7FF23180104130D2D00E31CA9F59C
:1057B000930500009307C1039306210503D7070053
:1057C00093872700B3E5E500E39AD7FE9397050199
:1057D00093D7074163840700930510009395050153
:1057E00093D50501138744039307810303560700EC
:1057F0009387270013072700239FC7FEE398F6FE31
:105800008327C10003278100B74600009386F6FF77
:10581000B38BE7401305810393870400130700044B
:10582000B386DB0013060000EFF04FA0035781039F
:105830008357C1019305040013058103B387E74033
:10584000B337F000B307F040231CF102EFF04FF53F
:105850006FF05FCE13074901835709001309290030
:1058600013042400231FF4FEE318E9FE6FF09FCC1D
:10587000E374B6EE9387FBFF9398070193D8080172
:1058800093070000930541031306C1060357060062
:1058900003D805001306E6FF3307F7403307074137
:1058A000935707012311E60093F717009385E5FF4F
:1058B000E31E36FD1307C1039307810583D5070057
:1058C0000356070093872700130727006398C50036
:1058D000E39697FF938B08006FF01FE8E37CB6FE1A
:1058E0009387EBFF939B070193DB0B0113060000EB
:1058F000930541031307C1068357070003D805002A
:105900001307E7FFB387C740B387074113D60701E3
:105910002311F700137616009385E5FFE31E37FD8C
:105920006FF09FE39307440113042400231F04FE38
:10593000E39C87FE6FF01FC00357C10183578103AB
:105940006304F700378600002319C40013072401FD
:105950009307040093872700239F07FEE31CF7FEAD
:1059600083572401378700001307F7FFB3E7E700E9
:105970002319F4006FF01FBC130101FD23248102E1
:105980002326110213840500930741001307E10148
:1059900093872700239F07FEE39CE7FE0356E5005D
:1059A0009317060193D7074163CA0706B78700001C
:1059B0009387F7FF231201003376F600630CF60697
:1059C0009307E5002313C1001307A10083D6E7FF67
:1059D0009387E7FF13072700231FD7FEE318F5FE81
:1059E000631206022314010093050400130541000D
:1059F000EFF00FDB8320C1020324810213010103B6
:105A000067800000930710009305F0FF1305410025
:105A10002314F100EFE01FC86FF01FFD9307F0FFA4
:105A20002312F100B78700009387F7FF3376F60063
:105A3000E318F6F8930705009306E50003D707007F
:105A400093872700631C0704E39AD7FE13074401DA
:105A50009307040093872700239F07FEE31CF7FEAC
:105A6000130724019307040093872700239F07FE51
:105A7000E31CF7FE83572401378700001307F7FF65
:105A8000B3E7E7002319F4008317E500E3D407F632
:105A900013050400EFE05F946FF0DFF513070401D6
:105AA0009307040093872700239F07FEE31CF7FE5C
:105AB000B7C7FF7F2328F4006FF0DFF383A8C5008A
:105AC000130101E183AE050003AE450003A3850089
:105AD000232E1103832505049308F0FF23201117BB
:105AE000930800092324811E232C411D2326111E07
:105AF0002322911E2320211F232E311D232A511DD5
:105B00002328611D2326711D2324811D2322911D1D
:105B10002320A11D232EB11B2328D103232AC10337
:105B2000232C6102232211172324C1002328D10032
:105B3000232AE100232E0101130A05001384070024
:105B4000638005020327450493071000B397E7001D
:105B500023A2E50023A4F500EF10903E23200A04C1
:105B6000930901069385090013050103EFF0DFE0B7
:105B700013850900EFE01F8B032781003335A00058
:105B80002320A40093073000E302F7149307400199
:105B90002326F100E31E07608357210703274116E0
:105BA00093C7F7FF232CE100139717016318070031
:105BB00013850900EFE01F80E316054093070009F5
:105BC0002322F1161307C107938709001306410723
:105BD00083D607009387270013072700231FD7FECC
:105BE000E398C7FE0356E10823220100931706013C
:105BF00093D7074163DE070013161601B7070100AC
:105C0000135616019387F7FF2317C1082322F100CB
:105C1000B73A018093878A6D938B47019306000002
:105C20009307810913870B00930DC10A6F00800051
:105C30008356070093872700239FD7FE130727006B
:105C4000E398B7FF63020616B78700009387F7FF54
:105C5000E30CF6588317C108E3DE075C9305C10720
:105C600013850B00EFE09F8F630C0514E34C050CCC
:105C70008357E108E39207668317C1089304000085
:105C80001309011663C80702B73701809387876D30
:105C9000138487111306C1079306090093050600B4
:105CA00013050400EFF0CFBA8317C1089384F4FF03
:105CB000E3D207FE1304010D130B810E130704003A
:105CC0009307C1071306010983D6070093872700AE
:105CD00013072700231FD7FEE398C7FE9306000093
:105CE0009307810913870B006F008000835607001C
:105CF00093872700239FD7FE13072700E398B7FF5A
:105D0000B73701801387876D9387876D37FDFFFF56
:105D1000930C8702930DC712138C87116F00C0007C
:105D2000938D4D01938C4C019305040013850B005A
:105D3000EFE0DF82930705009305040013850D0053
:105D40006356F004EFE09F81930705009306090076
:105D5000130604009305040013850C0063C00702BA
:105D6000EFF00FAF130681099306090093050600B3
:105D700013850C00EFF0CFADB384A4019357FD0160
:105D8000338DA701135D1D40E39C8CF91306810937
:105D90009306090093850B0013050600EFF0CFEC86
:105DA000930C41126F0000039307C1079306E108AB
:105DB00003D7070093872700E31207EAE39AD7FE89
:105DC00093040000930C4112130901161304010DF2
:105DD000130B810E9305040013058109EFE08FE892
:105DE000130781099307040083D6070093872700D0
:105DF00013072700231FD7FEE39867FF93050400CE
:105E00001305C1072318010AEFE0CFE59307C10787
:105E1000035704001304240093872700239FE7FE01
:105E2000E31864FF13058109130609009305C107F0
:105E3000231A0108EFF04F800355C11A6314051CA3
:105E4000130D41091304E107930B610B93858A6DD0
:105E50001305C107EFE08FF06306051A1307000072
:105E600093060D006F00C001131717002390F60072
:105E7000131707019386E6FF13570701638486040F
:105E800083D7060013960701135606419397170010
:105E900063540600136717009397070193D7070110
:105EA0001376270093E51700E30006FC131717008D
:105EB0002390B600131707019386E6FF13570701D7
:105EC000E39086FC1307410B9307C10783D60700B5
:105ED0009387270013072700231FD7FEE398A7FF08
:105EE0002316010C130700009306C10C6F00C001BC
:105EF000131717002390F600131707019386E6FF88
:105F0000135707016384760583D7060013960701AC
:105F10001356064193971700635406001367170042
:105F20009397070193D707011376270093E517008E
:105F3000E30006FC131717002390B60013170701A0
:105F40009386E6FF13570701E39076FD13070000E1
:105F50009306C10C6F00C001131717002390F600C1
:105F6000131707019386E6FF13570701638476052D
:105F700083D706001396070113560641939717001F
:105F800063540600136717009397070193D707011F
:105F90001376270093E51700E30006FC131717009C
:105FA0002390B600131707019386E6FF13570701E6
:105FB000E39076FD1306000093060D001307C10C55
:105FC00083D50600835707009386E6FF1307E7FF94
:105FD000B387B700B387C70013D607012391F60034
:105FE00013761600E31E77FD1305810913060900D9
:105FF0009305C107EFE05FE40355C11A9384F4FFF2
:10600000E30605E48327410083268100130730005F
:10601000B337F000B307F04093F7D7009387070238
:106020002302F1128327C1006394E600B38797002F
:106030001307A002138407006354F7001304A0029F
:106040001307A0006308E54C130505031307E002DE
:10605000A302A1122303E112E3CE071E93077112DC
:106060002322F100930B0000130D410B130B410988
:10607000130CE107930D610B1306000093050B0051
:106080006F00C001131616002390F50013160601C9
:106090009385E5FF135606016384850583D70500C4
:1060A0001395070113550541939717006354050095
:1060B000136616009397070193D7070113752600FF
:1060C00093E81700E30005FC131616002390150152
:1060D000131606019385E5FF13560601E39085FD2F
:1060E00013060D009307C10783D507009387270088
:1060F00013062600231FB6FEE39867FF2316010C44
:10610000130600009305C10C6F00C00113161600A2
:106110002390F500131606019385E5FF135606013B
:106120006384B50583D70500139507011355054111
:1061300093971700635405001366160093970701A1
:1061400093D707011375260093E81700E30005FCB9
:106150001316160023901501131606019385E5FF0B
:1061600013560601E390B5FD130600009305C10C1C
:106170006F00C001131616002390F50013160601D8
:106180009385E5FF135606016384B50583D70500A3
:1061900013950701135505419397170063540500A4
:1061A000136616009397070193D70701137526000E
:1061B00093E81700E30005FC131616002390150161
:1061C000131606019385E5FF13560601E390B5FD0E
:1061D0001305000093050B001306C10C83D80500BE
:1061E000835706009385E5FF1306E6FFB387170183
:1061F000B387A70013D507012391F5001375150088
:10620000E31EB6FD130609009305C10713058109B6
:10621000EFE09FC28357C11A03274100938507030C
:10622000330677012300B600938B1B00E35674E519
:106230001345F4FF1355F5413375A40013091500F8
:1062400033092701B30BA70013074000635EF7046F
:1062500013075000E386E7028347E9FF1307E9FFCE
:1062600093F7F707634A047A9306E0021306800364
:1062700093050003638ED7006358F67A8347F7FFD0
:106280002300B7001307F7FF93F7F7076FF09FFEA0
:106290008347F7FF93068003E3FAF60293071003A0
:1062A00093841400A30FF7FEB73501801386040012
:1062B0009385456D13850B00EF20C06A8357210736
:1062C000032781012328911693C7F7FF2322E116A4
:1062D00013971701631E070013850900EFE0CFB97C
:1062E0006310052213850900EFE0CF8C631A0520A7
:1062F00083264101034741129387140023A0F6002F
:1063000093870C00630A07029306E002630CD71C14
:1063100003C7170093871700E31A07FE930650047C
:1063200063E6FC006F0040016388970103C7F7FF35
:106330009387F7FFE31AD7FE2380070093870C00AB
:10634000930600021306D00203C707006304D700B8
:106350006316C700938717006FF01FFF13840C00AC
:106360006F00C00003C70700138406002300E40089
:106370009306140093871700E31607FE8326810017
:10638000930720000347F4FF6386F6128327C100BA
:106390009386070063D49700938604009307000355
:1063A0006316F702B307944163D2F60213060003A3
:1063B0006F00800063DCE6008347E4FFA30F04FE68
:1063C0001304F4FF33079441E386C7FE03278100DB
:1063D000930730006302F70A8327010123220A048E
:1063E000938697009307700163F2D70C1307100090
:1063F0009307400093971700138647019305070002
:1064000013071700E3F8C6FE2322BA0413050A0097
:10641000EF1080282320AA0493850C009304050024
:10642000EF20005C8327C101638807003304944197
:106430003384840023A087008320C11E0324811E8F
:106440000329011E8329C11D032A811D832A411DA1
:10645000032B011D832BC11C032C811C832C411C8D
:10646000032D011C832DC11B138504008324411EB1
:106470001301011F678000008327C100B3849700C8
:1064800063CE0452832741010327010183A707003C
:10649000B307F7002328F1008327010123220A0410
:1064A0009386370093077001E3E2D7F49305000069
:1064B0006FF0DFF593070003E310F7F2B3079441A1
:1064C00093061000E3C4F6EE6FF01FF1032C0101F8
:1064D000232681019307A00263D087ED2326F100D4
:1064E0006FF08FEB03C70700E30A07E203C717004B
:1064F00093871700A38FE7FEE31A07FE6FF01FE2F2
:1065000003274101B72700009387F7702320F70086
:106510006FF0DFE213071003A302E1121307E0029A
:106520002303E11293841400635EF02A93070003AF
:10653000A303F112930781121304F4FF2322F10045
:106540006FF05FB2130D410B13070D009307C107E6
:106550001306010983D60700938727001307270036
:10656000231FD7FEE398C7FEB74700009387E708CD
:106570002313F10CB73701809387876D138B870C3A
:10658000B78700009387F7FF2322F102B7C7FFFF09
:1065900093872700130E000193040000930C41120F
:1065A000130901161304010D130CA10A2324F1028F
:1065B000930609001306810993050D0013050B00CE
:1065C0002320C103EFE05FEA032E01021307C10499
:1065D0009307810983D607009387270013072700B5
:1065E000231FD7FEE398B7FF832741028355E105B8
:1065F00033F6F500832781023305F600635AA03C89
:10660000130600093306A640130704009307C104CC
:1066100083D607009387270013072700231FD7FE81
:10662000E39837FF6358C0069307F0001307040090
:1066300063DCC702130606FF935646001387160055
:10664000131717003307E40093070400938727000C
:10665000239F07FEE39CE7FE130600083306A640CF
:10666000939646003306D640B73701809387876DEF
:10667000131616003386C700835606238357070078
:10668000B3F7D7002310F7009395050193D5054183
:1066900063C20516930781091307040003D6070098
:1066A0008356070093872700130727006314D60239
:1066B000E316FCFE13070D009307810983D607003C
:1066C0009387270013072700231FD7FEE398B7FF00
:1066D000B384C401B73701809387876D130B4B01D7
:1066E0009387C712135E1E00E314FBEC8357610C03
:1066F0000357E1081306810CB387E70037C7FFFF94
:10670000130727F7B387E7002313F10C1307C1071B
:1067100093070D0083D607009387270013072700F0
:10672000231FD7FEE398C7FE1307000093078109D4
:106730006F00800003D70B0093872700239FE7FE9D
:10674000938B2B00E398B7FFB73701801387876DD2
:106750009387876DB71D0000130B8702938B8711FA
:106760006F00000193DD1D0063047B2B130B4B01B5
:1067700093050D0013850B00EFD05FDE13070500B6
:1067800093050D0013050B006344E028EFD01FDDD7
:10679000E34AA0FC9306090013060D0093050D00C3
:1067A00013050B00EFE05FCC130681099306090087
:1067B0009305060013050B00EFE09F89B384B40135
:1067C0006FF05FFA930C4112B73501809385056B2A
:1067D00013850C00B7240000EF20C0189384F470D8
:1067E0006FF0DFAD930B7112E39007AC23227101C0
:1067F0006FF05F879307C104130704006F00C000A8
:106800009306E105E388F6E803D607008356070000
:106810009387270013072700E304D6FE8357210E32
:1068200003274102B377F7006394E70213050400DE
:106830002320C103EFD01FB8032E0102E31C05E49F
:1068400013050400EFD05FE3032E0102E31405E417
:106850009305C10E13850B002320C103EFD09FC009
:106860009305811013050400EFD0DFBF0356C10E5E
:106870000355A110835EE10E1346F6FF13160601C1
:10688000135606012316C10EB385AE40032E010236
:1068900093060500635EB00693860C001307811013
:1068A00093070112835507001307270093862600DC
:1068B000239FB6FEE318F7FE231E01121307811073
:1068C0009306C10E6F00800003D606001307270051
:1068D000231FC7FE93862600E318F7FE231001123C
:1068E0001307C10E93870C00130FC11383D6070043
:1068F0009387270013072700231FD7FEE398E7FF9E
:106900008356A110B305D54123120110138506004B
:106910006380052E2326D1029307F0F663CEF50699
:106920001305C10E2320C103EFD0DFD6032E0102D1
:106930008326C10293050500930701121306411037
:106940000355C10E035781106300E53013050000A5
:1069500003D70700835E06009387E7FF3307A7404E
:106960003307D741135507012391E7001307A110FF
:10697000137515001306E6FFE39CE7FC13061000F1
:106980009307090013070004130581102320C10396
:10699000EFE0CF89032E0102930504001305811057
:1069A0002320C103EFE0CFDF032E01026FF09FCE63
:1069B00083270101138CF7FF6FF09FB183274101FB
:1069C0002302011213840C0023A007006FF0DFAC38
:1069D000930704001307410E93872700239F07FEA8
:1069E000E39CE7FE6FF05FCA83274100930C4112DE
:1069F000638A0706B73501809385856B13850C0084
:106A0000B7240000EF1010769384F4706FF01F8BA2
:106A1000130B810E6FF00FBC93071003230FF9FEC9
:106A2000938414006FF05F88938717002300F700AA
:106A30006FF09F87930C4112B73501809385056DE8
:106A400013850C00B7240000EF10D0719384F4700C
:106A50006FF0DF868357C11A930B6112130971120D
:106A60006FF08FFEB73501809385456C13850C0060
:106A7000B7240000EF10106F9384F4706FF01F8440
:106A8000930581091305C107EFE08FD193858A6DC6
:106A900013058109EFD09FAC631005FCE346048029
:106AA0008347E9FF138727FD133717001347F7FFC5
:106AB0003387EB000347070013771700630607FED1
:106AC0001307E9FF93F7F7076FF00FFA93871700A3
:106AD000A30FF7FE6FF04FFD1304010D93050400A3
:106AE0001305C107374D0000EFD0DF979304000076
:106AF000130B810E1309C10C930C210D130DEDFF27
:106B0000130C50FD8357810E93F777006398070CA1
:106B10001307410B9307040083D6070093872700D0
:106B200013072700231FD7FEE39867FF1305410BC8
:106B30002316010CEFD00FF11305410BEFD08FF0AE
:106B4000130600009306090013070B0083D5060007
:106B5000835707009386E6FF1307E7FFB387B70065
:106B6000B387C70013D607012391F60013761600EA
:106B7000E31E97FD8357610B0357810B9387370003
:106B8000231BF10A630007021305410BEFD08FEBC3
:106B90008357610B0357810B93871700231BF10A5F
:106BA000E31407FE8357C10C639A07028357610BF6
:106BB0006366FD02130704009307410B83D60700A9
:106BC0009387270013072700231FD7FEE39827FF8B
:106BD0002314010E9384F4FFE39684F39305C10715
:106BE00013050400EFE0CFBB130901166FF00F8D02
:106BF0001307C1109307010F83DE07000356070038
:106C000093872700130727006398CE0213066110AD
:106C1000E394C7FE0357C10E835781106302F70642
:106C2000930704001307410E93872700239F07FE55
:106C3000E39CE7FE6FF01FA66366D60D9307011273
:106C4000130641106FF0DFCF13050000130FE10EA4
:106C500083DE0700035706009387E7FF1306E6FF6E
:106C60003307D7013307A700135507012391E70026
:106C700013751500E31EE6FD130600006FF05FD0EC
:106C800013870600639206068317E11063CE07049C
:106C9000930601126F0000022390F60013171700ED
:106CA000131707019386E6FF9307A11013570701F7
:106CB000E384F6CE83D706001396070113560641E8
:106CC0009397170063540600136717009397070103
:106CD00093D707011376270093E51700E30E06FA12
:106CE0002390B6006FF09FFB1306C11093070112AB
:106CF000631207086382C7080357060013062600BD
:106D00006FF01FFF13860C00130781109307011209
:106D1000035507001307270013062600231FA6FEAE
:106D2000E318F7FE231E0112130581101307C10E8D
:106D300013064110835E0700130727001305250083
:106D4000231FD5FFE318C7FE231001121305C10E40
:106D500013870C00130FC113835E0700130727006E
:106D600013052500231FD5FFE318E7FF23120110A9
:106D70006FF01FBD138516002315A1106FF0DFC142
:106D8000032785008327C5000326050083264500C9
:106D9000130101FC13050100930541012324E100C7
:106DA0002326F100232E11022320C1002322D1002B
:106DB000EFE09FBC835761021305000093C7F7FF04
:106DC00013971701631A070013054101EFD08FDEF7
:106DD00013351500130515008320C10313010104A9
:106DE000678000001305050F67800000376501808C
:106DF0001305859D67800000376501801305859D1B
:106E000067800000130101FD232E310123261102AA
:106E1000232481022322910223202103232C4101D8
:106E2000232A510123286101232671012324810192
:106E3000232291019387B500130760019309050090
:106E40006366F7069307000163E6B71EEF00500480
:106E50009304000113062000930780013759018035
:106E60001309094EB307F90003A44700138787FFEE
:106E7000630AE420832744008326C4000326840099
:106E800093F7C7FFB307F40003A747002326D600F4
:106E900023A4C600136717001385090023A2E70087
:106EA000EF00407F130584006F00801993F487FF83
:106EB00063C2071863E0B418EF00807D9307701F6A
:106EC00063F6974693D794006386071A130740002A
:106ED000636CF73C93D7640013869703138587038D
:106EE00093163600375901801309094EB306D900AD
:106EF00003A44600938686FF638686029305F0000E
:106F00006F000001635C07320324C400638C8600B9
:106F10008327440093F7C7FF33879740E3D4E5FE08
:106F20001306050003240901930889006308141758
:106F3000032544009306F0001375C5FFB307954081
:106F400063CCF640232A19012328190163D6073E92
:106F50009307F01F63EAA72E937785FF9387870037
:106F600083254900B307F90083A607001355550090
:106F7000130710003317A7003367B700938587FF07
:106F80002326B4002324D4002322E90023A0870071
:106F900023A686009357264093051000B395F5006D
:106FA0006368B710B3F7E500639407029395150083
:106FB0001376C6FFB3F7E50013064600639A070091
:106FC00093951500B3F7E50013064600E38A07FE24
:106FD0001308F00013133600330369001305030090
:106FE0008327C500130E06006302F52E03A7470092
:106FF0001384070083A7C7001377C7FFB306974022
:107000006342D82EE3C206FE3307E400832647001E
:10701000032684001385090093E616002322D70077
:107020002326F60023A4C700EF00C06613058400E2
:107030006F0000019307C00023A0F90013050000B2
:107040008320C10203248102832441020329010217
:107050008329C101032A8101832A4101032B0101F4
:10706000832BC100032C8100832C410013010103F9
:107070006780000093060020130600041305F00348
:107080006FF05FE603A4C70013062600E39487DED3
:107090000324090193088900E31C14E9032749002C
:1070A0009357264093051000B395F500E37CB7EEA7
:1070B00003248900832A440013FBCAFF63689B00F2
:1070C000B3079B401307F0006346F714B7670180CE
:1070D000B76C018083AA87A803A78CA79307F0FF4A
:1070E000330A6401B38A5401630AF734B717000006
:1070F0009387F700B38AFA00B7F7FFFFB3FAFA00F5
:1071000093850A0013850900EF1000799307F0FFBB
:10711000930B0500630CF52863684529376C0180E3
:10712000130C0CAD83250C00B385BA002320BC00E2
:10713000938705006304AA3A83A68CA71307F0FF80
:10714000638CE63A338A4B41B307FA002320FC00F4
:1071500093FC7B0063860C30B7170000B38B9B4118
:1071600093858700938B8B00B3859541B38A5B0130
:107170009387F7FFB385554133FAF50093050A006D
:1071800013850900EF1040719307F0FF6300F53C91
:1071900033057541B30A450183250C002324790189
:1071A00093EA1A00B305BA002320BC0023A25B01B6
:1071B000630824359306F00063F86635032744001E
:1071C00093074BFF93F787FF137717003367F70099
:1071D0002322E400130650003307F4002322C700E3
:1071E0002324C70063EEF63683AA4B0013840B00FA
:1071F000B767018003A747A86374B70023A2B7A8A5
:10720000B767018003A707A86376B71A23A0B7A8BA
:107210006F00401A13E714002322E400B304940023
:107220002324990093E717001385090023A2F40093
:10723000EF004046130584006FF09FE08326C400F2
:10724000032684006FF01FC4935795001307400076
:107250006372F71413074001636AF7229386C70528
:107260009385B70593963600B306D90083A7060029
:10727000938686FF6388F61C03A747001377C7FF32
:107280006376E50083A78700E398F6FE83A6C70030
:10729000032749002326D4002324F40023A48600D6
:1072A00023A687006FF01FCF130740016376F71204
:1072B00013074005636AF71E93D7C4001386F706C9
:1072C0001385E706931636006FF0DFC1130E1E001C
:1072D00093773E0013058500638E07108327C50052
:1072E0006FF09FD00326840093E514002322B4009E
:1072F0002326F60023A4C700B3049400232A990090
:107300002328990093E7160023A6140123A414014F
:1073100023A2F4003307E400138509002320D700DB
:10732000EF004037130584006FF09FD113D634006F
:10733000938784006FF09FB23307A4008327470030
:107340001385090093E717002322F700EF0080342C
:10735000130584006FF0DFCE13E714002322E4004E
:10736000B3049400232A99002328990013E71700F7
:1073700023A6140123A4140123A2E4003305A400CE
:107380002320F50013850900EF00C03013058400A9
:107390006FF01FCB93576500938697039385870300
:1073A000939636006FF05FEC630E2411032489007E
:1073B000832A440093FACAFFB3879A4063E69A008F
:1073C0001307F000E348F7E413850900EF00802C71
:1073D000130500006FF0DFC61386C7051385B705D8
:1073E000931636006FF01FB0832783001306F6FF55
:1073F0006392671C93773600130383FFE39607FEBF
:107400000327490093C7F5FFB3F7E7002322F900EC
:1074100093951500E3EEB7C8E38C05C833F7F50084
:10742000631A07009395150033F7F500130E4E000D
:10743000E30A07FE13060E006FF0DFB9938A0A0114
:107440006FF01FCC0325490093D52540130710008A
:107450003317B7003367A7002322E9006FF09FE3DB
:10746000B3855B01B305B0409395450113DA45013F
:1074700093050A0013850900EF1000429307F0FFFF
:10748000E318F5D0130A00006FF01FD11307400571
:107490006362F7089357C5009386F7069385E7065E
:1074A000939636006FF05FDC130740156362F708B0
:1074B00093D7F40013868707138577079316360052
:1074C0006FF05FA2376C0180130C0CAD83270C00AA
:1074D000B387FA002320FC006FF01FC613174A0180
:1074E000E31C07C403248900B30A5B0193EA1A0072
:1074F000232254016FF0DFCF23AC7CA76FF05FC570
:1075000013840B006FF0DFCE9307100023A2FB0063
:107510006FF09FEB130740156362F7069357F50072
:107520009386870793857707939636006FF0DFD3AE
:10753000130740556362F70693D724011386D707D4
:107540001385C707931636006FF0DF99938C8CFF75
:10755000B38A9A01B38A7A41130A00006FF0DFC33D
:107560009305840013850900EFC09F9C03248900C4
:1075700083250C00832A44006FF09FC713074055F2
:107580006364F702935725019386D7079385C7074E
:10759000939636006FF05FCD9306803F1306F00799
:1075A0001305E0076FF01F949306803F9305E007F3
:1075B0006FF09FCB832749006FF09FE593773500ED
:1075C00093F6F50F638A07029307F6FF630E060230
:1075D0001306F0FF6F0080011305150013773500C7
:1075E000630E07009387F7FF6380C7020347050018
:1075F000E314D7FE678000009307060013073000EE
:107600006366F702639607001305000067800000B9
:10761000B307F5006F00C00013051500E386A7FE51
:1076200003470500E31AD7FE678000003707010013
:10763000939885001307F7FFB3F8E80093F5F50F6B
:10764000B3E5B80093980501B3E8B8003708FFFE2A
:10765000B78580801308F8EF938505081303300081
:107660000327050033C7E800330607011347F7FF78
:107670003377E6003377B700E31C07F89387C7FF3B
:1076800013054500E36EF3FCE39407F86FF0DFF7B2
:1076900067800000678000008327C504130101FF95
:1076A000232481002322910023261100232021017D
:1076B0001304050093840500638E070213952400CC
:1076C000B387A70003A50700630605040327050089
:1076D00023A0E70023280500232605008320C100FE
:1076E00003248100832441000329010013010101C7
:1076F000678000001306100293054000EF20806DA4
:107700002326A40493070500E31A05FA13050000D5
:107710006FF0DFFC130910003319990013065900AC
:10772000131626009305100013050400EF20806A4D
:10773000E30E05FC23229500232425016FF09FF919
:107740006380050203A745008327C504131727009C
:10775000B387E70003A7070023A0E50023A0B70035
:1077600067800000130101FE232A910083A4050114
:1077700037030100232C8100232821012326310116
:10778000232E1100232441011389050093090500CC
:107790001384060013884501930800001303F3FFC8
:1077A000832708001308480093881800B3F6670081
:1077B000B386C60293D70701B387C702B386860094
:1077C00013DE060133F76600B386C70193970601FF
:1077D0003387E700232EE8FE13D40601E3C298FCAA
:1077E000630204028327890063D0F4049387440072
:1077F00093972700B307F90023A28700938414000E
:10780000232899008320C10103248101832441019D
:107810008329C100032A81001305090003290101FE
:1078200013010102678000008325490013850900C8
:1078300093851500EFF05FE6130A0500630C05045D
:10784000032609019305C9001305C5001306260088
:1078500013162600EF20C07C0327490083A7C90424
:1078600013172700B387E70003A707002320E900C9
:1078700023A027019387440013090A009397270048
:10788000B307F90023A287009384140023289900EA
:107890006FF05FF7B7460180374501809386C69247
:1078A000130600009305500B13050594EF20C04B01
:1078B000130101FE232C8100232A9100232821019A
:1078C0002326310123244101138886009307900069
:1078D000232E1100232251013348F8029389060018
:1078E0001309050013840500130A0600930407001A
:1078F00063D8D70C930710009305000093971700E7
:1079000093851500E3CC07FF13050900EFF0DFD8DE
:1079100093050500630A050A930710002328F50064
:10792000232A95009307900063D64709930A940091
:1079300093840A003304440183C604001306A000A4
:1079400013050900938606FDEFF0DFE19384140030
:1079500093050500E39284FE13048AFF33848A00B2
:1079600063563A03B3894941B3093401834604009D
:107970001306A00013050900938606FDEFF09FDEB5
:107980001304140093050500E39289FE8320C101CE
:107990000324810183244101032901018329C100BA
:1079A000032A8100832A4100138505001301010287
:1079B000678000001304A400130A90006FF05FFAC0
:1079C000930500006FF05FF4B746018037450180F2
:1079D0009386C692130600009305E00C13050594E8
:1079E000EF2080383707FFFF3377E5009307050066
:1079F00013050000631607009397070113050001A4
:107A0000370700FF33F7E70063160700130585000B
:107A100093978700370700F033F7E70063160700F6
:107A20001305450093974700370700C033F7E70079
:107A300063160700130525009397270063C8070006
:107A400013971700130515006354070067800000A3
:107A50001305000267800000832705001307050057
:107A600093F677006384060293F61700130500006F
:107A7000639E060693F627006380060893D71700D7
:107A80002320F7001305100067800000939607017C
:107A900093D60601130500006396060093D70701ED
:107AA0001305000193F6F70F639606001305850092
:107AB00093D7870093F6F7006396060013054500F9
:107AC00093D7470093F63700639606001305250009
:107AD00093D7270093F61700639C060093D71700EF
:107AE0001305150063960700130500026780000068
:107AF0002320F7006780000093D727002320F7009A
:107B00001305200067800000130101FF232481007A
:107B1000138405009305100023261100EFF0DFB752
:107B2000630005028320C100232A8500032481000D
:107B3000130710002328E5001301010167800000EE
:107B4000B7460180374501809386C6921306000030
:107B50009305001413050594EF200021130101FE85
:107B6000232821012326310103A9050183290601C8
:107B7000232A910023244101232E1100232C81006C
:107B8000138A050093040600634C3901138709002A
:107B90009384050093090900130A060013090700DE
:107BA00083A7840083A5440033842901B3A78700F9
:107BB000B385F500EFF05FAE630C051A13034501C2
:107BC00093182400B308130193070300637813018B
:107BD00023A0070093874700E3EC17FF13084A012F
:107BE000131E2900938E440193952900330EC8017A
:107BF000B385BE00637CC80B93875401130F40000C
:107C000063FEF514370601001306F6FF6F0000014E
:107C10001308480013034300637AC809832F080040
:107C2000B3F4CF006394040C93DF0F01E3820FFEE3
:107C3000032703009302030093860E0093040700BA
:107C40009303000083A7060093D904013377C7008C
:107C5000B3F7C700B387F70383A4420093824200BF
:107C60009386460033F9C400B3873701B3877700A2
:107C70009393070133E7E30023AEE2FE03D7E6FF69
:107C800093D707013307F703330727013307F700BB
:107C900093530701E3E8B6FAB307E30123A0E70033
:107CA0001308480013034300E36AC8F763488000E1
:107CB0006F0080011304F4FF6308040083A7C8FF6A
:107CC0009388C8FFE38807FE8320C101232885002D
:107CD0000324810183244101032901018329C10077
:107CE000032A81001301010267800000930303004F
:107CF00093820E001309000003A7020083AF030064
:107D000093834300B376C700B38696029357070167
:107D100033F7CF0093DF0F0193824200B3879702BE
:107D2000B386E600B386260113D70601B3F6C60074
:107D3000B387F701B387E70013970701B366D7004E
:107D400023AED3FE13D90701E3E8B2FAB307E30188
:107D500023A02701832F08006FF01FED338F95407C
:107D6000130FBFFE137FCFFF130F4F006FF09FE97C
:107D7000B7460180374501809386C69213060000FE
:107D80009305D01513050594EF10107E130101FE25
:107D9000232C81002326310123244101232E1100AD
:107DA000232A91002328210193773600130406002B
:107DB00093090500138A05006394070C13542440AB
:107DC00013090A006308040683A48904638E040C63
:107DD0009377140013090A006390070213541440A8
:107DE000630A040403A50400630805069304050060
:107DF00093771400E38407FE1386040093050900BB
:107E000013850900EFF09FD5630809060327490091
:107E100083A7C9041354144013172700B387E7003E
:107E200003A707002320E90023A027011309050069
:107E3000E31A04FA8320C101032481018324410150
:107E40008329C100032A81001305090003290101C8
:107E5000130101026780000013860400938504006B
:107E600013850900EFF09FCF23A0A4002320050075
:107E7000930405006FF0DFF7130905006FF01FF69C
:107E80009387F7FF37470180130787999397270058
:107E9000B307F70003A6070093060000EFF09F8CDE
:107EA000130A05006FF09FF1930510271385090051
:107EB000EFF09FC523A4A904930405002320050027
:107EC0006FF01FF1130101FE2324410103AA0501F4
:107ED00083A785002326310193595640338A4901EF
:107EE000232C8100232A91002328210123225101E0
:107EF000232E110013091A009384050013040600B1
:107F000083A54500930A050063D8270193971700BE
:107F100093851500E3CC27FF13850A00EFF0CFF718
:107F2000630C05101308450163543003938959000D
:107F30009399290033073501930708009387470079
:107F400023AE07FEE39CE7FE9389C9FE33083801A0
:107F500003A70401938744011373F4011316270048
:107F60003386C7006304030A93050002B3856540A6
:107F7000930808009306000003A7070093884800B1
:107F800093874700331767003367D70023AEE8FEB7
:107F900003A7C7FFB356B700E3E0C7FE138754013A
:107FA00093074000636AE600B30796409387B7FEE5
:107FB00093F7C7FF938747003308F8002320D800C2
:107FC00063840600130A090003A7440083A7CA04B8
:107FD0008320C10113172700B387E70003A7070019
:107FE000232845010324810123A0E40023A0970056
:107FF00003290101832441018329C100032A81004F
:10800000832A4100130101026780000003A70700D3
:108010009387470013084800232EE8FEE3F6C7FACB
:1080200003A707009387470013084800232EE8FEA4
:10803000E3EEC7FC6FF05FF9B7460180374501807A
:108040009386C692130600009305901D13050594B0
:10805000EF1090510327050183A7050113080500C0
:108060003305F7406314F70493972700130848017A
:10807000938545013307F800B387F5006F00800052
:108080006376E8028326C7FF03A6C7FF1307C7FF6F
:108090009387C7FFE386C6FEB3B6C6003305D0405C
:1080A0001375E5FF13051500678000006780000069
:1080B00083A7050103270601130101FF2324810083
:1080C00023229100232021012326110093840500FF
:1080D000130406003389E7406394E71A93162700D8
:1080E0009385450113074601B387D5003307D700B1
:1080F0006F00800063FCF51803A6C7FF8326C7FF47
:108100009387C7FF1307C7FFE306D6FE6360D61643
:1081100083A54400EFF04FD86302051A03AE0401B3
:1081200083220401938F4401931E2E0013084401FF
:108130009392220093034501B708010023262501ED
:10814000B38EDF01B3025800138F030013830F00B7
:10815000930700009388F8FF032703008325080096
:10816000130F4F00B3761701B386F600B3F715016E
:10817000B386F64093D5050193570701B387B740FF
:1081800013D70641B387E70013970701B3F616012B
:10819000B366D70013084800232EDFFE1303430005
:1081A00093D70741E36A58FAB38582409385B5FEB9
:1081B0001304540193D525001307000063E48200E3
:1081C000139725003387E3001308400063E682001D
:1081D0009385150013982500B38F0F01B383030116
:1081E00063FEDF05B70801001388030093850F00C5
:1081F0009388F8FF03A705001308480093854500FE
:10820000337617013306F60093560641935707015C
:10821000B387D7009396070133761601B3E6C600FD
:10822000232ED8FE93D70741E3E6D5FD1387FEFF43
:10823000B30FF74113F7CFFF3387E300639A0600CC
:108240008327C7FF130EFEFF1307C7FFE38A07FE4E
:108250008320C100032481002328C5018324410019
:1082600003290100130101016780000093870400C6
:108270001309100093040400138407006FF05FE9F2
:10828000E34609FE130900006FF09FE89305000024
:10829000EFF08FC0630205048320C1000324810036
:1082A000930710002328F500232A050083244100AA
:1082B000032901001301010167800000B746018016
:1082C000374501809386C69213060000930500246B
:1082D00013050594EF105029B746018037450180FA
:1082E0009386C69213060000930520231305059478
:1082F000EF109027B707F07FB3F5B700B707C0FCC2
:10830000B385F5006358B00093070000138507009C
:1083100067800000B305B04093D545419307300115
:1083200063C8B700B7070800B3D5B7406FF0DFFDEB
:108330001387C5FE9306E001930500009307100024
:10834000E3C6E6FCB7070080B3D7E7001385070054
:1083500067800000130101FE232A91008324050198
:10836000232C81001304450193942400B30494004A
:108370002328210103A9C4FF23263101232441011D
:108380001305090093890500232E1100EFF08FE5F6
:1083900013070002B307A74023A0F9009307A0002A
:1083A000138AC4FF63D0A708130555FF6370440503
:1083B00083A784FF63000504B306A74033D7D70023
:1083C0003319A9003369E900138684FF3707F03FAA
:1083D0003367E900B397A7006372C40203A644FFA2
:1083E000B356D600B3E7D7006F00400193070000F3
:1083F000631405063707F03F3367E9008320C101A6
:108400000324810183244101032901018329C1003F
:10841000032A810013850700930507001301010259
:10842000678000009306B000B386A640B707F03F10
:108430003357D9003367F700930700006376440190
:1084400083A784FFB3D7D700130555013315A900BF
:10845000B367F5006FF09FFA3315A9003707F03FB7
:108460003367E500930700006FF05FF9130101FD2A
:10847000232C4101138A0500930510002322910249
:1084800023202103232E31012326110223248102DC
:10849000232A51019304060093890600130907005B
:1084A000EFF08F9F630A051093D744013707100040
:1084B0001306F7FF939657011304050033769600D1
:1084C00093FAF77F638406003366E6002326C10033
:1084D00063080A081305810023244101EFF0CFD778
:1084E0000327C100930705006302050C03268100E2
:1084F00093060002B386A640B316D700B3E6C600C3
:108500003357A700232AD4002326E100B334E00028
:1085100093841400232CE4002328940063840A0627
:10852000938ADABCB38AFA001305500323A05901D9
:10853000B307F5402320F9008320C102130504008E
:108540000324810283244102032901028329C101FA
:10855000032A8101832A410113010103678000007E
:108560001305C100EFF04FCF930710002328F4004C
:108570008327C10093041000232AF4009307050207
:10858000E3900AFA139724003307E4000325070158
:108590009387E7BC23A0F900EFF0CFC49394540075
:1085A000B384A440232099006FF01FF98326810033
:1085B000232AD4006FF09FF5B7460180374501802C
:1085C0009386C692130600009305A0301305059408
:1085D000EF108079130101FD232021031389050089
:1085E0009305810023261102232481022322910274
:1085F000232E310193090500EFF0DFD59304050028
:1086000013840500130509009305C100EFF09FD402
:108610008327090103A709018326C1003307F74017
:108620008327810013175700B387D740B307F7009C
:1086300093060500635EF002939747013384870039
:108640001386060013850400938605009305040035
:10865000EF50D0728320C10203248102832441029F
:10866000032901028329C10113010103678000006E
:1086700013974701B385E5406FF09FFC130101FF9D
:10868000232021012326110023248100232291008D
:10869000930770011309050063DAA70437670180A7
:1086A000832787A58325C7A537670180032407A6ED
:1086B000832447A61385070013060400938604004D
:1086C000EF60C0771309F9FF93070500E31409FE73
:1086D0008320C10003248100832441000329010079
:1086E000138507001301010167800000B74701806F
:1086F0001319350093878799338927018327090147
:108700008320C10003248100832549018324410083
:108710000329010013850700130101016780000090
:10872000832606019385F5FF93D555409385150063
:10873000930746019396260093952500B386D700AC
:10874000B305B50063F8D7021307050003A80700B7
:108750009387470013074700232E07FFE3E8D7FE60
:10876000B387C6409387B7FE93F7C7FF9387470049
:108770003305F5006378B50013054500232E05FE8B
:10878000E36CB5FE678000000327050113D6554052
:10879000930645016352C70293172700B387F6007B
:1087A00063F2F60403A7C7FF9387C7FFE30A07FE38
:1087B000130510006780000093172600B387F600AA
:1087C000E350E6FE93F5F501E38C05FC03A60700F4
:1087D000130510003357B600B315B700E302B6FC1B
:1087E000678000001305000067800000130101FF8F
:1087F00023229100B7040080232481002326110046
:1088000093C4F4FF1304060023200600B3F6B4005B
:108810003706F07F938705001307050063D0C6066F
:10882000B3E8A600638C080433F6C500138805007E
:108830009308000063120602B767018083A6C7A6EB
:1088400003A687A6EF60805F130705001388050065
:10885000B3F6B4009308A0FC93D64641B707108046
:108860009387F7FF938626C03378F800B386160106
:10887000B707E03FB367F8002320D4008320C1008E
:10888000032481008324410013050700938507001A
:108890001301010167800000130101FF23248100FF
:1088A0002322910013040500B7640180138505009D
:1088B0002326110023AC04B8EF50C02E9307F0FF1D
:1088C000630CF5008320C100032481008324410050
:1088D000130101016780000083A784B9E38407FEC8
:1088E0008320C1002320F40003248100832441005D
:1088F0001301010167800000130101F6930EC10806
:10890000232AF10837030080B707FFFF138E050005
:108910001343F3FF2326D108938787209305810013
:1089200093860E00232E1106232AF1002328E10846
:10893000232C0109232E11092324C101232CC10159
:10894000232E6100232861002322D101EF80DF9DC7
:1089500083278100238007008320C1071301010AB8
:1089600067800000130E050037650180130101F6D2
:10897000032545A7930E8108232AF10837030080B9
:10898000B707FFFF1343F3FF2324C1082326D108B1
:10899000938787201386050093860E009305810038
:1089A000232E1106232AF1002328E108232C010994
:1089B000232E11092324C101232CC101232E610080
:1089C000232861002322D101EF801F968327810095
:1089D000238007008320C1071301010A678000007C
:1089E000B367B50093F737006392070803A7050044
:1089F000B7867F7F9386F6F7B377D700B387D70024
:108A0000B3E7E700B3E7D7001306F0FF639EC7069E
:108A1000130605001308F0FF2320E60003A7450016
:108A20009385450013064600B377D700B387D70078
:108A3000B3E7E700B3E7D700E38007FF83C705008C
:108A400003C7150083C625002300F600638A0700CC
:108A5000A300E600630607002301D6006394060026
:108A600067800000A30106006780000093070500EF
:108A700003C705009387170093851500A38FE7FEB2
:108A8000E31807FE67800000130605006FF01FFB68
:108A90009377350013070500639C0704B7867F7F33
:108AA0009386F6F79305F0FF0326070013074700A8
:108AB000B377D600B387D700B3E7C700B3E7D700D3
:108AC000E384B7FE8346C7FF0346D7FF8347E7FF2C
:108AD0003307A74063800604630A06023335F000BB
:108AE0003305E5001305E5FF67800000E38806FA1B
:108AF000834707001307170093763700E39807FEB4
:108B00003307A7401305F7FF678000001305D7FF61
:108B1000678000001305C7FF67800000B3E7A5006A
:108B200093F7370013070500639807069307300093
:108B300063F4C7063703FFFEB78880801303F3EFA3
:108B400093880808130E300083A60500B3876600DB
:108B500013C8F6FFB3F70701B3F71701639E0702C7
:108B60002320D7001306C6FF13074700938545004F
:108B7000E36CCEFC9385150093071700630406028F
:108B800083C6F5FF1308F6FFA38FD7FE638E06009A
:108B90001387070013060800938515009307170035
:108BA000E31006FE678000003306C700630A080072
:108BB00093871700A38F07FEE39CC7FE6780000022
:108BC0006780000083278600130101FD232A5101DD
:108BD0002326110223248102232291022320210330
:108BE000232E3101232C4101232861012326710109
:108BF00023248101930A060063880714130B0500E0
:108C00008329060003A5050083A4850013840500BD
:108C10006F00400D8357C40013F70748630A070825
:108C20008326440183250401130719009394160039
:108C3000B386D40093D4F601330AB540B384D4008C
:108C400093D41440330747011386040063F6E4000D
:108C5000930407001306070093F707406386070A8B
:108C60009305060013050B00EFE0CF99130C0500E8
:108C7000630A050A8325040113060A00EF10403A2F
:108C80008357C40093F7F7B793E707082316F40058
:108C900033054C01338A4441232A940023244401A0
:108CA000232884012320A40093040900130A090047
:108CB00013060A0093850B00EF1040480327840039
:108CC0000325040083A78A00B304974033054501B8
:108CD000232494002320A4003389274123A42A01BC
:108CE0006304090603A9490083AB0900138A040041
:108CF00093898900E30809FEE37E99F09304090053
:108D0000130A09006FF0DFFA13050B00EF1000558E
:108D1000130C0500E31E05F68325040113050B0063
:108D2000EFB00FA19307C0002320FB008357C400BE
:108D30001305F0FF93E707042316F40023A40A00A9
:108D400023A20A006F00C00023A20A00130500003E
:108D50008320C102032481028324410203290102EA
:108D60008329C101032A8101832A4101032B0101C7
:108D7000832BC100032C81001301010367800000D5
:108D800083D7C500130101ED232C41112328611164
:108D90002320A111232611122324811223229112B0
:108DA00023202113232E3111232A5111232671113F
:108DB0002324811123229111232EB10F93F7070849
:108DC0002326D100138A0500130B0500130D06009E
:108DD0006386070083A70501E3860756B74701802E
:108DE000930AC104938707ACB74B0180B744018055
:108DF00023205105232401042322010413870A00A0
:108E00002328010023220102232401022326010238
:108E100023240100232AF100938BCBC29384C4C383
:108E200083470D006380072013040D009306500252
:108E30006386D7388347140013041400E39A07FEAF
:108E40003309A4416300A41F8326810483274104BE
:108E50002320A701B3862601938717002322270129
:108E60002324D1042322F104930670001307870002
:108E700063CEF6348326810083470400B38626013F
:108E80002324D1006380071A83461400130D1400B5
:108E9000A30D0102930CF0FF13040000930D0000DA
:108EA0001309A005130C90009309A002130D1D00D7
:108EB000938706FE6364F904032641019397270014
:108EC000B387C70083A7070067800700130400006B
:108ED000938706FD83460D00931524003384850097
:108EE0001314140033848700938706FD130D1D00AF
:108EF000E372FCFE938706FEE370F9FC63840612BE
:108F00002306D108A30D010213091000130C100051
:108F10009309C108930C000013FF2D0063040F0098
:108F20001309290013FE4D088327810403264104F9
:108F300063160E00B3062441E34AD0028346B10310
:108F40001305160093058700638006049306B1039A
:108F5000938717002320D700930610002322D70001
:108F60002324F1042322A10493067000E3CEA60C6F
:108F7000930F2600930607011306050013870500CB
:108F800013850F0093850600630C0F029306C1033F
:108F90002320D70093872700930620002322D700A1
:108FA0002324F1042322A10413077000E34CA70C2F
:108FB000130605001387050013051500938585002A
:108FC000930600086302DE60B38C8C416346906BAD
:108FD000B307FC0023203701232287012324F10457
:108FE0002322A104130770006342A77493F84D0075
:108FF00063860800330C24416348801F63542401B6
:109000001304090003278100330787002324E100AC
:10901000639E077283470D002322010413870A0011
:10902000E39407E083278104E392074C8357CA0047
:1090300093F70704E398074E8320C112032481129B
:109040000325810083244112032901128329C111C0
:10905000032A8111832A4111032B0111832BC11093
:10906000032C8110832C4110032D0110832DC10F7F
:10907000130101136780000013050B00232CE1008E
:10908000EFD0DFD683274500138507002326F102A2
:10909000EFF01FA09307050013050B002324F10236
:1090A000EFD0DFD403278500832781022322E1024A
:1090B00003278101E398071683460D006FF01FDF39
:1090C00083460D0093ED0D026FF05FDE93ED0D0111
:1090D00093F70D026382071E8327C10093897700EF
:1090E00093F989FF83A6490003AC0900938789009F
:1090F0002326F100138E060063C8061E9306F0FFB8
:1091000013890D006388DC00B366CC0113F9FDF709
:109110006384067AE31C0E0093069000E3E8860160
:1091200093070C03A307F10E930D0900130C100015
:109130009309F10E6F00C00693ED0D0193F70D0238
:10914000638607148327C1009389770093F989FF09
:1091500003AC090003AE4900938789002326F10080
:1091600013F9FDBF93060000A30D01021306F0FFE3
:109170006380CC1A3366CC01937DF9F76314065EE5
:1091800063980C3E639E0672137C19009309010FCD
:1091900063080C0093070003A307F10E9309F10E77
:1091A00013890C0063D48C0113090C008347B103AD
:1091B000B337F0003309F9006FF01FD63309A4412B
:1091C000E314A4C9834704006FF0DFCB1306010446
:1091D00093050A0013050B00EFF0DF9EE31805E48A
:1091E00013870A006FF01FC993060001032741048B
:1091F00063D08607930C0001930970006F00C000D4
:10920000130C0CFF63D68C05938707011307170017
:1092100023A0750123A295012324F1042322E10454
:1092200093858500E3DEE9FC1306010493050A003B
:1092300013050B00EFF01F99E31A05DE130C0CFF6A
:10924000832781040327410493850A00E3CE8CFB26
:10925000B38787011307170023A0750123A2850197
:109260002324F1042322E10493067000E3D8E6D816
:109270001306010493050A0013050B00EFF09F94F9
:10928000E31605DA832781046FF05FD70326C10058
:1092900093F70D01930646006392077E93F70D0442
:1092A000E38C07188327C100130E00002326D1008A
:1092B00003DC07006FF0DFEA0326C10093F70D011E
:1092C000930646006398077893F70D04E386071426
:1092D0008327C1002326D100039C0700135EFC41B5
:1092E00093060E00E3DC06E0B3368001330EC04186
:1092F000330EDE409306D002A30DD1021306F0FF19
:10930000330C804113890D0093061000E394CCE6E2
:1093100013061000E380C6E0130620006384C6260F
:109320009309010F1316DE0193767C0093573C00DE
:1093300093860603336CF600135E3E00A38FD9FEBE
:109340003366CC01938509009389F9FFE31C06FC81
:10935000937719006382072693070003638EF62430
:109360009385E5FFA38FF9FE9307010F338CB74078
:10937000930D0900938905006FF09FE28327C100D8
:10938000A30D010283A9070093864700E386090421
:109390009307F0FF6388FC7813860C0093050000A8
:1093A00013850900232CD1002326E100EFE00FA153
:1093B0000327C10083268101E3040514330C3541E2
:1093C0002326D100930C00006FF09FDD8326C1009F
:1093D000A30D01021309100083A70600938646001F
:1093E0002326D1002306F108130C10009309C108AD
:1093F0006FF05FB28327C10013E92D00B786FFFF2E
:1094000003AC0700B73D01809387470093C60683EE
:109410002326F10093870D4F231ED102130E000067
:109420002328F100930620006FF01FD40326C1000B
:1094300093F70D0283260600130646002326C1007B
:109440006390076093F70D016392077893F70D041B
:10945000E398070893F80D20638A08768327810034
:109460002380F6006FF0DF9B83460D0093ED0D081F
:109470006FF0DFA383460D0093051D00E38A360BD2
:10948000938706FD138D0500930C0000E362FCA298
:1094900083460D0093952C0033839501131313001D
:1094A000B30CF300938706FD130D1D00E372FCFE61
:1094B0006FF01FA083460D0093ED4D006FF01F9FCE
:1094C0009307B00283460D00A30DF1026FF01F9EBB
:1094D0008327C10083460D0003A40700938747003C
:1094E0002326F100E354049C3304804093ED4D00A7
:1094F0006FF0DF9B83460D0093ED1D006FF01F9B07
:109500008347B10383460D00E392079A9307000255
:10951000A30DF1026FF09F9983460D009307C006DB
:109520006388F66693ED0D016FF05F9883460D003A
:10953000930780066386F66493ED0D046FF01F9722
:1095400013E90D0193770902638407388327C1006B
:10955000930610009389770093F989FF9387890018
:1095600003AC090003AE49002326F1006FF0DFBF12
:1095700013061000638EC6781306200013890D00B1
:10958000E390C6DA9309010F832701019376FC006B
:109590009389F9FFB386D70003C6060093574C00A2
:1095A0009316CE0133ECF600135E4E002380C90003
:1095B000B366CC01E39A06FC9307010F338C374165
:1095C000930D09006FF0DFBDB3062441E35ED09E2A
:1095D000130E00016352DE74130F70006F00C000A1
:1095E000938606FF635EDE04938707011306160069
:1095F000232097002322C7012324F1042322C1043E
:1096000013078700E35ECFFC1306010493050A00ED
:1096100013050B00232CD100EFF0CFDAE31805A0DF
:1096200083268101130E000183278104938606FFA0
:109630000326410413870A00130F7000E346DEFA85
:1096400013061600130E8700B387D7002320970058
:109650002322D7002324F1042322C104130770001E
:109660006340C754B38C8C411305160093058E00DC
:1096700013070E00E35E909513030001635C935F94
:10968000130E70006F00C000938C0CFF635A93059B
:1096900093870701130616002320970023226700F3
:1096A0002324F1042322C10413078700E35ECEFCC8
:1096B0001306010493050A0013050B00EFF08FD089
:1096C000E316059613030001938C0CFF8327810496
:1096D0000326410413870A00130E7000E34A93FB2C
:1096E0001305160013068700B38797012320970000
:1096F000232297012324F1042322A10413077000DD
:109700006340A7201307060013051500B307FC00EC
:1097100023203701232287012324F1042322A104DB
:109720001307700093058600E352A78C130601040B
:1097300093050A0013050B00EFF0CFC8E318058E60
:109740008327810493850A006FF05F8A1306010462
:1097500093050A0013050B00EFF0CFC6E30C058A52
:109760006FF0DF8C13890D006FF09FBA9305000135
:1097700063D0D508930F0001930270006F00C00002
:10978000938606FF63D6DF0693870701130616004C
:10979000232077012322F7012324F1042322C1048B
:1097A00013078700E3DEC2FC1306010493050A00D9
:1097B00013050B002320D102232EC101232CE1012C
:1097C000EFF04FC0E314058683260102930F0001DA
:1097D00083278104938606FF03264104032EC101DB
:1097E000032F810113870A0093027000E3CEDFF894
:1097F000B387D700130616002322D7002320770152
:109800002324F1042322C104930670001307870068
:1098100063D6C6F21306010493050A0013050B0074
:10982000232EC101232CE101EFF0CFB9E310058015
:109830008327810403264104032EC101032F8101E4
:1098400013870A006FF08FEF1306010493050A00D7
:1098500013050B00232EC101232CE101EFF08FB67D
:10986000631605FC0326410483278104032EC101EE
:10987000032F8101930541051305160013870A0084
:109880006FF08FF01306010493050A0013050B0017
:10989000232CC101EFF00FB3631A05F8032641042E
:1098A00083278104032E81019305410513051600CA
:1098B00013870A006FF0CFF0E3940C86930D090034
:1098C000930C0000130C00009309010F6FF05F8DE3
:1098D0000326C10093770901930646006396071893
:1098E00093770904638807368327C100130E0000AD
:1098F0002326D10003DC0700930610006FF0DF86FB
:109900001306010493050A0013050B00EFF08FAB5B
:10991000631E05F003254104832781049305410557
:109920001305150013870A006FF08FEA937709403B
:109930002320F102930D00009309010F6F004003F3
:1099400093050E001306A0009306000013050C00FB
:10995000232EE100232CC101EF40003E032E8101A4
:109960000327C101630C0E30130C0500138E050094
:1099700093050E001306A0009306000013050C00CB
:10998000232EE100232CC101EF40407E83270102FA
:1099900013050503A38FA9FE032E81010327C1012F
:1099A0009389F9FF938D1D00E38C07F8832741020B
:1099B00083C60700E396B6F99307F00FE382FDF83C
:1099C00063160E0093079000E3F887BF8327810298
:1099D0008325C102232EC101B389F94013860700F4
:1099E00013850900232CE100EFF04F930327410278
:1099F000032EC1011306A000834517009306000043
:109A000013050C00B337B000B307F70093050E0041
:109A10002322F102EF40403203278101930D000021
:109A20006FF09FF48327410283460D00638007C8CF
:109A300083C70700638C07C693ED0D406FF00FC717
:109A4000032681009357F64123A0C60023A2F60007
:109A50006FF00FBD032C06002326D100135EFC41DE
:109A600093060E006FF04FE92326D100032C060069
:109A7000130E0000930610006FF00FEF032C06008A
:109A8000130E00002326D1006FF08FED13890D0017
:109A90006FF05FABB7370180938747502328F10001
:109AA00093F70D02638007068327C100938977002F
:109AB00093F989FF03AC090003AE4900938789003D
:109AC0002326F10013F61D00630E06003366CC0159
:109AD000630A060013060003230EC102A30ED1027F
:109AE00093ED2D0013F9FDBF930620006FF0CFE733
:109AF000B73701809387074F2328F10093F70D02B2
:109B0000E39407FA8325C10093F70D0113864500FE
:109B1000638A070403AC0500130E00002326C1006E
:109B20006FF05FFA13850900232CE1002326D10092
:109B3000EFE01FF603278101130C0500930C0000D2
:109B40006FF00FE693050004EFD0CFAB2320AA00FF
:109B50002328AA006300052093070004232AFA00A3
:109B60006FF0CFA793F70D04638A07088327C1001E
:109B7000130E00002326C10003DC07006FF09FF4E2
:109B800083461D0093ED0D20130D1D006FF00FB2E5
:109B900083461D0093ED0D02130D1D006FF00FB1F4
:109BA0001306010493050A0013050B00EFF08F81E3
:109BB000631E05C6032641048327810493054105DE
:109BC0001305160013870A006FF00FC0832781006A
:109BD00023A0F6006FF0CFA493076000138C0C0055
:109BE00063F49701130C6000B73E018013090C0069
:109BF0002326D10093898E516FF0CFB193F70D20BA
:109C00006386070C8327C100130E00002326C100C2
:109C100003CC07006FF01FEB93F70D20638C070850
:109C20008327C1002326D100038C0700135EFC416B
:109C300093060E006FF04FCC93F70D20638207065A
:109C40008327C100130E00002326D10003CC070098
:109C50006FF00FD193770920638807028327C10033
:109C6000130E00002326D10003CC0700930610003A
:109C70006FF08FCF138605006FF01FA7930790003A
:109C8000E3E487CF6FF05F938327C100130E0000DA
:109C90002326D10003AC0700930610006FF0CFCC51
:109CA0008327C100130E00002326D10003AC070058
:109CB0006FF00FCB8327C1002326D10003AC070030
:109CC000135EFC4193060E006FF00FC38327C100A3
:109CD000130E00002326C10003AC07006FF09FDEC7
:109CE000832781002390F6006FF08F931306010401
:109CF00093050A0013050B00EFE0DFEC6FF00FB3E4
:109D0000138C0C002326D100930C00006FF04FC978
:109D100013890D006FF0CFC0138E050013060500E8
:109D20006FF09F929307F0FF2324F1006FF0CFB004
:109D30008327C10083AC07009387470063D40C00DE
:109D4000930CF0FF83461D002326F100138D0500C0
:109D50006FF0CF959307C0002320FB009307F0FF1F
:109D60002324F1006FF04FADB767018003A747A729
:109D7000130101FF93870600130806002326110034
:109D80008328C70093060500138705001386070084
:109D900063000802B74701809387C7C4B7450180B5
:109DA0009385C5C513850800EF004011EF204012D0
:109DB000373801809307882F1308882F6FF01FFE14
:109DC000130101FF9306060013060000232611006D
:109DD000EFF09FF9B385C502130101FF2324810031
:109DE00023261100EFD00F8213040500630805023B
:109DF0000326C5FF130740021376C6FF1306C6FFEE
:109E00006360C706930630019307050063E2C6024C
:109E100023A0070023A2070023A407008320C1007A
:109E20001305040003248100130101016780000071
:109E300023200500232205009307B00163F0C70427
:109E4000232405002326050093070501E312E6FC01
:109E50002328050093078501232A05006FF05FFB87
:109E600093050000EF605FF08320C100130504003C
:109E7000032481001301010167800000930785001E
:109E80006FF01FF9130101FC1303C1022326D10255
:109E900093060300232E11002328E102232AF10256
:109EA000232C0103232E110323266100EF00D03A57
:109EB0008320C1011301010467800000130E050017
:109EC00037650180130101FC032545A713038102B7
:109ED0002324C1022326D102138605009306030022
:109EE00093050E00232E11002328E102232AF102FC
:109EF000232C0103232E110323266100EF00D0350C
:109F00008320C1011301010467800000130101FFD8
:109F1000232611002324810023229100630C0602D2
:109F2000B7450180938505C9130506001304060093
:109F3000EF00500AB7440180631205021385C4C8BC
:109F40008320C10003248100832441001301010107
:109F500067800000B74401806FF05FFE9385C4C83E
:109F600013050400EF001007E30A05FCB735018074
:109F70009385852F13050400EF00D005E30005FC51
:109F8000130500006FF0DFFBB767018003C507A171
:109F9000678000003767018093070500032547A706
:109FA00013860500938507006FF05FF6B7670180A1
:109FB00003A3C79C670003006380050263020604D5
:109FC000638806048347060023A0F50003450600C6
:109FD0003335A00067800000130101FF9305C10025
:109FE00063040602638A06028347060023A0F50085
:109FF000034506003335A00013010101678000000E
:10A000001305000067800000130500006FF0DFFEFD
:10A010001305E0FF678000001305E0FF6FF0DFFD30
:10A02000B3C7A50093F73700B308C50063920706CE
:10A030009307300063FEC7049377350013070500CC
:10A040006398070613F6C8FF930706FE636CF708CC
:10A05000637CC702938605009307070003A80600E8
:10A06000938747009386460023AE07FFE3E8C7FEC9
:10A070009307F6FFB387E74093F7C7FF938747003F
:10A080003307F700B385F5006368170167800000A8
:10A0900013070500E37C15FF83C7050013071700AE
:10A0A00093851500A30FF7FEE36817FF6780000094
:10A0B00083C605001307170093773700A30FD7FE59
:10A0C00093851500E38007F883C605001307170082
:10A0D00093773700A30FD7FE93851500E39A07FC0B
:10A0E0006FF05FF683A6450083A2050083AF85006D
:10A0F00003AFC50083AE050103AE450103A385018F
:10A1000003A8C5012322D70083A6050223205700F8
:10A110002324F7012326E7012328D701232AC70197
:10A12000232C6700232E07012320D70213074702A1
:10A1300093854502E368F7FA6FF09FF163F6A50295
:10A14000B387C5006372F5023307C500630A060EC4
:10A1500083C6F7FF9387F7FF1307F7FF2300D700A6
:10A16000E398F5FE678000009307F00063E8C702FC
:10A17000930705009306F6FF630C060C9386160002
:10A18000B386D70003C70500938717009385150092
:10A19000A38FE7FEE398D7FE67800000B3E7A50032
:10A1A00093F737006390070A930806FF93F808FFB8
:10A1B00093880801330815011387050093070500EC
:10A1C00083260700130707019387070123A8D7FEFB
:10A1D000832647FF23AAD7FE832687FF23ACD7FE1B
:10A1E0008326C7FF23AED7FEE31CF8FC1377C60017
:10A1F000B38515011378F600630E07041387050075
:10A2000093880700130E300003230700130747004D
:10A21000B306E84023A06800B386D50093884800C1
:10A22000E364DEFE1307C8FF1377C7FF1307470079
:10A2300013763600B387E700B385E5006FF09FF330
:10A24000678000009306F6FF930705006FF01FF389
:10A2500067800000130608006FF0DFF1130101FDB5
:10A260002320210323261102232481022322910289
:10A27000232E3101232C4101232A5101232861017E
:10A28000232671012324810113090600638405221A
:10A290001384050093090500EFD08FBF9304B90024
:10A2A0009307600163FE970E93F484FF1387040005
:10A2B00063CE040E63EC240F8327C4FF930A84FF4C
:10A2C00013FAC7FF338B4A01635CEA18B756018063
:10A2D000938B064E03A68B0083264B00630E6623EA
:10A2E00013F6E6FF3306CB0003264600137616006E
:10A2F0006314061A93F6C6FF3306DA00635EE6328D
:10A3000093F7170063940702032C84FF338C8A4170
:10A3100083274C0093F7C7FFB386D700B38B460162
:10A3200063DAEB34B30BFA0063D2EB0C930509004C
:10A3300013850900EFC01FAD13090500630C050468
:10A340008327C4FF130785FF93F7E7FFB387FA005E
:10A350006382E7301306CAFF9307400263E6C73003
:10A360001307300183260400636CC726930705009A
:10A370001307040023A0D7008326470023A2D70099
:10A380000327870023A4E700930504001385090031
:10A39000EF901FBA13850900EFD0CFAF6F00C00157
:10A3A0009304000113070001E3F824F19307C000B0
:10A3B00023A0F900130900008320C10203248102B5
:10A3C000832441028329C101032A8101832A410197
:10A3D000032B0101832BC100032C8100130509000D
:10A3E0000329010213010103678000008327CC00C9
:10A3F00003278C001306CAFF930640022326F700AA
:10A4000023A4E70013098C00330B7C0163E4C62E00
:10A4100093053001032704009307090063F2C50286
:10A420002324EC00032744009307B0012326EC000B
:10A4300063E2C7300327840093070C0113048400F0
:10A4400023A0E70003274400138A0B00930A0C00A3
:10A4500023A2E700032784001304090023A4E700D4
:10A4600083A74A0033079A409306F00093F717003A
:10A4700063ECE606B367FA0023A2FA0083274B00D9
:10A4800093E717002322FB0013850900EFD08FA06C
:10A49000130904006FF05FF293F71700E39807E8E1
:10A4A000032C84FF338C8A4183274C0093F7C7FF2A
:10A4B0006FF05FE7032481028320C10283244102FD
:10A4C000032901028329C101032A8101832A410151
:10A4D000032B0101832BC100032C8100930506008F
:10A4E000130101036FC01F92B3E7970023A2FA0084
:10A4F000B3859A001367170023A2E50083274B005A
:10A50000938585001385090093E717002322FB003C
:10A51000EF901FA26FF05FF793F6C6FF3306DA00E5
:10A52000938504016350B60E93F71700E39007E09C
:10A53000032C84FF338C8A4183274C0093F7C7FF99
:10A54000B386D700338B4601E34EBBDC8327CC00B8
:10A5500003278C001306CAFF930640022326F70048
:10A5600023A4E70013098C0063EEC6209305300195
:10A57000032704009307090063F2C5022324EC00BB
:10A58000032744009307B0012326EC0063E4C720AF
:10A590000327840093070C011304840023A0E70021
:10A5A0000327440023A2E7000327840023A4E70035
:10A5B00033079C00B3079B4023A4EB0093E71700ED
:10A5C0002322F70083274C001385090093F7170017
:10A5D000B3E4970023229C00EFD0CF8B6FF0DFDD38
:10A5E0002320D500832644001307B0012322D50081
:10A5F0006360C712832684001307840093078500D5
:10A600006FF05FD7B38A9A00B307964023A45B012B
:10A6100093E7170023A2FA008327C4FF13850900DC
:10A620001309040093F71700B3E49700232E94FE58
:10A63000EFD04F866FF05FD88327CB0003278B00C6
:10A64000130A0600338BCA002326F70023A4E70071
:10A650006FF01FE18327C5FF93F7C7FF330AFA00A6
:10A66000338B4A016FF0DFDF93050400EFF01FAD7D
:10A670006FF09FD18327CB0003278B001306CAFFFF
:10A68000930640022326F70023A4E70003278C004B
:10A690008327CC0013098C00330B7C012326F700A1
:10A6A00023A4E70063E8C6049306300103270400EF
:10A6B00093070900E3F6C6D82324EC0003274400DF
:10A6C0009307B0012326EC0003278400E3F6C7D6E6
:10A6D0002328EC000327C40093074002232AEC0040
:10A6E000032704016304F60693078C011304040195
:10A6F0006FF01FD59305040013050900EFF01FA4A8
:10A7000013040900138A0B00930A0C006FF05FD545
:10A71000032784002324E5000327C4002326E50043
:10A72000832604016302F60413070401930705015D
:10A730006FF05FC4832784002328FC008327C400B4
:10A74000232AFC0003270401E310D6FA232CEC0093
:10A750000327440193070C0213048401232EEC0009
:10A76000032704006FF0DFCD2328D50083264401A2
:10A770001307840193078501232AD50083268401CA
:10A780006FF05FBF9305040013050900EFF01F9BF6
:10A790006FF01FE2832784002328FC008327C40076
:10A7A000232AFC00032704016308D60093078C01C9
:10A7B000130404016FF09FDE232CEC0003274401F7
:10A7C00093070C0213048401232EEC0003270400DA
:10A7D0006FF0DFDC3367B5009303F0FF13773700CA
:10A7E00063100710B7877F7F9387F7F7032605006D
:10A7F00083A60500B372F6003363F600B382F2005D
:10A80000B3E26200639272106316D6080326450015
:10A8100083A64500B372F6003363F600B382F200FC
:10A82000B3E26200639E720C6316D60603268500AF
:10A8300083A68500B372F6003363F600B382F2009C
:10A84000B3E262006398720C6316D6040326C50057
:10A8500083A6C500B372F6003363F600B382F2003C
:10A86000B3E262006392720C6316D60203260501FE
:10A8700083A60501B372F6003363F600B382F200DB
:10A88000B3E26200639C720A13054501938545019A
:10A89000E30ED6F41317060193970601631EF70023
:10A8A0001357060193D706013305F7409375F50F4B
:10A8B00063900502678000001357070193D70701D3
:10A8C0003305F7409375F50F63940500678000002A
:10A8D0001377F70F93F7F70F3305F7406780000002
:10A8E0000346050083C60500130515009385150072
:10A8F0006314D600E31606FE3305D64067800000D9
:10A900001305450093854500E31CD6FC13050000A4
:10A91000678000001305850093858500E312D6FC4F
:10A9200013050000678000001305C5009385C5006E
:10A93000E318D6FA1305000067800000130505012F
:10A9400093850501E31ED6F813050000678000001B
:10A9500083A74506130101FD232861012326110267
:10A96000232481022322910223202103232E31015B
:10A97000232C4101232A5101232671012324810123
:10A9800013972701130B06006358070A83278600D5
:10A99000832B06001389050093090500930AF0FF35
:10A9A0006388070803AC4B0003A40B00135A2C0068
:10A9B00063060A06930400006F00C00013044400FD
:10A9C000630C9A048325040013060900138509000B
:10A9D000EF10504993841400E31255FF1305F0FF64
:10A9E0008320C1020324810223240B0023220B00B5
:10A9F00083244102032901028329C101032A810121
:10AA0000832A4101032B0101832BC100032C810008
:10AA1000130101036780000083278B00137CCCFFA8
:10AA2000B38787412324FB00938B8B00E39C07F6BD
:10AA3000130500006FF0DFFAEF10904D6FF05FFA32
:10AA400003278600630407006FF09FF023220600AF
:10AA50001305000067800000130101ED232E311162
:10AA6000232A51112320A1112326111223248112FC
:10AA70002322911223202113232C41112328611119
:10AA8000232671112324811123229111232EB10F2A
:10AA90002326D100930A050093890500130D0600B3
:10AAA00063060500832785036388076A0397C90047
:10AAB000931707019316270193D7070163CA06026C
:10AAC000B727000083A64906B367F70093970701ED
:10AAD00037E7FFFF93D707411307F7FF33F7E60088
:10AAE0002396F9009397070123A2E90693D707015C
:10AAF00013F787006304073E03A709016300073EBD
:10AB000093F7A7011307A000638AE73EB7470180C8
:10AB10009304C1049387C7C9B74B018037490180AB
:10AB20002320910423240104232201041387040019
:10AB300023280100232201022324010223260102EB
:10AB400023240100232AF100938B8BE0130989E170
:10AB500083470D00638E072413040D0093065002F3
:10AB60006386D7428347140013041400E39A07FE58
:10AB7000330AA441630EA42383268104832741045E
:10AB80002320A701B306DA00938717002322470189
:10AB90002324D1042322F104130670001307870035
:10ABA0006350F602E3840636130601049385090018
:10ABB00013850A00EFF0DFD9631005201387040026
:10ABC0008326810083470400B38646012324D100F5
:10ABD0006380071E83461400130D1400A30D0102A9
:10ABE000930CF0FF13040000930D0000130AA0055E
:10ABF000130C9000130BA002130D1D00938706FE8B
:10AC00006364FA040326410193972700B387C700C2
:10AC100083A707006780070013040000938706FDE1
:10AC200083460D009315240033848500131414000B
:10AC300033848700938706FD130D1D00E372FCFE2D
:10AC4000938706FEE370FAFC638406162306D10898
:10AC5000A30D0102130A1000130C1000130BC108FE
:10AC6000930C000093FF2D0063840F00130A2A0049
:10AC70008326410413FF4D088327810413861600A1
:10AC80009305060063160F0033084441E3440017A0
:10AC90000345B10313068700630C05029306B10355
:10ACA0002320D70093871700930610002322D70094
:10ACB0002324F1042322B10413077000E342B70CEC
:10ACC000938605001307060093851500130686007A
:10ACD000638E0F049306C1032320D70093872700B8
:10ACE000930620002322D7002324F1042322B10459
:10ACF00013077000E352B70EE3840726130601041E
:10AD00009385090013850A00232CE101EFF05FC44D
:10AD10006314050A8326410483278104032F8101DC
:10AD200013064105938516001387040013050008D8
:10AD30006306AF68B38C8C4163429077B307FC0025
:10AD400023206701232287012324F1042322B10455
:10AD5000130770006352B7026382072413060104CD
:10AD60009385090013850A00EFF09FBE6316050462
:10AD7000832781041386040093FE4D0063860E0032
:10AD8000330C4441634880236354440113040A0094
:10AD900003278100330787002324E100639E077A9D
:10ADA00083470D002322010413870400E39607DA8A
:10ADB00083278104E396076283D7C90093F70704CA
:10ADC000E39E07648320C1120324811203258100BE
:10ADD00083244112032901128329C111032A8111FD
:10ADE000832A4111032B0111832BC110032C8110E5
:10ADF000832C4110032D0110832DC10F130101136A
:10AE00006780000013850A00232CE100EFB01FFECD
:10AE100083274500138507002326F102EFD05FC783
:10AE20009307050013850A002324F102EFB01FFCED
:10AE300003278500832781022322E1020327810162
:10AE4000E398072A83460D006FF01FDB83460D0051
:10AE500093ED0D026FF05FDA93ED0D0193F70D02A4
:10AE6000638A07228327C100138B7700137B8BFF34
:10AE700083264B00032C0B0093078B002326F10045
:10AE80001388060063C006249306F0FF138A0D00A2
:10AE90006388DC00B3660C0113FAFDF7E38E060647
:10AEA000E318081293069000E3E4861393070C035B
:10AEB000A307F10E930D0A00130C1000130BF10EF3
:10AEC000138A0C0063D48C01130A0C008347B1036E
:10AED000B337F000330AFA006FF0DFD8938509002A
:10AEE00013850A00EF00D068E31A055283D7C90022
:10AEF0001307A00093F7A701E39AE7C08397E9003F
:10AF0000E3C607C08326C10013060D009385090020
:10AF100013850A00EF0010562324A1006FF09FEA6A
:10AF200093ED0D0193F70D02638007148327C10091
:10AF3000138B7700137B8BFF032C0B0003284B0034
:10AF400093078B002326F10013FAFDBF9306000040
:10AF5000A30D01021306F0FF638ACC1833660C01BF
:10AF6000937DFAF76314066863960C3E639A067A3B
:10AF7000137C1A00130B010FE3040CF49307000376
:10AF8000A307F10E130BF10E6FF09FF3330AA441E8
:10AF9000E314A4BF834704006FF09FC3232201047E
:10AFA00093FE4D0063800E72330C4441635C8071EC
:10AFB000138604001307000183264104E3588745E4
:10AFC000930C0001130B70006F0080019385260025
:10AFD0001306860093060700130C0CFF63D88C053C
:10AFE00093870701138716002320760123229601F9
:10AFF0002324F1042322E104E35AEBFC6388073A9B
:10B00000130601049385090013850A00EFF05F948D
:10B01000E31405DA83264104130C0CFF8327810413
:10B020001386040093851600E3CC8CFBB38787015D
:10B0300023207601232286012324F1042322B10454
:10B0400013077000E352B7D4638E0766130601043A
:10B050009385090013850A00EFF09F8FE31E05D446
:10B06000832781046FF05FD20326C10093F70D019F
:10B0700093064600E390070C93F70D04E38E072434
:10B080008327C100130800002326D10003DC07003A
:10B090006FF09FEB0326C10093F70D019306460066
:10B0A000E390070893F70D04E38807208327C10086
:10B0B0002326D100039C07001358FC419306080087
:10B0C000E3D406DCB3368001330800413308D840AE
:10B0D0009306D002A30DD1021306F0FF330C80417A
:10B0E000138A0D0093061000E39ACCE613061000B5
:10B0F000E388C6DA130620006388C626130B010F07
:10B100001316D80193767C0093573C009386060370
:10B11000336CF60013583800A30FDBFE33660C01C6
:10B1200093050B00130BFBFFE31C06FC93771A003F
:10B1300063860726930700036382F6269385E5FF5F
:10B14000A30FFBFE9307010F338CB740930D0A004A
:10B15000138B05006FF0DFD6EF1080396FF01F956D
:10B160008327C100A30D010203AB070093864700AC
:10B17000E3040B129307F0FFE38CFC0613860C002C
:10B180009305000013050B00232CD1002326E100BA
:10B19000EFC0CFC20327C10083268101E30C052441
:10B1A000330C65412326D100930C00006FF05FD172
:10B1B0008326C100A30D0102130A100083A7060015
:10B1C000938646002326D1002306F108130C1000B5
:10B1D000130BC1086FF0DFA883460D009307C0066C
:10B1E000E38EF60893ED0D016FF01FA183460D006D
:10B1F00093078006E38CF60693ED0D046FF0DF9F56
:10B2000013EA0D0193770A02638407528327C10072
:10B2100093061000138B7700137B8BFF93078B0033
:10B22000032C0B0003284B002326F1006FF05FD2A4
:10B2300083460D0093ED0D086FF01F9C8327C1001E
:10B2400013EA2D00B786FFFF03AC0700B73D01806E
:10B250009387470093C606832326F10093870D4FFB
:10B26000231ED102130800002328F10093062000BA
:10B270006FF01FCE0326C10093F70D028326060050
:10B28000130646002326C1006392076893F70D0159
:10B29000639E077E93F70D04E392070E93FE0D2045
:10B2A00063860E7E832781002380F6006FF05F8A1D
:10B2B0008327C10083460D0003A40700938747003E
:10B2C0002326F100E35A04923304804093ED4D00AD
:10B2D0006FF09F9283460D0093ED1D006FF0DF919C
:10B2E0008347B10383460D00E3980790930700025C
:10B2F000A30DF1026FF05F9083460D0093ED4D00BA
:10B300006FF09F8F9307B00283460D00A30DF102EB
:10B310006FF09F8E83460D0093051D00E38C661130
:10B32000938706FD138D0500930C0000E368FC8CE9
:10B3300083460D0013982C00330898011318180049
:10B34000B30CF800938706FD130D1D00E372FCFE9D
:10B350006FF0DF8A13061000E38EC60A1306200082
:10B36000138A0D00E39CC6D8130B010F832701013C
:10B370009376FC00130BFBFFB386D70003C60600D1
:10B3800093574C009316C80133ECF600135848004D
:10B390002300CB00B3660C01E39A06FC9307010F70
:10B3A000338C6741930D0A006FF09FB19305100035
:10B3B00093060000138604006FF01FC23308444157
:10B3C000E35A009713050001E3500507130F00012E
:10B3D000930F70006F00800113852600130787000C
:10B3E00093060600130808FF63500F0793870701B1
:10B3F00013861600232027012322E7012324F104CA
:10B400002322C104E3DACFFC638407161306010488
:10B410009385090013850A00232C0101EFF04FD317
:10B42000E31C05980328810183264104130F0001C2
:10B43000130808FF8327810413870400138516006F
:10B44000930F7000E3440FFB130F8700B3870701CE
:10B4500023202701232207012324F1042322A1040E
:10B46000130770006352A746638E076C130601042E
:10B470009385090013850A00EFF08FCDE31E059236
:10B4800083264104B38C8C41832781041306410534
:10B490009385160013870400E352908B1305000177
:10B4A0006358956913030001130F70006F0080014A
:10B4B000938526001307870093060600938C0CFFE4
:10B4C000635C9305938707011386160023202701E9
:10B4D000232267002324F1042322C104E35ACFFC72
:10B4E00063840706130601049385090013850A0087
:10B4F000EFF00FC6E312058C83264104130300010D
:10B50000938C0CFF83278104138704009385160016
:10B51000130F7000E34893FB93068700B3879701EE
:10B5200023202701232297012324F1042322B1049D
:10B53000130770006344B71A9385150013868600BD
:10B54000138706006FF08FFF93051000930600002D
:10B55000138704006FF09FF613060104938509001A
:10B5600013850A00EFF0CFBEE30C05826FF0DF8495
:10B570001305100093060000138704006FF09FE688
:10B58000638A071E130601049385090013850A00C8
:10B59000232EE101232CF101EFF08FBBE31E058088
:10B5A0008326410483278104032FC101832F810156
:10B5B0001306410593851600138704006FF04FF1C1
:10B5C0009307C1032326F104930720002328F104E5
:10B5D0009305100013064105938605001307060026
:10B5E00093851600130687006FF04FF4138A0D0041
:10B5F0006FF0DFAF9305000163D605619302000190
:10B60000930370006F00C0011385260013078700A5
:10B6100093060600130808FF63D802071386160076
:10B620009387070123207701232257002324F10465
:10B630002322C104E3DAC3FC638E07061306010468
:10B640009385090013850A0023200103232EE101BD
:10B65000232CF101EFF0CFAF631005F603280102B0
:10B660008326410493020001130808FF8327810405
:10B67000032FC101832F8101138704001385160056
:10B6800093037000E3CC02F9B3870701232077010D
:10B69000232207012324F1042322A104930670002E
:10B6A00063CAA60E130787009305150093060500CD
:10B6B0006FF00FDE930600001305100013870400DF
:10B6C0006FF05FF56354440113040A00832781007F
:10B6D000B38787002324F1006FF08FEC638A07346F
:10B6E000130601049385090013850A00EFF04FA6A5
:10B6F000631405EC83254104832781041306410567
:10B7000093851500138704006FF04FE32322010493
:10B71000138704006FF0CFCA639A0CF8930D0A00E8
:10B72000930C0000130C0000130B010F6FF04FF986
:10B730000326C10093770A01930646006390071A17
:10B7400093770A046386073C8327C100130800002F
:10B750002326D10003DC0700930610006FF04FFF93
:10B76000130641059305100093060000138704009B
:10B770006FF0CFDB63880F1C9307C1032326F1040E
:10B78000930720002328F1049306100013074105B6
:10B790006FF01FE5638E07261306010493850900E9
:10B7A00013850A00232EE101232CF101EFF04F9ABB
:10B7B000631405E08326410483278104032FC1011C
:10B7C000832F810113870400938516006FF04FCCFF
:10B7D00093770A402320F102930D0000130B010F11
:10B7E0006F004003930508001306A00093060000B5
:10B7F00013050C00232EE100232C0101EF20C05380
:10B80000032881010327C10163080832130C0500D6
:10B8100013880500930508001306A0009306000096
:10B8200013050C00232EE100232C0101EF2010143E
:10B830008327010213050503A30FABFE0328810133
:10B840000327C101130BFBFF938D1D00E38C07F849
:10B850008327410283C60700E396B6F99307F00FEA
:10B86000E382FDF86316080093079000E3F887B3BE
:10B87000832781028325C102232E0101330BFB4064
:10B880001386070013050B00232CE100EFD00FA94E
:10B89000032741020328C1011306A00083451700B6
:10B8A0009306000013050C00B337B000B307F70090
:10B8B000930508002322F102EF20004803278101AD
:10B8C000930D00006FF09FF49305150013068F0091
:10B8D0009306050013070F006FF0CFC52326D10094
:10B8E000032C060013080000930610006FF04FE6CB
:10B8F0008327410283460D00638007B083C707009A
:10B90000638C07AE93ED0D406FF00FAF03268100FF
:10B910009357F64123A0C60023A2F6006FF04FA371
:10B92000032C06002326D1001358FC41930608007F
:10B930006FF04FD5032C0600130800002326D1001A
:10B940006FF08FE093060000130641059305100089
:10B95000138704006FF08FBDB7370180938747507E
:10B960002328F10093F70D02638407068327C100A3
:10B97000138B7700137B8BFF032C0B0003284B00EA
:10B9800093078B002326F10013F61D00630E0600BB
:10B9900033660C01630A060013060003230EC1027E
:10B9A000A30ED10293ED2D0013FAFDBF93062000E4
:10B9B0006FF00FDA138A0D006FF0DF84B737018064
:10B9C0009387074F2328F10093F70D02E39007FABE
:10B9D0008325C10093F70D0113864500638A07068E
:10B9E00003AC0500130800002326C1006FF0DFF947
:10B9F00013050B00232CE1002326D100EFD04F8943
:10BA000003278101130C0500930C00006FF04FCB4E
:10BA10000347B10363160714E3940FBA93060000BB
:10BA20009305100013064105138704006FF00FB053
:10BA30001307100093070C002326610523288105B6
:10BA4000232481052322E104130641056FF0CFB2C0
:10BA500093F70D046380070A8327C10013080000D1
:10BA60002326C10003DC07006FF01FF283461D0090
:10BA700093ED0D20130D1D006FF00F9883461D00F0
:10BA800093ED0D02130D1D006FF00F9783278100BA
:10BA900023A0F6006FF0CF8B93076000138C0C008F
:10BAA00063EC970BB7380180130A0C002326D100F2
:10BAB000138B88516FF0CF9A93F70D206386071090
:10BAC0008327C1002326D100038C07001358FC41B3
:10BAD000930608006FF00FBB93F70D20638C070CE3
:10BAE0008327C100130800002326D10003CC0700E0
:10BAF0006FF08FC593F70D206384070A8327C10079
:10BB0000130800002326C10003CC07006FF0DFE715
:10BB100093770A20638A07068327C1001308000071
:10BB20002326D10003CC0700930610006FF04FC20C
:10BB3000930606006FF09F9E93079000E3E887CD81
:10BB40006FF0DF8513064105930510009306000092
:10BB5000138704006FF00F9E130C60006FF09FF4CA
:10BB60009307B1032326F104930710002328F1045F
:10BB700093051000130641056FF08F948327810011
:10BB80002390F6006FE0DFFC8327C100130800005C
:10BB90002326D10003AC0700930610006FF04FBBC3
:10BBA0008327C100130800002326C10003AC07004F
:10BBB0006FF09FDD8327C100130800002326D1000A
:10BBC00003AC07006FF04FB88327C1002326D100D4
:10BBD00003AC07001358FC41930608006FF08FAACE
:10BBE000130601049385090013850A00EFE05FD670
:10BBF0006FF08F9C138C0C002326D100930C000057
:10BC00006FF00FAC130506006FF01FA893851600A8
:10BC10006FF0CFC1138A0D006FF04FA99307F0FFAB
:10BC20002324F1006FF00F9A130F0600138505000F
:10BC30006FF0DF818327C10083AC07009387470043
:10BC400063D40C00930CF0FF83461D002326F10003
:10BC5000138D05006FE05FFA3767018093070500D9
:10BC6000032547A793060600138605009385070062
:10BC70006FE09FDE83D7C50003AE450603D3E50022
:10BC800083A8C50103A84502130101B893F7D7FFA4
:10BC900013070040232C8146231AF100138405006A
:10BCA0009307010793058100232A91462328214702
:10BCB000232E1146130905002326C107231B61000B
:10BCC00023221103232601032324F100232CF10056
:10BCD0002328E100232EE10023200102EFE0DFD73B
:10BCE00093040500635C05028357410193F7070441
:10BCF000638807008357C40093E707042316F40002
:10BD00008320C14703248147032901471385040089
:10BD10008324414713010148678000009305810097
:10BD200013050900EF000042E30005FC9304F0FF57
:10BD30006FF09FFBB767018003A3879C6700030038
:10BD4000638405029307F00F63E8C7002380C500F2
:10BD500013051000678000009307A0082320F5005A
:10BD60001305F0FF678000001305000067800000E6
:10BD7000B767018083A747A7130101FF2324810030
:10BD8000232291002326110093040500138405004B
:10BD90006386070003A787036300070E0317C40029
:10BDA000931707019376870093D7070163800604F2
:10BDB000832604016380060613F617006304060851
:10BDC0000326440123240400130500003306C04069
:10BDD000232CC400638606088320C100032481004D
:10BDE00083244100130101016780000093F60701DD
:10BDF0006384060C93F747006396070883260401C3
:10BE000013678700931707012316E40093D70701F0
:10BE1000E39406FA13F6072893050020E30EB6F81C
:10BE20009305040013850400EF00907B0317C40002
:10BE3000832604019317070193D7070113F6170010
:10BE4000E31006F813F627009305000063140600BC
:10BE5000832544012324B40013050000E39E06F665
:10BE600093F70708E38A07F6136707042316E4002D
:10BE70001305F0FF6FF05FF613850700EF004067D2
:10BE80006FF0DFF183250403638E0500930704043C
:10BE90006388F50013850400EF808F890317C400C1
:10BEA00023280402832604011377B7FD232204000C
:10BEB0002320D4006FF0DFF49307900023A0F40058
:10BEC000136707042316E4001305F0FF6FF0DFF09B
:10BED000130101FF1305600023261100EF10402A13
:10BEE00013051000EF40CFD88397C500130101FE62
:10BEF000232C810023263101232E1100232A9100B7
:10BF00002328210193F68700138405009309050077
:10BF1000639A0610371700001307078083A64500B1
:10BF2000B3E7E7002396F5006354D0180327840293
:10BF3000630A070C83A409009396070123A0090054
:10BF4000139637018325C40193D60601634806166C
:10BF5000930610001306000013850900E700070090
:10BF60009307F0FF630CF5188356C400032784027F
:10BF70008325C40193F64600638E060083264400A1
:10BF8000832704033305D540638607008327C40352
:10BF90003305F540130605009306000013850900DC
:10BFA000E70007009307F0FF631EF51003A70900E1
:10BFB0008317C400630807169306D0016306D700F1
:10BFC000930660016314D70C8326040137F7FFFF43
:10BFD0001307F77FB3F7E7002316F40023220400CA
:10BFE0002320D4008325040323A09900638C05003B
:10BFF000930704046386F50013850900EF705FF36F
:10C0000023280402130500008320C10103248101B9
:10C0100083244101032901018329C1001301010285
:10C020006780000003A90501E30E09FC83A4050055
:10C0300013970701135707011377370023A0250132
:10C04000B3842441930700006314070083A74501CC
:10C050002324F400634890006FF0DFFA3309A9004D
:10C06000E35290FA832744028325C4019386040097
:10C070001306090013850900E7800700B384A44074
:10C08000E34EA0FC8357C4001305F0FF93E70704B9
:10C090008320C1012316F40003248101832441017C
:10C0A000032901018329C1001301010267800000F7
:10C0B00003A7C503E34CE0E66FF0DFF403250405B6
:10C0C0006FF05FEB8357C40037F7FFFF1307F77F6D
:10C0D000B3F7E700832604019397070193D707413D
:10C0E0002316F400232204002320D40013973701E1
:10C0F000E35A07EE2328A4046FF0DFEE83A70900BC
:10C10000E38407E61307D0016388E70213076001A1
:10C110006384E7028357C40093E707042316F400FF
:10C120006FF09FEE37F7FFFF1307F77F83260401B9
:10C13000B3F7E7006FF0DFFA23A0990013050000C2
:10C140006FF09FEC130101FE232C8100232E1100C0
:10C150001304050063060500832785036380070237
:10C160008397C500639607028320C10103248101E0
:10C170001305000013010102678000002326B100AF
:10C18000EF0000378325C1008397C500E38E07FCCD
:10C1900013050400032481018320C101130101025E
:10C1A0006FF09FD49305050063080500B767018011
:10C1B00003A547A76FF01FF9B767018003A507A77D
:10C1C000B7C50080938545146F0050291305000002
:10C1D00067800000B7D50080938505716F00102837
:10C1E000130101FEB7C70080232E1100232C81000C
:10C1F000232A9100232821012326310123244101F0
:10C200002322510123206101032445009387471D08
:10C21000232EF5021307C52E930730002324E52EA5
:10C220002322F52E2320052E930740001309050035
:10C230002326F40013068000930500002322040641
:10C2400023200400232204002324040023280400C4
:10C25000232A0400232C04001305C405EF40DFB09B
:10C2600037DB008083248900B7DA008037DA00806A
:10C27000B7D90080130B0B24938A4A2A130ACA32B7
:10C2800093894939B707010023206403232254030B
:10C290002324440323263403232E8400938797000A
:10C2A00023A6F400130680009305000023A20406D1
:10C2B00023A0040023A2040023A4040023A8040054
:10C2C00023AA040023AC04001385C405EF40DFA9B2
:10C2D0000324C900B707020023A0640323A2540368
:10C2E00023A4440323A6340323AE94009387270199
:10C2F0002326F40023220406232004002322040022
:10C300002324040023280400232A0400232C0400EF
:10C310001305C4051306800093050000EF40DFA459
:10C320008320C101232064032322540323244403D4
:10C3300023263403232E8400032481019307100055
:10C34000232CF90283244101032901018329C1001F
:10C35000032A8100832A4100032B010013010102FB
:10C36000678000001305000067800000130101FFD3
:10C3700023229100130680069384F5FFB384C40240
:10C380002320210113890500232481002326110085
:10C3900093854407EFA01FA713040500630005025F
:10C3A0001305C50023200400232224012324A40014
:10C3B0001386840693050000EF401F9B8320C10075
:10C3C0001305040003248100832441000329010094
:10C3D0001301010167800000130101FEB7670180AE
:10C3E0002328210103A907A723263101232E1100A9
:10C3F00083278903232C8100232A910093090500B8
:10C400006386070A1309092E9304F0FF8327490066
:10C41000032489009387F7FF63D807006F000008A3
:10C4200013048406638C97060317C4009387F7FFF1
:10C43000E31807FEB707FFFF9387170023220406C0
:10C440002320040023220400232404002326F400D4
:10C4500023280400232A0400232C04001306800050
:10C46000930500001305C405EF401F902328040224
:10C47000232A040223220404232404048320C10168
:10C4800013050400032481018324410103290101D0
:10C490008329C10013010102678000000324090001
:10C4A000630C0400130904006FF05FF61305090024
:10C4B000EFF01FD36FF01FF59305400013850900BF
:10C4C000EFF0DFEA2320A90013040500E31C05FCBC
:10C4D0009307C00023A0F9006FF05FFAB7670180EF
:10C4E00003A507A7B7D50080938505716F00007776
:10C4F0008327850363840700678000006FF05FCEA9
:10C50000678000006780000067800000678000008F
:10C51000B767018003A547A7B7C500809385C51CF1
:10C520006F008069B767018003A547A7B7C5008082
:10C53000938545366F004068130101FD2324810275
:10C54000232E310123286101232611022322910287
:10C5500023202103232C4101232A5101130B050021
:10C560009389050013040600EFD01FA29307100063
:10C570006310F5029387F9FF1307E00F636AF70072
:10C5800013F7F90F2306E100130910006F00C00232
:10C590009306C405138609009305C10013050B001B
:10C5A000EF0090799307F0FF130905006304F50A83
:10C5B000630E05080347C10093040000130AF0FF4F
:10C5C000930AA0006F00800283270400938617005F
:10C5D0002320D4002380E700938414009307C10034
:10C5E000B387970063F4240703C7070083278400F9
:10C5F0009387F7FF2324F400E3D807FC8326840104
:10C60000930507001306040013050B0063C4D7004D
:10C61000E31C57FBEF009058E31045FD1309F0FFB2
:10C620008320C10203248102832441028329C101A2
:10C63000032A8101832A4101032B0101130509000B
:10C640000329010213010103678000001389090017
:10C650006FF01FFD8357C40093E707042316F4000F
:10C660006FF01FFC8317C600139727016340070272
:10C6700003274606B7260000B3E7D700B726000019
:10C680003367D7002316F6002322E6066FF0DFEAB1
:10C69000130101FEB7670180232C810003A447A783
:10C6A000232E110013860500930505006306040080
:10C6B00083278403638007048317C6001397270129
:10C6C0006340070203274606B7260000B3E7D700FA
:10C6D000B72600003367D7002316F6002322E606AC
:10C6E00013050400032481018320C1011301010209
:10C6F0006FF09FE42324A100130504002326C1004A
:10C70000EFF01FDF0326C100832581006FF0DFFA01
:10C7100083278600638E073283D7C500130101FD8E
:10C7200023248102232C4101232A510123261102B3
:10C730002322910223202103232E3101232861018A
:10C740002326710123248101232291012320A101A9
:10C7500013F78700130A0600930A050013840500E7
:10C760006306070803A705016302070813F72700FC
:10C7700083240A00630C0708832744028325C4012D
:10C78000370B00809309000013090000134B0BC006
:10C790001386090013850A00630209049306090041
:10C7A00063742B0193060B00E78007006358A028F1
:10C7B00083278A00B389A9003309A9403385A7409C
:10C7C0002324AA00630A0520832744028325C40189
:10C7D0001386090013850A00E31209FC83A90400EB
:10C7E00003A94400938484006FF09FFA930504002A
:10C7F00013850A00EFF0CFD7631C053A8357C400B6
:10C8000083240A0013F72700E31807F613F717002D
:10C8100063140724832C840003250400370B008055
:10C82000934BEBFF130C000013090000134BFBFFAD
:10C83000630E090E13F70720630C0724138D0C00F9
:10C840006362992F13F70748630A07088329440195
:10C85000832504011307190093961900B386360146
:10C8600093D9F601330DB540B389D90093D9194056
:10C870003307A7011386090063F6E900930907004F
:10C880001306070093F707406384072E93050600FD
:10C8900013850A00EFA00FD7930C05006302053043
:10C8A0008325040113060D00EFD08FF78357C400D2
:10C8B00093F7F7B793E707082316F4003385AC0125
:10C8C000B387A941232894012320A400232A3401FB
:10C8D000930C09002324F400130D090013060D0026
:10C8E00093050C00EFD09F85032784008327040065
:10C8F00093090900B30C9741B387A701232494013E
:10C900002320F4001309000003268A00330C3C01A5
:10C91000B309364123243A016380090C832C840037
:10C92000032504008357C400E31609F003AC040098
:10C9300003A94400938484006FF09FEF83A944000F
:10C9400003AC040093848400E38A09FE1386090083
:10C950009305A00013050C00EFA05FC66304051249
:10C9600013051500330B854193070B00938B0900CA
:10C9700063F43701938B0700032504008327040128
:10C980008326440163F8A700032984003389260124
:10C990006342790963C8DB1A832744028325C401F3
:10C9A00013060C0013850A00E78007001309050031
:10C9B0006356A008330B2B4113051000630A0B16B6
:10C9C00003268A00330C2C01B389294133092641FF
:10C9D00023242A01631A0908130500008320C102D9
:10C9E0000324810283244102032901028329C10116
:10C9F000032A8101832A4101032B0101832BC100FA
:10CA0000032C8100832C4100032D0100130101033D
:10CA10006780000093050C0013060900EFD00FF2A9
:10CA2000832704009305040013850A00B3872701B8
:10CA30002320F400EFF00FF1E30E05F68317C40096
:10CA400093E707042316F4001305F0FF6FF01FF9B6
:10CA50001305000067800000130B000013050000A1
:10CA6000130C000093090000E38A09ECE31E05EEB5
:10CA7000138609009305A00013050C00EFA01FB456
:10CA8000E31005EE93871900138B07006FF01FEE7C
:10CA90008327040163E2A70483274401636EF9023C
:10CAA0009306090063F42B0193060B00B3C6F6024C
:10CAB000032744028325C40113060C0013850A00D2
:10CAC000B386F602E700070093090500E358A0F6D5
:10CAD000330939416FF05FE393890C006374990166
:10CAE000930909001386090093050C00EFD00FE5A8
:10CAF0008327840003270400B387374133073701B6
:10CB00002324F4002320E400E39407FC93050400AD
:10CB100013850A00EFF00FE3E31205F23309394100
:10CB20006FF09FDE930C0900130D09006FF01FDBFF
:10CB30009305040013850A00EFF0CFE0E30205E857
:10CB40006FF0DFEF13860B0093050C00EFD00FDFC3
:10CB5000832784000326040013890B00B3877741E1
:10CB6000330676012324F4002320C4006FF09FE4F1
:10CB700013850A00EFD08FEE930C0500E31005D467
:10CB80008325040113850A00EF708FBA8317C40050
:10CB90001307C00023A0EA0093F7F7F76FF05FEAEE
:10CBA0001307C0008317C40023A0EA006FF05FE9F9
:10CBB0001305F0FF6FF09FE2130101FE232821010E
:10CBC0002326310123244101232251012320610125
:10CBD000232E1100232C8100232A9100138B0500A2
:10CBE000930A052E130A0000930910001309F0FFA1
:10CBF00083A44A0003A48A009384F4FF63C604025A
:10CC00008357C4009384F4FF63FCF9008317E400A6
:10CC10001305040063862701E7000B00336AAA00AE
:10CC200013048406E39E24FD83AA0A00E3920AFC0F
:10CC30008320C101032481018324410103290101CF
:10CC40008329C100832A4100032B010013050A0038
:10CC5000032A81001301010267800000130101FD16
:10CC600023202103232E3101232C4101232A5101AA
:10CC70002328610123267101232611022324810226
:10CC800023229102930A0500938B0500130B052EB6
:10CC9000130A0000930910001309F0FF83244B00CE
:10CCA00003248B009384F4FF63C804028357C400F9
:10CCB0009384F4FF63FEF9008317E40093050400F6
:10CCC00013850A0063862701E7800B00336AAA00F8
:10CCD00013048406E39C24FD032B0B00E3100BFCE0
:10CCE0008320C1020324810283244102032901021B
:10CCF0008329C101832A4101032B0101832BC10038
:10CD000013050A00032A8101130101036780000053
:10CD1000130101F923248106138405008395E5009E
:10CD200023229106232021072326110693040600BF
:10CD30001389060063CA050413068100EF00502F13
:10CD4000634405040327C100B7F700008320C10630
:10CD5000B3F7E70037E7FFFFB387E7000324810657
:10CD600093B717002320F9009307004023A0F40095
:10CD700037150000832441060329010613050580A9
:10CD800013010107678000008357C40023200900B6
:10CD900093F70708638407028320C10603248106F2
:10CDA0009307000423A0F40003290106832441060D
:10CDB0001305000013010107678000008320C106EE
:10CDC000032481069307004023A0F40003290106F1
:10CDD000832441061305000013010107678000004A
:10CDE00083D7C500130101FE232C8100232E1100DF
:10CDF000232A91002328210193F72700138405009B
:10CE0000638807029387350423A0F50023A8F50063
:10CE10009307100023AAF5008320C1010324810198
:10CE200083244101032901011301010267800000ED
:10CE30009306C1001306810093040500EFF05FED37
:10CE4000832581001309050013850400EF909FFBE3
:10CE50008317C4006308050437C700801307471D04
:10CE600023AEE402032781008326C10093E707086D
:10CE70002316F4002320A4002328A400232AE4007E
:10CE800063980604B3E727018320C1012316F40049
:10CE900003248101832441010329010113010102BB
:10CEA0006780000013F70720E31807F693F7C7FF22
:10CEB00093E72700130734042316F40093071000A8
:10CEC0002320E4002328E400232AF4006FF0DFF499
:10CED0008315E40013850400EF00101C63160500A1
:10CEE0008317C4006FF01FFA0357C4001377C7FFFE
:10CEF000136717009317070193D707416FF09FF847
:10CF0000130101FF9305000823248100232611004B
:10CF100013040500EF901FEF232EA42C63040502D9
:10CF2000930705082320050013054500E31CF5FEC3
:10CF3000130500008320C1000324810013010101B7
:10CF4000678000001305F0FF6FF0DFFE8327C52D1B
:10CF50006386070013050000678000006FF05FFA2A
:10CF6000130101FE232A9100232E1100232C81009E
:10CF70009307F0019304050063EAB70213840500E8
:10CF80008325C52D63840504131424003384850090
:10CF9000032504002320C4008320C1010324810150
:10CFA0008324410113010102678000008320C10135
:10CFB00003248101930760012320F50083244101AC
:10CFC0001305F0FF13010102678000002326C10052
:10CFD000EFF01FF3930705001305F0FFE39E07FA38
:10CFE00083A5C42D0326C1006FF01FFA130101FFB2
:10CFF0002322910023261100232481009307F001AE
:10D000009304050063EAB70A8327C52D138405003E
:10D010006384070413972500B387E70003A707007D
:10D02000630C070293061000630CD7069306F0FF0B
:10D030006308D7041385050023A00700E700070055
:10D04000130500008320C1000324810083244100D4
:10D05000130101016780000013850400EF00001E2A
:10D0600013060400032481008320C10093050500FA
:10D070001385040083244100130101016F00801512
:10D080008320C10003248100930760012320F50061
:10D090008324410013051000130101016780000083
:10D0A0008320C10003248100832441001305000074
:10D0B0001301010167800000930760012320F50040
:10D0C0001305F0FF6FF01FF89307F00163E6B70A4E
:10D0D0008327C52D130101FE232C9100232E11005F
:10D0E00093040500638C070413972500B387E700BA
:10D0F00003A70700630A07029306F0FF6306D7063B
:10D10000930610006308D7041385050023A00700C9
:10D11000E7000700130500008320C101832481017B
:10D1200013010102678000008320C1018324810173
:10D130001305100013010102678000002326B100CF
:10D14000EFF01FDC6316050283A7C42D8325C10001
:10D150006FF09FF98320C101832481011305300002
:10D160001301010267800000130520006FF0DFFA51
:10D170001305F0FF6FF05FFA1305F0FF6780000002
:10D18000B76701809305050003A547A76FF01FE669
:10D190003767018093070500032547A7138605001D
:10D1A000938507006FF0DFDBB767018003A547A712
:10D1B0008327C52D638607001305000067800000E4
:10D1C0006FF01FD4B76701809305050003A547A73B
:10D1D0006FF09FEF130101FF1387050023248100E7
:10D1E0002322910013040500B76401809305060013
:10D1F000130507002326110023AC04B8EF00500EDE
:10D200009307F0FF630CF5008320C1000324810025
:10D2100083244100130101016780000083A784B9C2
:10D22000E38407FE8320C1002320F400032481004F
:10D230008324410013010101678000006F00D005C5
:10D24000130101FF23248100138405008395E50069
:10D2500023261100EF0000716340050283270405B7
:10D260008320C100B387A7002328F404032481008E
:10D2700013010101678000008357C40037F7FFFFE7
:10D280001307F7FFB3F7E7008320C1002316F4006C
:10D2900003248100130101016780000013050000D1
:10D2A000678000008397C500130101FE232C8100D5
:10D2B000232A91002328210123263101232E110046
:10D2C00013F7071013840500930405008395E50008
:10D2D0001309060093890600631E070237F7FFFF54
:10D2E0001307F7FFB3F7E7002316F40003248101C7
:10D2F0008320C10193860900130609008329C10018
:10D300000329010113850400832441011301010253
:10D310006F0040339306200013060000EF00C05D4D
:10D320008317C4008315E4006FF05FFB130101FF56
:10D3300023248100138405008395E5002326110032
:10D34000EF00805B9307F0FF6304F5028357C4008E
:10D35000371700008320C100B3E7E7002328A404A7
:10D360002316F400032481001301010167800000EB
:10D370008357C40037F7FFFF1307F7FFB3F7E70042
:10D380008320C1002316F40003248100130101014E
:10D39000678000008395E5006F008031130101FE76
:10D3A000232C8100232A910023282101232E110000
:10D3B0002326310113090500938405001304060098
:10D3C0006306050083278503638807140317C400D9
:10D3D00083268401937787002324D40093160701C2
:10D3E00093D606016382070883270401638E07062C
:10D3F0001396260193F9F40F93F4F40F635E060875
:10D400000327040083264401B307F74063DED70AED
:10D4100083268400130617002320C4009386F6FF9A
:10D420002324D400230037010327440193871700E6
:10D430006308F70C8357C40093F71700638607004F
:10D440009307A000638EF40A8320C10103248101A5
:10D45000032901018329C1001385040083244101AC
:10D460001301010267800000930504001305090001
:10D47000EFE01F90631E05080317C40093F9F40F33
:10D48000832704019316070193D6060113962601FC
:10D4900093F4F40FE34606F683264406372600008D
:10D4A0003367C70037E6FFFF1306F6FFB3F6C60083
:10D4B0002316E400032704002322D4068326440114
:10D4C000B307F740E3C6D7F493050400130509003A
:10D4D000EFE05FC7631E0502032704008326840074
:10D4E00093071000130617009386F6FF2320C4004D
:10D4F0002324D4002300370103274401E31CF7F25F
:10D500009305040013050900EFE0DFC3E30E05F205
:10D510009304F0FF6FF05FF3EFE09FFD6FF01FEB00
:10D520003767018093070500032547A71386050089
:10D53000938507006FF09FE6130101FE232C810005
:10D54000232A9100B7670180232E110083A7879CAF
:10D55000130405009384060063820502E780070038
:10D560009307F0FF6306F5028320C10103248101C4
:10D5700083244101130101026780000013060000AB
:10D5800093054100E78007009307F0FFE31EF5FCD9
:10D5900023A004009307A0088320C1012320F400E6
:10D5A00003248101832441011301010267800000EB
:10D5B000130101FEB7670180232C8100232A91000B
:10D5C000232E110083A447A7B767018083A7879CF8
:10D5D00013040600630A050213860500930604007F
:10D5E0009305050013850400E78007009307F0FF0B
:10D5F000630AF5028320C1010324810183244101D0
:10D6000013010102678000009306060093054100A4
:10D610001306000013850400E78007009307F0FF5E
:10D62000E31AF5FC232004008320C10103248101B7
:10D630009307A00823A0F4008324410113010102F1
:10D6400067800000130101FF138705002324810078
:10D65000232291009305060013040500B76401809E
:10D6600013860600130507002326110023AC04B817
:10D67000EF00405D9307F0FF630CF5008320C100CD
:10D68000032481008324410013010101678000000D
:10D6900083A784B9E38407FE8320C1002320F4001C
:10D6A00003248100832441001301010167800000ED
:10D6B000130101FF2324810023229100130405009C
:10D6C000B7640180138505002326110023AC04B83C
:10D6D000EF0000309307F0FF630CF5008320C100DA
:10D6E00003248100832441001301010167800000AD
:10D6F00083A784B9E38407FE8320C1002320F400BC
:10D70000032481008324410013010101678000008C
:10D71000130101FF232611002324810023229100FD
:10D720002320210163800502138405009304050072
:10D730006306050083278503638C070A8317C400EB
:10D74000639207028320C1000324810013090000B3
:10D75000832441001305090003290100130101017D
:10D76000678000009305040013850400EFE0CFF705
:10D770008327C40213090500638A07008325C401B7
:10D7800013850400E7800700634C05068357C40037
:10D7900093F70708639E070683250403638C05003F
:10D7A000930704046386F50013850400EF604FF8C7
:10D7B000232804028325440463880500138504009C
:10D7C000EF600FF723220404EFE09FD32316040039
:10D7D000EFE05FD38320C100032481008324410054
:10D7E00013050900032901001301010167800000EE
:10D7F000EFE01FD08317C400E38607F46FF09FF6B5
:10D800008357C4001309F0FF93F70708E38607F86E
:10D810008325040113850400EF608FF16FF0DFF7BB
:10D82000B76701809305050003A547A76FF05FEE7A
:10D83000130101FF13870500232481002322910097
:10D8400013040500B7640180930506001305070063
:10D850002326110023AC04B8EF00001D9307F0FF4E
:10D86000630CF5008320C100032481008324410060
:10D87000130101016780000083A784B9E38407FED8
:10D880008320C1002320F40003248100832441006D
:10D890001301010167800000130101FF23248100AF
:10D8A0002322910013040500B7640180138505004D
:10D8B0002326110023AC04B8EF00801E9307F0FF6D
:10D8C000630CF5008320C100032481008324410000
:10D8D000130101016780000083A784B9E38407FE78
:10D8E0008320C1002320F40003248100832441000D
:10D8F0001301010167800000130101FF1387050078
:10D9000023248100232291009305060013040500BF
:10D91000B764018013860600130507002326110053
:10D9200023AC04B8EF00001E9307F0FF630CF50072
:10D930008320C100032481008324410013010101DD
:10D940006780000083A784B9E38407FE8320C100B9
:10D950002320F400032481008324410013010101EA
:10D9600067800000130101FF138705002324810055
:10D97000232291009305060013040500B76401807B
:10D9800013860600130507002326110023AC04B8F4
:10D99000EF00401C9307F0FF630CF5008320C100EB
:10D9A00003248100832441001301010167800000EA
:10D9B00083A784B9E38407FE8320C1002320F400F9
:10D9C00003248100832441001301010167800000CA
:10D9D000130101FF23261100232481009305000079
:10D9E00013060000930600001307000093070000D1
:10D9F000930890037300000013040500634C0500B6
:10DA00008320C100130504000324810013010101D8
:10DA10006780000033048040EF305F902320850052
:10DA20001304F0FF6FF0DFFD130101F723229108CB
:10DA300023261108938405002324810893050100FF
:10DA40001306000093060000130700009307000070
:10DA500093080005730000001304050063440502E9
:10DA60001385040093050100EF00C0228320C10844
:10DA700013050400032481088324410813010109CC
:10DA80006780000033048040EF305F8923208500E9
:10DA90001304F0FF6FF0DFFC130510006780000037
:10DAA000130101F99305810023261106EFF0DFF73A
:10DAB0009307F0FF630EF5000325C1008320C10624
:10DAC0001355D50013751500130101076780000079
:10DAD0008320C106130500001301010767800000C1
:10DAE000130101FF23261100EF305F838320C10063
:10DAF000930760012320F5001305F0FF13010101D6
:10DB000067800000130101FF2326110023248100F8
:10DB10009306000013070000930700009308E0033A
:10DB20007300000013040500634C05008320C1004E
:10DB30001305040003248100130101016780000024
:10DB400033048040EF308FFD232085001304F0FF65
:10DB50006FF0DFFD130101FF232611002324810054
:10DB60009306000013070000930700009308F003DA
:10DB70007300000013040500634C05008320C100FE
:10DB800013050400032481001301010167800000D4
:10DB900033048040EF308FF8232085001304F0FF1A
:10DBA0006FF0DFFD376301808327C3A8130101FFF6
:10DBB00023261100130805006398070213050000CF
:10DBC00093050000130600009306000013070000F1
:10DBD0009308600D730000001307F0FF9307050022
:10DBE0006304E5042326A3A83305F8009305000089
:10DBF00013060000930600001307000093070000BF
:10DC00009308600D730000008327C3A83308F80051
:10DC1000631C05018320C1002326A3A813850700E8
:10DC20001301010167800000EF304FEF8320C10036
:10DC30009307C0002320F5001305F0FF1301010135
:10DC400067800000130101FF2326110023248100B7
:10DC500093060000130700009307000093080004D8
:10DC60007300000013040500634C05008320C1000D
:10DC700013050400032481001301010167800000E3
:10DC800033048040EF308FE9232085001304F0FF38
:10DC90006FF0DFFD130101FF83A3450183A285011E
:10DCA00083AFC50103AF050283AE050303AE0504D0
:10DCB00003A3850303A8850483A8C50403A68505DB
:10DCC000232681002324910003A4050183A4850059
:10DCD0002322210103A9050083A6C50503A7850604
:10DCE00083A7C50623102501231195002322850053
:10DCF00023147500231555002316F5012317E5019C
:10DD00002328D5012326C50523246504232C0501DA
:10DD1000232E15012324C5022326D5020324C10086
:10DD2000232CE502232EF5028324810003294100E0
:10DD30001301010167800000930805009387050027
:10DD40001308060013850600138308006394062851
:10DD5000B74601809386C6ED63F6C50E370701000E
:10DD60006378E60C1307F00F3337C700131737003B
:10DD70003355E600B386A60083C6060013050002ED
:10DD80003387E600B306E540630CE500B397D700A0
:10DD900033D7E8003318D600B365F7003393D800C3
:10DDA00093580801B3D7150313160801135606013B
:10DDB00013570301B3F6150313850700B305F602E5
:10DDC0009396060133E7E600637EB7003307070149
:10DDD0001385F7FF636807016376B7001385E7FFD4
:10DDE000330707013307B740B37717031313030152
:10DDF00013530301335717039397070133E3670066
:10DE0000B306E60213060700637CD3003303680001
:10DE10001306F7FF636603016374D3001306E7FF7D
:10DE2000131505013365C500930500006F00400E12
:10DE30003705000113070001E36CA6F21307800108
:10DE40006FF01FF363160600130710003358C70264
:10DE5000370701006370E80C1307F00F63740701C4
:10DE6000130580003357A800B386E60003C70600F9
:10DE7000130600023307A700B306E6406316E60A5E
:10DE8000B387074193051000935808011316080142
:10DE90001356060113570301B3F61703B3D717033D
:10DEA0009396060133E7E600330EF602138507006A
:10DEB000637EC701330707011385F7FF6368070116
:10DEC0006376C7011385E7FF330707013307C741AF
:10DED000B3771703131303011353030133571703C6
:10DEE0009397070133E36700B306E60213060700C2
:10DEF000637CD300330368001306F7FF63660301F6
:10DF00006374D3001306E7FF131505013365C500DD
:10DF1000678000003707000113050001E364E8F49F
:10DF2000130580016FF01FF43318D800B3D5E70054
:10DF30003393D800B397D70033D7E800935808013C
:10DF40003366F70033F715039317080193D70701DA
:10DF500013550601B3D51503131707013367A7003F
:10DF6000B386B70213850500637ED7003307070128
:10DF70001385F5FF636807016376D7001385E5FF16
:10DF800033070701B306D74033F71603131606010C
:10DF900013560601B3D6160313170701B388D70229
:10DFA000B367C7001387060063FE1701B387070135
:10DFB0001387F6FF63E8070163F617011387E6FF8F
:10DFC000B387070193150501B3871741B3E5E50052
:10DFD0006FF09FEB63E6D5183707010063F4E604A2
:10DFE0001307F00FB335D7009395350037470180FD
:10DFF00033D5B6001307C7ED3307A7000347070063
:10E00000130500023307B700B305E5406316E502C8
:10E0100013051000E3EEF6EE33B5C8001345150006
:10E020006FF01FEF3707000193050001E3E0E6FC06
:10E03000930580016FF09FFB3353E600B396B60063
:10E040003363D30013550301B31EB60033D6E70084
:10E05000B376A602B397B70033D7E8003368F7006A
:10E060009317030193D70701135708013356A602EC
:10E070009396060133E7E600338FC702130E0600BE
:10E08000637EE70133076700130EF6FF63686700DE
:10E090006376E701130EE6FF330767003307E741B6
:10E0A000B376A7023357A702939606013386E70299
:10E0B0009317080193D70701B3E7F600930607000B
:10E0C00063FEC700B38767009306F7FF63E8670046
:10E0D00063F6C7009306E7FFB387670013150E01C9
:10E0E000370E01003365D5009306FEFF3378D50067
:10E0F000B387C740B3F6DE001356050193DE0E0169
:10E100003303D802B306D602135703013308D803EA
:10E110003308D800330707013306D6036374D700EA
:10E120003306C601935607013386C60063E6C7026D
:10E13000E39CC7CEB70701009387F7FF3377F7005B
:10E14000131707013373F300B398B8003307670060
:10E1500093050000E3FEE8DA1305F5FF6FF0DFCC6E
:10E1600093050000130500006FF09FDA9308060086
:10E17000138706009307050013880500639C062299
:10E18000B74601809386C6ED63FCC50C37030100DA
:10E19000637E660A1303F00F6374C30013078000E5
:10E1A0003353E600B386660003CE0600330EEE005E
:10E1B000130700023303C741630CC701B395650021
:10E1C000335EC501B31866003368BE00B31765003F
:10E1D00013D608013377C8021395080113550501BA
:10E1E00093D607013358C80213170701B366D70047
:10E1F0003308050363FA0601B386160163E61601C8
:10E2000063F40601B3861601B386064133F7C602EE
:10E210009397070193D70701B3D6C602B306D50279
:10E2200013150701B367F50063FAD700B387170129
:10E2300063E6170163F4D700B3871701B387D740AC
:10E2400033D56700930500006780000037030001A5
:10E2500013070001E36666F4130780016FF05FF4B3
:10E260006316060013061000B358160337060100A4
:10E2700063F2C80A1306F00F6374160113078000D7
:10E2800033D6E800B386C60003CE0600330EEE0098
:10E29000130700023303C7416318C709B38515414B
:10E2A00013D70801139508011355050113D607016B
:10E2B000B3F6E502B3D5E50293960601B3E6C600D0
:10E2C000B305B50263FAB600B386160163E616011C
:10E2D00063F4B600B3861601B385B640B3F6E50223
:10E2E0009397070193D70701B3D5E502B305B502AC
:10E2F00013950601B367F50063FAB700B3871701FA
:10E3000063E6170163F4B700B3871701B387B7401B
:10E310006FF01FF33706000113070001E3E2C8F6B0
:10E32000130780016FF0DFF5B398680033D7C5019C
:10E33000B3176500335EC50113D50801B376A70294
:10E34000B3956500336EBE009395080193D5050122
:10E3500013560E013357A70293960601B3E6C60083
:10E360003387E50263FAE600B386160163E6160119
:10E3700063F4E600B38616013386E640B376A60260
:10E38000131E0E01135E0E013356A602939606016C
:10E390003386C502B3E5C60163FAC500B38515012E
:10E3A00063E6150163F4C500B3851501B385C54067
:10E3B0006FF01FEFE3EAD5E83707010063FCE604DE
:10E3C000130EF00F3337DE0013173700B748018004
:10E3D00033D3E6009388C8EDB388680003CE080005
:10E3E000330EEE00130700023303C741631EC70359
:10E3F00063E4B600636AC500B307C540B385D54082
:10E400003335F5003388A5401385070093050800D0
:10E410006FF09FE3B708000113070001E3E816FB64
:10E42000130780016FF09FFA3357C601B396660059
:10E43000336FD700B3D7C50113570F01B3F8E70205
:10E44000B39565003358C5013368B80093150F01C3
:10E4500093D5050193560801331666003315650000
:10E46000B3D7E70293980801B3E6D800B38EF5025C
:10E470009388070063FED601B386E6019388F7FF11
:10E4800063E8E60163F6D6019388E7FFB386E60109
:10E49000B386D641B3FEE6021318080113580801EB
:10E4A000B3D6E602939E0E01B3EE0E01B385D502FC
:10E4B0009387060063FEBE00B38EEE019387F6FFDE
:10E4C00063E8EE0163F6BE009387E6FFB38EEE01CC
:10E4D000B385BE4093980801B70E0100B3E8F80079
:10E4E0009387FEFF33F8F8009356060193D808018E
:10E4F000B377F6003307F802B387F8023308D8027F
:10E50000B388D8023308F80093560701B386060192
:10E5100063F4F600B388D801B70701009387F7FFCB
:10E5200013D80601B3F6F600939606013377F70089
:10E53000B30818013387E60063E61501639E1501F1
:10E54000637CE5003306C7403337C7003307E70174
:10E55000B388E840130706003307E5403335E5008C
:10E56000B3851541B385A540B397C50133576700FF
:10E5700033E5E700B3D565006FF01FCD130101FD52
:10E5800023248102232A51012324810123261102FD
:10E590002322910223202103232E3101232C410128
:10E5A0002328610123267101232291011304050010
:10E5B000130C0600938A06007329200093D74501A7
:10E5C000939BC5001397570193DBCB0013DAF5013A
:10E5D000630C070213FBF77F9307F07F6308FB08C8
:10E5E0001357D501939B3B00B36B7701B7078000AE
:10E5F000B3EBFB0093193500130B1BC0930C000009
:10E60000930400006F008008B3E7AB00638E070E31
:10E6100063800B0413850B00EF401033130755FF85
:10E620009307C00163CCE7029306D001930985FFED
:10E63000B386E640B39B3B01B356D400B3EB7601FF
:10E64000B31934019305D0C0338BA5406FF01FFB85
:10E65000EF40902F130505026FF05FFC930B85FDD3
:10E66000B31B7401930900006FF0DFFD33E4AB00CE
:10E670006306040A9397CB0093090500130BF07F00
:10E68000930C300093040001E3CC07F613D74A0142
:10E690001395CA009316570193070C001354C50035
:10E6A0009375F77F93DAFA01638406081307F07F06
:10E6B0006386E50E9357DC011315340033E5A7009C
:10E6C000370480003364850093173C00138515C020
:10E6D0001307000093962C00B3E6E600B305AB40A9
:10E6E0009386F6FF1305E00033465A016360D510A8
:10E6F0003745018093962600130585E2B386A60070
:10E7000083A6060067800600930B000093090000B3
:10E71000130B0000930C10006FF09FEE930B0000A2
:10E7200093090000130BF07F930C20006FF05FED56
:10E73000B3678401638407086302040413050400BB
:10E74000EF40902093050500938655FF9307C00185
:10E7500063CED7021307D001938785FF3307D740D5
:10E760003315F4003357EC003364A700B317FC00F3
:10E770001307D0C03305B7406FF09FF513050C00A9
:10E78000EF40901C930505026FF01FFC138585FD7B
:10E790003314AC00930700006FF09FFD33668401D3
:10E7A000630806021317C4001305F07F634C0702C9
:10E7B00013073000930400016FF0DFF11304000031
:10E7C0009307000013050000130710006FF09FF07F
:10E7D00013040000930700001305F07F13072000C7
:10E7E0006FF05FEF130730006FF0DFEE63667401C8
:10E7F00063968B2E63E4F92E1395FB0113D7190052
:10E800009396F90193DB1B00B369E50013158400AF
:10E8100013D887013368A8001355050133D3AB0221
:10E82000131E0801135E0E019398870093D7090108
:10E83000B3FBAB02930F030033076E02939B0B01F4
:10E84000B3E7770163FEE700B3870701930FF3FF98
:10E8500063E8070163F6E700930FE3FFB38707015F
:10E86000B387E740B3DEA7029399090193D9090161
:10E87000B3F7A70213830E003307DE039397070154
:10E88000B3E7F90063FEE700B38707011383FEFFD8
:10E8900063E8070163F6E7001383EEFFB387070120
:10E8A0003387E740939F0F01B7070100B3EF6F0075
:10E8B0001383F7FF33FF6F0093D20F0193DE08013C
:10E8C00033F3680033046F02B3896202338FEE03BF
:10E8D000B3033F01135F0401330F7F00B382D20300
:10E8E00063743F01B382F200B703010093570F0135
:10E8F0009383F3FFB3825700B3777F0093970701A9
:10E9000033747400B38787006368570013840F0063
:10E910006314570463F2F604B386160133BF16017D
:10E92000330F0F013307E7011384FFFF6366E8002D
:10E930006314E80263E2160363665700639EE20015
:10E9400063FCF600B386160133BF1601330F0F01C7
:10E950001384EFFF3307E701338FF6403307574047
:10E96000B3B6E6013307D7409307F0FF6304E8121C
:10E97000B352A70293570F013377A7029386020081
:10E98000B30F5E021317070133E7E700637EF70159
:10E99000330707019386F2FF636807016376F70187
:10E9A0009386E2FF330707013307F741B35FA702FE
:10E9B00093170F0193D707013377A702330EFE0396
:10E9C0001317070133E7E70093870F00637EC70142
:10E9D000330707019387FFFF636807016376C70169
:10E9E0009387EFFF3307070193960601B3E6F6001E
:10E9F0009397060193D707013307C74113DE06013A
:10EA0000330FF30233036E02338ECE03B38EFE0256
:10EA100093570F01B38E6E00B387D70163F667007B
:10EA200037050100330EAE0013D307013303C301D2
:10EA3000370E0100130EFEFF33F5C7011315050154
:10EA4000337FCF013305E501636867006314673ED8
:10EA500093870600630005043307E8009387F6FFF9
:10EA600063640703636667006314673C63F0A8028E
:10EA70009387E6FF93961800B3B816013388080110
:10EA80003307070193880600631467006384A800B6
:10EA900093E717001388F53F635A001913F77700BF
:10EAA000630A070A1307200093E414006302E90ACB
:10EAB000130730006308E908631E090813F7F7001D
:10EAC000930640006308D70813874700B337F70061
:10EAD0003304F400930707006F00C0079385F5FF28
:10EAE000930600006FF09FD213060A0013840B00F8
:10EAF0009387090013870C00930630006300D73218
:10EB0000930610006306D73093062000E314D7F86D
:10EB10006F00000113860A006FF01FFE93E484006B
:10EB200013050000930700001307F07F6F00C00576
:10EB30003704080093070000130600001307300095
:10EB40006FF09FFB63180600138787006FF01FF8B4
:10EB5000E31C06FE13177400635A0700370700FF13
:10EB60001307F7FF3374E400138805401307E07FB1
:10EB7000634E070713D737009317D401B3E7E700B5
:10EB8000135534001307080013174701B706F07F29
:10EB90001315C5003377D7001355C5003365A7009B
:10EBA0001316F6013367C5009305070013850700A8
:10EBB0006384040073A014008320C1020324810233
:10EBC00083244102032901028329C101032A81010F
:10EBD000832A4101032B0101832BC100032C8100F7
:10EBE000832C41001301010367800000930720007C
:10EBF000630AF90293073000630AF900631A0900F7
:10EC0000930700001307F07F6F000001E30A06FE80
:10EC10009307F0FF1307E07F93E454001385070088
:10EC20006FF09FF6E31E06FC6FF09FFE13071000C7
:10EC30006316080693F6770013070400638A060438
:10EC40001307200093E414006300E9041307300065
:10EC50006304E90213070400631C090293F6F7003A
:10EC6000130540006386A60213B7C7FF13471700BA
:10EC7000330787006F00C00113070400631A060002
:10EC800013B787FF6FF09FFE13070400E31A06FE19
:10EC90001357870113471700137717001305100048
:10ECA000330505419306800363CCA60E9306F0015D
:10ECB00063C2A6069385E54133D8A700B316B40016
:10ECC000B397B700B3E60601B337F000B3E7F60039
:10ECD0003355A40093F6770063800608930620005E
:10ECE00093E414006308D90693063000630ED90438
:10ECF0006314090693F6F70093054000638EB6048B
:10ED000093864700B3B7F6003305F50093870600F6
:10ED10006F008004930610FEB3860641930800023C
:10ED2000B356D40013080000630615019385E5432C
:10ED30003318B400B367F800B337F000B3E7F60058
:10ED4000130500006FF01FF9631806009386870013
:10ED50006FF05FFBE31C06FE9316850063DE060082
:10ED600093E41400130500009307000063160702E4
:10ED7000130710006FF05FE193D637009317D501AA
:10ED8000B3E7D70013553500E30007E013F714008D
:10ED9000E30C07DE1307000093E424006FF0DFDECE
:10EDA000B3E78700638407029307200093E414000D
:10EDB000630EF902930730006302F9029307100013
:10EDC000631409009307500093D7370093E424009D
:10EDD00013050000130700006FF01FDB930790007E
:10EDE000E30406FE930710006FF01FFE93079000E8
:10EDF000E31C06FC6FF01FFF3705080093070000B7
:10EE00001307F07F13060000930400016FF0DFD7B3
:10EE100013050000930700006FF0DFFB37050800C3
:10EE2000930700001307F07F130600006FF0DFD593
:10EE300093860700938706006FF09FC5130101FDBD
:10EE40002324810223286101232291012326110218
:10EE50002322910223202103232E3101232C41015F
:10EE6000232A510123267101232481011304050063
:10EE7000930C0600138B06007329200093D74501DD
:10EE80009399C5001397570193D9C90093DAF501F7
:10EE9000630C070293FBF77F9307F07F6388FB08FF
:10EEA0009357D50193993900B3E93701B70780002B
:10EEB000B3E9F900131A3500938B1BC0130C000043
:10EEC000930400006F008008B3E7A9006380071077
:10EED0006380090413850900EF400027130755FFDD
:10EEE0009307C00163CCE7029307D001130A85FFA3
:10EEF000B387E740B3994901B357F400B3E9370149
:10EF0000331A4401930BD0C0B38BAB406FF01FFB9F
:10EF1000EF408023130505026FF05FFC930985FD28
:10EF2000B3193401130A00006FF0DFFD33E4A900C8
:10EF30006308040A9397C900130A0500930BF07F36
:10EF4000130C300093040001E3CC07F613574B0178
:10EF50001314CB009316570193870C001354C4006D
:10EF60001375F77F135BFB01638606081307F07FB9
:10EF70006306E50E93D7DC011314340033E48700F5
:10EF8000B70780003364F400130515C093973C0065
:10EF90001307000093162C00B3E6E600B38BAB001A
:10EFA0009386F6FF1306E000B3C56A0113851B00C4
:10EFB000636AD6163746018093962600130646E606
:10EFC000B386C60083A6060067800600930900008A
:10EFD000130A0000930B0000130C10006FF05FEE9B
:10EFE00093090000130A0000930BF07F130C20001C
:10EFF0006FF01FEDB3679401638207086300040498
:10F0000013050400EF404014930655FF9307C00119
:10F0100063CED7021307D001930785FF3307D7408C
:10F020003314F40033D7EC0033648700B397FC004B
:10F030001307D0C03305A7406FF09FF513850C0070
:10F04000EF408010130505026FF01FFC130485FDCF
:10F0500033948C00930700006FF09FFD336694019A
:10F06000630806021317C4001305F07F634C070200
:10F0700013073000930400016FF0DFF11304000068
:10F080009307000013050000130710006FF09FF0B6
:10F0900013040000930700001305F07F13072000FE
:10F0A0006FF05FEF130730006FF0DFEE37040800FA
:10F0B000930700001307F07F9305000093040001FD
:10F0C00013174701B706F07F1314C4003377D70036
:10F0D0001354C4009395F501336487003367B4007B
:10F0E00013850700930507006384040073A01400D0
:10F0F0008320C102032481028324410203290102E7
:10F100008329C101032A8101832A4101032B0101C3
:10F11000832BC100032C8100832C410013010103C8
:10F1200067800000370601001307F6FF93560A01B7
:10F1300013DE0701337AEA00B3F7E70033034E0327
:10F14000B38E4703338FF6023308E30113D30E0166
:10F1500033030301B388C6036374E301B388C800B3
:10F160003378E300B3FEEE001356030113180801D1
:10F17000135304013374E4003308D801330F8A02B7
:10F18000B38E8602330A43033307DA01135A0F01A1
:10F19000330AEA00B38666026376DA0137070100B4
:10F1A000B386E600935E0A01B38EDE00B706010067
:10F1B0009382F6FF337A5A00337F5F0013D7090139
:10F1C000131A0A01B3F95900330AEA01B302EE0235
:10F1D000B30F4601338F3703330E3E0313560F012F
:10F1E000B307F702330EFE003306C6016374F60060
:10F1F000B382D200B70601009387F6FF135E0601C3
:10F200003376F600337FFF0013160601B3878902B9
:10F210003306E601330E5E0033048702330FE30248
:10F2200013D707013303330333038300330367002A
:10F2300063748300330FDF00370701001307F7FF04
:10F24000B376E300B3F7E70093960601B388F801BD
:10F25000B386F60033BA4801B386D6013387460138
:10F26000B388C80033B6C800B30FC701B382CF005C
:10F27000B3B6D6013337470133E7E60033B6C200F1
:10F280001353030133BECF01330767003366CE004B
:10F29000939798003307C7003307E701B3E70701E7
:10F2A00013179700B337F00093D8780113D4720185
:10F2B000B3E71701939292009316770033648700A7
:10F2C000B3E7570063D0060A13D7170093F7170068
:10F2D000B367F7001317F401B3E7E7001354140002
:10F2E0001308F53F6358001113F777006308070808
:10F2F0001307200093E414006300E90813073000AB
:10F300006306E906631C090613F7F700930640003D
:10F310006306D70613874700B337F7003304F400BA
:10F32000930707006F00800593850A001384090086
:10F3300093070A0013070C00930620006302D728E6
:10F34000930630006306D72893061000E31AD7F817
:10F3500013040000930700006F00402493050B0086
:10F360006FF09FFD13850B006FF09FF7639805000A
:10F37000138787006FF05FFAE39C05FE1317740094
:10F38000635A0700370700FF1307F7FF3374E400E1
:10F39000130805401307E07F634E070113D73700BA
:10F3A0009317D401B3E7E7001354340013070800A0
:10F3B0006FF01FD193072000630AF9029307300012
:10F3C000630AF900631A0900930700001307F07F2E
:10F3D0006F000001E38A05FE9307F0FF1307E07F4B
:10F3E00093E45400138407006FF09FCDE39E05FC67
:10F3F0006FF09FFE130710006316080693F6770060
:10F4000013070400638A06041307200093E4140022
:10F410006300E904130730006304E90213070400E2
:10F42000631C090293F6F700130640006386C602C8
:10F4300013B7C7FF13471700330787006F00C001DA
:10F4400013070400639A050013B787FF6FF09FFE50
:10F4500013070400E39A05FE1357870113471700AB
:10F460001377170093061000B38606411306800336
:10F47000634CD60E1306F0016342D6061305E54130
:10F480003316A40033D8D700B397A700336606011C
:10F49000B337F000B367F6003354D40093F6770027
:10F4A000638006089306200093E414006308D906DD
:10F4B00093063000630ED9046314090693F6F7002F
:10F4C00013064000638EC60493864700B3B7F60068
:10F4D0003304F400938706006F008004130610FEC7
:10F4E00033060641930800023356C4001308000097
:10F4F000638616011305E5433318A400B367F800CB
:10F50000B337F000B367F600130400006FF01FF983
:10F5100063980500938687006FF05FFBE39C05FE10
:10F520009316840063DE060093E4140013040000C5
:10F530009307000063160702130710006FF05FB80F
:10F5400093D637009317D401B3E7D7001354340090
:10F55000E30807B613F71400E30407B61307000027
:10F5600093E424006FF0DFB5B3E7870063840702FC
:10F570009307200093E41400630EF9029307300010
:10F580006302F90293071000631409009307500007
:10F5900093D7370093E424001304000013070000FE
:10F5A0006FF01FB293079000E38405FE93071000ED
:10F5B0006FF01FFE93079000E39C05FC6FF01FFFA8
:10F5C00013040000930700001307F07F6FF05FAF94
:10F5D00037040800930700001307F07F930500002D
:10F5E0006FF01FAE83270500832E4500032F850093
:10F5F0008326C50003A7050083A2450083AF8500CD
:10F6000003A3C500130101FF732620003788000003
:10F6100013D606011308F8FF139E06019315030184
:10F6200093D8F6013376060193560301135E0E015B
:10F6300093D50501B3F606011353F301631E0601CA
:10F6400033E8D7013368E8013368C801631208085A
:10F65000639CC60A6F008000639A060133685700F6
:10F660003368F8013368B800631608041305100006
:10F670006396C6026394E70263925E026310FF031F
:10F68000631EBE0063846802639A060033E5D701F7
:10F690003365E5013365C5013335A0001301010170
:10F6A00067800000736018006F00000613050000FB
:10F6B0006FF0DFFE378500001305F5FF6310A60429
:10F6C000B3E7D701B3E7E701B3E7C70163880702F0
:10F6D00013150E0113550541E35605FCB7870000CD
:10F6E0009387F7FF13051000E39AF6FA3367570084
:10F6F0003367F7013367B700E30207FA9395050113
:10F7000093D50541E3D005FA130510006FF01FF9FA
:10F71000832F050003284500032E850083A20500E2
:10F720000325C50083A8450083AE850083A6C500D8
:10F73000130101FFF3272000B787000013560501CE
:10F740009387F7FF931505011393060113D706015D
:10F750003376F60093D505011355F50113530301D4
:10F760003377F70093D6F6016310F602B3E70F0183
:10F77000B3E7C701B3E7B7006384070C73601800F1
:10F780001305E0FF6F000005631AF700B3E71201ED
:10F79000B3E7D701B3E76700E39207FE6314060AF5
:10F7A000B3E70F01B3E7C701B3E7B70093B717009B
:10F7B000631A070033EF1201336FDF01336F6F00FD
:10F7C00063040F06638207081305F0FF63840600D5
:10F7D00013850600130101016780000093070000F4
:10F7E0006FF05FFD6356E600E31605FE6F008006CE
:10F7F0006360B306639E650263ECCE05631EDE03A1
:10F8000063E808056314180163E4F205E36E18FD6C
:10F8100063141801E3EA5FFC130500006FF09FFB1F
:10F82000130510006FF01FFBE39807FE6F00400206
:10F83000E3EC65FA6FF05FFEE368DEFB6FF0DFFD7F
:10F84000E306C7F4E30C07F86394A600E35CC7F88B
:10F85000E30805FC1305F0FF6FF0DFF7832F0500C9
:10F8600003284500032E850083A205000325C5005B
:10F8700083A8450083AE850083A6C500130101FF60
:10F88000F3272000B7870000135605019387F7FF81
:10F89000931505011393060113D706013376F6007D
:10F8A00093D505011355F501135303013377F70081
:10F8B00093D6F6016310F602B3E70F01B3E7C70171
:10F8C000B3E7B7006384070C7360180013052000CA
:10F8D0006F000005631AF700B3E71201B3E7D70121
:10F8E000B3E76700E39207FE6314060AB3E70F016C
:10F8F000B3E7C701B3E7B70093B71700631A070070
:10F9000033EF1201336FDF01336F6F0063040F06B3
:10F91000638207081305F0FF638406001385060061
:10F920001301010167800000930700006FF05FFD85
:10F930006356E600E31605FE6F0080066360B306BB
:10F94000639E650263ECCE05631EDE0363E8080573
:10F950006314180163E4F205E36E18FD63141801E3
:10F96000E3EA5FFC130500006FF09FFB1305100036
:10F970006FF01FFBE39807FE6F004002E3EC65FAAF
:10F980006FF05FFEE368DEFB6FF0DFFDE306C7F4B8
:10F99000E30C07F86394A600E35CC7F8E30805FCF2
:10F9A0001305F0FF6FF0DFF7130101F42328210B9B
:10F9B0002324410B2322510B2320610B232C81098B
:10F9C000232A91091309050083A6050083A7450092
:10F9D00003A5850083AAC500832C0600032B4600DF
:10F9E000032C8600032AC600232E110A232C810A29
:10F9F000232A910A2326310B232E71092328A109DA
:10FA00002326B109F32420003786000013970A014A
:10FA100093D90A01135707011306F6FF232651074E
:10FA20002320D1062322F1062324A1062328D10274
:10FA3000232AF102232CA102232EE102B3F9C900EB
:10FA400093DAFA0163800906638EC916370501004F
:10FA50003367A700232EE102130601039307C103B6
:10FA600003A7070083A6C7FF9387C7FF13173700B5
:10FA700093D6D6013367D70023A2E700E312F6FE40
:10FA80008327010337C5FFFF130515009397370040
:10FA90002328F102B389A900930B0000130400008E
:10FAA0006F00801433E6D7003366A6003366E600A5
:10FAB000630606206300070613050700EF30C068E1
:10FAC000930645FF93D7564093F6F601638E0606DC
:10FAD0001307C0FF3387E702130301031308000273
:10FAE000939527003308D8401307C7003307E30076
:10FAF0006314E30813070108B305B70003270103E4
:10FB00009387F7FFB316D70023A8D5FA9306F0FF23
:10FB10006F00000A63080500EF300063130505025B
:10FB20006FF01FFA638A070013850700EF30C0618A
:10FB3000130505046FF0DFF813850600EF30C06091
:10FB4000130505066FF0DFF71306C0FF3386C70203
:10FB50001307C10393063000B305C70083A5050052
:10FB60009386F6FF1307C7FF2322B700E3D6F6FEFE
:10FB70009387F7FF6FF09FF90326C7FF83280700DD
:10FB8000330EB70033560601B398D800336616011A
:10FB90002320CE001307C7FF6FF09FF513972700B0
:10FBA000130601033307E600232007009387F7FFBE
:10FBB000E396D7FEB7C9FFFF93891901B389A9401E
:10FBC0006FF09FEDB3E7D700B3E7A700B3E7E70017
:10FBD000638C070E1317070113570741930B30006F
:10FBE00013040001E34C07EA13150A0137870000EC
:10FBF00093570A01135505011307F7FF2326410701
:10FC000023209107232261072324810723209105C4
:10FC100023226105232481052326A104B3F7E700ED
:10FC2000135AFA016386070A6384E71C3707010049
:10FC30003365E5002326A104930501041307C104DD
:10FC4000832607000326C7FF1307C7FF93963600D6
:10FC50001356D601B3E6C6002322D700E392E5FE91
:10FC60000327010437C5FFFF1305150013173700DD
:10FC70002320E1043385A7009306000033073501F4
:10FC80002324E100130717002322E10013972B0020
:10FC90003367D7001307F7FF1306E000B3C74A0125
:10FCA0006362E61C3746018013172700130606EA35
:10FCB0003307C70003270700670007009309000008
:10FCC000930B10006FF09FDD930B20006FF01FDD92
:10FCD000B3679B01B3E78701B3E7A700638007140D
:10FCE000630E0504EF304046930645FF93D7564018
:10FCF00093F6F601638006081307C0FF3387E70217
:10FD00001303010413080002939527003308D84019
:10FD10001307C7003307E3006316E308130701085E
:10FD2000B305B700032701049387F7FFB316D70085
:10FD300023A0D5FC9306F0FF6F00400A630A0C0075
:10FD400013050C00EF304040130505026FF0DFF99A
:10FD5000630A0B0013050B00EF30003F1305050489
:10FD60006FF09FF813850C00EF30003E1305050679
:10FD70006FF09FF71306C0FF3386C7021307C10455
:10FD800093063000B305C70083A505009386F6FFF0
:10FD90001307C7FF2322B700E3D6F6FE9387F7FFCA
:10FDA0006FF05FF90326C7FF83280700330EB70003
:10FDB00033560601B398D800336616012320CE00CF
:10FDC0001307C7FF6FF05FF51397270013060104B1
:10FDD0003307E600232007009387F7FFE396D7FE5B
:10FDE000B7C7FFFF938717013385A7406FF0DFE8A0
:10FDF000336B9B01336B8B01336BAB0063060B02E0
:10FE000013150501135505416346050213850700C7
:10FE100093063000130400016FF05FE61305000045
:10FE2000930610006FF09FE51385070093062000EE
:10FE30006FF0DFE413850700930630006FF01FE4D6
:10FE40001304000137870000232EE104232C010452
:10FE5000232A0104232801041307F7FF9307000056
:10FE60006F00D0198325010303250104B7080100A1
:10FE70001386F8FF93D3050113570501B3F5C500A9
:10FE80003375C500B306B702330AB5023383A30244
:10FE90003388660093560A01B3860601B389E302EC
:10FEA00063F46600B3891901032E410493D8060157
:10FEB000B3F6C600337ACA0093960601B3864601AC
:10FEC000935F0E01337ECE003303BE022326D100A2
:10FED0002320D1063386C303B386BF023388C6000E
:10FEE00093560301B3860601B38BF30363F6C60092
:10FEF00037060100B38BCB0013D60601B70E010005
:10FF00002320C1001386FEFF33F8C6003373C300FD
:10FF10001318080133086800B38608012320D102B2
:10FF20008326410393D2060133F6C6003303A602AB
:10FF3000338AA20293580301B306C702B38646016F
:10FF4000B386D800330F570263F44601330FDF0145
:10FF500093D80601370A0100B388E801930EFAFF2F
:10FF6000138B0800B3F8D6013373D30193980801BB
:10FF7000B30EC603B3886800B386CF0293DA0E01CE
:10FF80003383C203B3866600B386DA00338F5F0221
:10FF900063F46600330F4F0113D306013303E3010B
:10FFA000B70A0100232861001383FAFFB3F6660045
:10FFB000B3FE6E0093960601B38DD60183268104AD
:10FFC00033F3660093DE0601330AB302338C630217
:10FFD000935C0A01338FBE02330F8F01338FEC0124
:10FFE000B386D30363748F01B3865601935A0F010E
:10FFF000B386DA00370D0100232AD1009306FDFFF6
:02000004800179
:10000000337FDF00337ADA00131F0F01330F4F0104
:10001000032A8103232CE101B376DA00135F0A017E
:10002000330AAF02B38AA602B30CD702B38C4C01D9
:1000300013DA0A01330A9A01B30CAF02330CE70357
:1000400063749A01330CAC01935C0A01338C8C010C
:10005000232E8101370C0100130DFCFF337AAA0116
:10006000B3FAAA01131A0A01B30C5A01032A0102B6
:10007000B3894901032A010033B80901B389190181
:10008000330A0A01B30B7A01338C6B01B3B819013F
:10009000B30A1C01B3B81A01333C6C01B3681C01EC
:1000A000B3BB0B01B38B780183288101338ABA017A
:1000B000B33DBA0103280101330A1A01B3381A010A
:1000C000232C110183284101B38B0B012320310123
:1000D00023223107832981013388BB01B30818012A
:1000E000B38A3801B33DB8018329C1010328410116
:1000F000330A9A01338C3A01B3B80801B33C9A0130
:1001000003288101B3099C01138B09008329010194
:10011000B3BA0A010328C101B3BB3B01B3EA5801DA
:10012000B3EDBB01333C0C01B33C9B01B38D5D01CE
:10013000B36C9C0133889D01232A01010328C1046B
:100140002324410793580801337DA8013308BD02D9
:10015000B38AA303935B0801B385B802B385550145
:10016000B385BB00B383130363F65501370C01005D
:10017000B383830193DA0501B3837A00370C01005E
:10018000832AC103232E71009303FCFFB3F575008E
:100190003378780093950501B3F37A00B3850501B0
:1001A00013D80A01B30B0703B38AA30233077702FC
:1001B00093DD0A013305A8023307A7003387ED005A
:1001C0006374A700B38B8B01370C0100930DFCFF08
:1001D000135507013377B70133057501131707016D
:1001E000B3FDBA012320A102B38A6202B30DB701A5
:1001F0003305C3023387CE02935C050133075701F1
:100200003387EC00B38BD20363745701B38B8B013C
:10021000935A0701B3897A01B70B0100938AFBFF58
:100220003377570133755501131707013307A700BB
:10023000B30ACF032328E100232231033387C60307
:10024000B38CDF0213550701B38C5C0133059501B4
:10025000338CEF0363745501330C7C01935A050111
:10026000338C8A01B70A0100938AFAFF337555016E
:1002700013150501337757013307E5008329C101C1
:1002800003254101B30ABB00B3B5BA00B30C350175
:10029000832901023385BC00B38ABA01B3BDBA0118
:1002A000B30B3501B389BB01232631038329010137
:1002B000032B4102B335B500B38A3A01B3B93A0111
:1002C00023243103B389BB01B3896901032B810264
:1002D0000325010223283101B38AEA00B3896901A9
:1002E000138B090033B7EA00B3898901232A31014E
:1002F000B389E900B3BBAB00232C31010325C10254
:100300008329C10123265107B33DB501B3BC3C018C
:100310000325010183294102B3EDBB01B3E5BC0014
:10032000B33B35010325410183298102B385B50122
:10033000333C850103258101B33D3B01B3EDBB0196
:100340003337E5003367EC00B38DB50133856602C2
:10035000B38DED00330C6F02935505013387DE0238
:10036000330787013387E500B38BEE03637687019C
:10037000B7050100B38BBB0093550701370C010093
:10038000B38B75019305FCFF3377B700B375B500E8
:10039000B38CA20313170701B305B7003305CD02D1
:1003A0003386C80213570501330696013307C70089
:1003B000B382120363749701B3828201135607015B
:1003C000B70C0100B30256001386FCFF3377C70059
:1003D000131707013376C500338C0F033306C700AC
:1003E000B38F7F023387C303330EC803135507014E
:1003F000B38FCF01B30FF50163F4CF01330C9C0130
:1004000013DE0F01330E8E01370C01001305FCFFC4
:10041000B3FFAF00939F0F013377A700B30CAF0377
:100420003385EF00B38FA603B386D80213D70F012D
:10043000B38696013307D700330F1F036374970108
:10044000330F8F0193560701370C0100338FE601FC
:100450009306FCFF3377D70013170701B3F6DF00CD
:10046000B306D700B38F0E0333876302B38E7E02C9
:10047000935C070133036802B38E6E00B38EDC0118
:1004800063F46E00B38F8F0113D30E01B30FF3012A
:1004900037030100832981011303F3FFB3FE6E00CC
:1004A00033776700939E0E01B38EEE003387B90059
:1004B000B335B700B38D7D01B389BD003307C700E5
:1004C0003336C700338C59003307A700138B09005C
:1004D000B309CC002328E1063337A7003385C901CF
:1004E000B30CE50023283101B389DC00B3B6D90091
:1004F000232A310183290101B3BB7D01B335BB0040
:1005000033B6C900B3325C00B3E2C20033B7EC00CB
:10051000B3E5BB003335C5013365E500B385550050
:10052000B385A500B385E5013386D50033BFE5016A
:1005300083254101B336D600B366DF003387D5018A
:10054000B385A303330FF601232AE1063337D7011E
:100550003306EF003337E600333FFF01336FEF0020
:10056000330DA80313D70501B3837802B383A30126
:1005700033880803B308770063F6A8013707010042
:100580003308E80033F768001317070133F36500F9
:1005900093D8080133036700B388D8000327C1004C
:1005A0008326010033066600B388E8013333660012
:1005B000B369D700B388680033880801336A3A0109
:1005C000939ADA00232E0107232CC10633EA4A014D
:1005D00013070106930501078326C70003260701B9
:1005E0001307470093D636011316D600B3E6C600AC
:1005F000232ED7FEE392E5FE83268106832A010699
:100600000327C106232CD10483264106333A400137
:10061000336A5A01232AD104232EE10423284105F9
:100620009316B70063D40614131AFA0113070105D1
:100630009305C105832607000326470013074700DB
:1006400093D616001316F601B3E6C600232ED7FE86
:10065000E392E5FE0327C105333A40011357170023
:10066000232EE10403270105336A470123284105AE
:1006700003274100B74600009386F6FFB306D70074
:100680006350D02603270105137677006302061016
:1006900013052000032641058325C10513641400BA
:1006A0006386A40E130530006388A40C6392040EC5
:1006B0001375F70013084000630C050D130747007E
:1006C0002328E104133747003306C7003337E60019
:1006D000232AC104032681053306C7003337E60009
:1006E0003307B700232CC104232EE1046F00400A16
:1006F00093870A00032701032328E104032741030A
:10070000232AE10403278103232CE1040327C103E7
:10071000232EE104130720006386EB5413073000F7
:100720006382EBF213071000E394EBF4232E010431
:10073000232C0104232A0104232801046F00805084
:1007400093070A0003270104938B06002328E10482
:1007500003274104232AE10403278104232CE10415
:100760000327C104232EE1046FF0DFFA0327810081
:100770002322E1006FF0DFEF639C0700130787007F
:100780002328E104133787006FF01FF4E39807FE76
:100790000327C1051316B70063500602B706F0FF22
:1007A0009386F6FF3377D700232EE1040327410019
:1007B000B7460000B306D700130701051305C105AE
:1007C000032607008325470013074700135636000A
:1007D0009395D5013366B600232EC7FEE312E5FEDE
:1007E000378700001307E7FF634CD7080327C105CD
:1007F00013573700232EE104138706000325C10594
:10080000131717019397F7001357170133E7E70002
:100810002316A1062317E1068325010503264105BA
:10082000832681058327C106630404007320140016
:100830008320C10B0324810B2320B9002322C9008C
:100840002324D9002326F9008324410B8329C10ADC
:10085000032A810A832A410A032B010A832BC10937
:10086000032C8109832C4109032D0109832DC10823
:10087000130509000329010B1301010C6780000017
:1008800013072000638AE404130730006384E40242
:100890006394040237870000232E0104232C0104F3
:1008A000232A0104232801041307F7FF13645400CB
:1008B0006FF0DFF4E38007FE1307F0FF232EE1045F
:1008C000232CE104232AE1042328E10437870000D4
:1008D0001307E7FF6FF09FFDE38007FE6FF09FFBBC
:1008E00013071000639006080326010583254105C0
:1008F00003258105137876000327C105630E0804DC
:1009000013082000136414006386040513083000E4
:10091000638A0403639204041378F600930840008A
:10092000630C18031306460013364600B385C50052
:1009300033B6C5003305C5003336C5003307C700DD
:100940006F008001639A0700130686001336860045
:100950006FF0DFFDE39A07FE1357470113471700B7
:1009600013771700930510003386D5409306400790
:1009700063CCC626935856409306000093050000AA
:10098000639815051376F601139828006310060680
:1009900013053000130601059305000033051541CA
:1009A0003303060103230300938515001306460055
:1009B000232E66FEE356B5FE93054000B38815412D
:1009C0009305100063501009938508006F0080079D
:1009D00013952500130801053305A800032505001C
:1009E00093851500B3E6A6006FF09FF99305010803
:1009F000B385050183A505FD130E0002330ECE401D
:100A0000B395C501B3E6B6001305300093050105A3
:100A1000338805011303000033051541130848000E
:100A20006346A30213080108131525003305A80027
:100A30000328C10593054000B38515413356C8000E
:100A40002328C5FC130540006F004004931E2300BB
:100A500093050105032F0800B38ED5018325C8FF38
:100A6000331FCF0113031300B3D5C500B3E5E50170
:100A700023A0BE006FF09FFA13962500130801050E
:100A80003306C8002320060093851500E396A5FED3
:100A900003260105B336D000B3E6C6002328D104EF
:100AA00013F67600630E0604130620000328C10522
:100AB000136414006388C40A130630006388C406F4
:100AC0006390040413F6F600630CB6020325410597
:100AD000938646002328D10493B646003385A600AA
:100AE000B336D500232AA104032581053385A6004A
:100AF000232CA1043335D50033060501232EC10470
:100B00008326C1051396C600635A0608232E0104E6
:100B1000232C0104232A0104232801041364140054
:100B20006310070C130710006FF05FCDE39A07FC0A
:100B300083254105938686002328D10493B6860039
:100B4000B385B600B3B6D500232AB1048325810549
:100B5000B385B600232CB104B3B5D50033860501A7
:100B60006FF0DFF9E38E07F80326410593868600D0
:100B7000832581052328D10493B686003386C600D9
:100B8000B336D600232AC1043386B600232CC10411
:100B90003336D600330606016FF05FF69306010583
:100BA0001305C10503A6060083A5460093864600EB
:100BB000135636009395D5013366B60023AEC6FEB4
:100BC000E312D5FE8326C10593D63600232ED10429
:100BD000E30607C213771400E30207C213070000FD
:100BE000136424006FF09FC183264105032701058C
:100BF0003367D700832681053367D7008326C10575
:100C00003367D700630E0702232E0104232C01044F
:100C1000232A01042328B1041307200013641400BD
:100C2000638EE402130730006382E402130750006E
:100C30006382040203270105135737002328E104C8
:100C400013642400130700006FF05FBBE39407FEFA
:100C5000130790002328E1046FF0DFFDE39A07FEFD
:100C60006FF05FFD37870000232E0104232C010461
:100C7000232A0104232801041307F7FF6FF01FB88C
:100C8000130101F983A6050003A7450083A785008A
:100C9000232291062320210783A4C5001309050000
:100CA0002326110623248106232E3105232C4105FA
:100CB000232A510523286105232671058328060070
:100CC0000325460083258600832EC600F3292000D5
:100CD000232CF1022324F1009397040113941400B0
:100CE00093D70701232E91022328D102232AE10260
:100CF0002320D1002322E1002326F1001354140104
:100D000093D4F401930F01001308C1008327080056
:100D10000327C8FF1308C8FF939737001357D7015D
:100D2000B3E7E7002322F800E3920FFF83260100D8
:100D300093970E01139E1E009396360093D70701DA
:100D4000232ED1032320D10023281103232AA1021B
:100D5000232CB10223281101232AA100232CB10046
:100D6000232EF100135E1E0193DEFE01130F01011D
:100D70001306C101832706000327C6FF1306C6FF1B
:100D8000939737001357D701B3E7E7002322F60004
:100D9000E312CFFE03270101B78700009387F7FF17
:100DA000131737002328E1006310FE028325810119
:100DB00083274101B3E7B7008325C101B3E7B7003B
:100DC000B3E7E7006394070093CE1E00B307C44166
:100DD000E39E9E3A6350F03A032841008328810045
:100DE0008325C10063120E10832E4101032581016A
:100DF000832FC10133E3AE003363F3013363E300B8
:100E000063120304378700001307F7FF6390E702BC
:100E1000336718013367B7003367D70063080700EB
:100E20001397D50063440700130E00012320D1025D
:100E300023220103232411032326B10213040E00ED
:100E40006F00000A1383F7FF631A03043387E60079
:100E5000B336D70033860E01B307D600B3B6D7003A
:100E6000333806013368D8002322F102B307150195
:100E70002320E1023387070133380701B3B7170195
:100E8000B3E70701B385BF00B385B7002324E102B0
:100E90002326B102930710006F000023378700005C
:100EA0001307F7FF6384E7006F1010003367180122
:100EB0003367B7003367D70013040000630A0700E5
:100EC0003704040033F48500133414001314440071
:100ED0002320D10223220103232411032326B1025C
:100EE000130800006F000074378700001307F7FF36
:100EF0006312E404B3671801B3E7B700B3E7D700A0
:100F000013070000638A07003707040033F7E50082
:100F100013371700131747002320D10223220103A0
:100F2000232411032326B1029307040013040700AE
:100F30006FF01FFB0327C101370508003367A700C7
:100F4000232EE100130740076354F7006F108076EB
:100F50001383070013555340130E0000930700003E
:100F60006396A7041373F30113172500631C03048E
:100F700013033000930700003303A340B30EE600D1
:100F800083AE0E009387170013064600232ED6FF6C
:100F9000E356F3FE930740003385A7409307100004
:100FA000635CA006930705006F00000713972700F6
:100FB0003307EF000327070093871700336EEE0017
:100FC0006FF01FFA93070104B387E70083A707FDBB
:100FD000930F0002B38F6F40B397F7013306EF0012
:100FE00013073000336EFE00930E00003307A74056
:100FF0001306460063C6EE0213060104131727000A
:101000003307E6000326C10193074000B387A740DA
:1010100033536600232867FC130640006F00C003AB
:101020008327C6FF8323060093922E00B3D7670061
:10103000B393F301B3025F00B3E7770023A0F2009C
:10104000938E1E006FF0DFFA139727003307EF002F
:101050002320070093871700E398C7FE03270101A9
:10106000B337C001B367F7002328F10083270101DC
:1010700003264101B387F600B3B6D7003306C80094
:101080002320F102B307D600B3B6D7002322F10222
:1010900083278101333806013368D800B387F8000D
:1010A00033870701B3B717018328C101333807011C
:1010B000B3E70701B3851501B385B7002324E10227
:1010C0002326B102930704000327C1029316C70029
:1010D00063C406006F10404DB706F8FF9386F6FF15
:1010E0003377D7002326E1020327010293871700F5
:1010F0001305C1029316F701130701020326070027
:101100008325470013074700135616009395F501F2
:101110003366B600232EC7FEE312E5FE0327C102A5
:10112000135717002326E1023337D000832601022C
:1011300033E7E6002320E102378700001307F7FFBB
:10114000639AE77CE380090213073000E398E90221
:10115000E38A04009307F0FF2326F1022324F1021F
:101160002322F1022320F102B78700009387E7FFD3
:101170006F00500003264101832581018328C101AE
:10118000638E072EB3078E406310041003234100C3
:1011900003258100032FC100B36EA300B3EEEE015F
:1011A000B3EEDE0063940E04B78600009386F6FF6C
:1011B0006390D702B366B600B3E61601B3E6E60065
:1011C000638806009396D80063C4060013040001E8
:1011D0002320E1022322C1022324B102232611038A
:1011E00013080000638E072C6F00C043938EF7FF37
:1011F00063980E04B386E60033B7E6003308C300F5
:10120000B307E80033B7E7003336C8003366E600BB
:101210002322F102B307B5003387C7003336C70076
:10122000B3B7B700B3E7C700B3081F01B38817010E
:101230002320D1022324E102232611036FF09FC54E
:10124000B78600009386F6FF6384D7006F10C0470F
:10125000B366B600B3E61601B3E6E6001304000079
:10126000638A06003704040033F488001334140042
:10127000131444002320E1022322C1022324B102DB
:10128000232611036FF0DFC5B78600009386F6FFB3
:101290006310DE04B367B600B3E71701B3E7E700F6
:1012A00013040000638A07003704040033F4880045
:1012B00013341400131444002320E1022322C1023A
:1012C0002324B1022326110393070E006FF05FC1A0
:1012D0008326C10037050800B3E6A6002326D10007
:1012E0009306400763D4F6006F10C03E938E07004C
:1012F0009307000233C3FE02130F000093070000A0
:1013000063CA670493060300635403009306000056
:1013100093F7FE0113152300639A07049306300028
:10132000B3866640B30EA80083AE0E009387170005
:1013300013084800232ED8FFE3D6F6FE930740009B
:1013400033836740930710006350600893070300DE
:101350006F00800793962700B386DF0083A6060000
:1013600093871700336FDF006FF09FF99307000238
:10137000B3EEFE029396260013080104B306D800CC
:1013800083A606FC3385AF0093020000B387D741E4
:10139000B396F600336FDF0093063000B3866640E5
:1013A0001305450063C6D202130501049396260077
:1013B000B306D5000325C10093074000B3876740FB
:1013C000B35ED50123A0D6FD130530006F00C00326
:1013D0000328C5FF03240500939322003358D80146
:1013E0003314F400B3837F003368880023A0030123
:1013F000938212006FF0DFFA93962700B386DF0026
:1014000023A0060093871700E358F5FE832601000A
:10141000B337E001B3E7F6002320F1008327010092
:1014200083264100B307F70033B7E700B306D600C1
:101430002320F102B387E60033B7E7002322F1024D
:101440008327810033B6C6003366E600B387F50014
:101450003387C700B3B7B7008325C1003336C70051
:10146000B3E7C700B388B800B38817012324E102AB
:101470002326110393070E006FF01FC5B78E0000DF
:10148000930714001388EEFF33F80701032F410080
:10149000832F81000323C100631A083E3365FF01D7
:1014A000336565003365D500631204306314050E9F
:1014B0002320E1022322C1022324B10223261103A7
:1014C0008325010203264102832681020327C102EC
:1014D000B3E7C500B3E7D700B3E7E70063940700BD
:1014E0006F10C00F232AC1022328B102232CD1027E
:1014F000232EE102130601039307C10303A707008C
:1015000083A6C7FF9387C7FF1317170093D6F6016B
:101510003367D70023A2E700E312F6FE8327010317
:101520009397170013F77700631407006F10800973
:10153000130720008326C103136414006394E90099
:101540006F100008130730006394E9006F10400625
:10155000638409006F10000713F7F70013064000BB
:101560006314C7006F1000069387470093B74700C6
:10157000032741033387E7003337F70083278103CD
:10158000B307F700B3B7E700B387D700232EF10204
:101590006F104003B367B600B3E71701B3E7E70086
:1015A000639C07002320D1022322E1032324F103BB
:1015B000232661026FF0DFF03387E600B307CF0028
:1015C000B336D7002320E1023387D70033B6E701D3
:1015D000B336D700B366D600B385BF003386D500D7
:1015E000B336D600B3B5F501B3E5D500B3081301A2
:1015F000B38515012322E1022324C1029397C5007C
:1016000063C607002326B1026FF09FEBB707F8FF10
:101610009387F7FFB3F5F5002326B1021308040002
:101620009307100003270102937677006380060674
:10163000930620000325C10213641400E380D97EC1
:1016400093063000E380D97A639209049376F70019
:1016500013064000638CC60283254102130747002E
:101660002320E10213374700B305B70033B7E50085
:101670002322B10283258102B305B7002324B102DE
:10168000B3B5E500B386A5002326D10263080800A0
:101690001377140063040700136424000327C102B6
:1016A0009316C70063D20602B7860000938717001F
:1016B0009386F6FFE380D77AB706F8FF9386F6FFA6
:1016C0003377D7002326E102130701029305C102F5
:1016D00083260700032647001307470093D63600EA
:1016E0001316D601B3E6C600232ED7FEE392E5FE1D
:1016F0000327C10237860000935637002326D10204
:101700001307F6FF639AE7028325410203270102CC
:101710003367B700832581023367B7003367D7008B
:10172000630C07002326C1022324010223220102A5
:1017300023200102930400008325C102939717011F
:1017400093D717019394F400B3E4F400231EB1027D
:10175000231F9102032601028326410203278102EF
:101760008327C10363040400732014008320C1068F
:10177000032481062320C9002322D9002324E90061
:101780002326F900832441068329C105032A810504
:10179000832A4105032B0105832BC104130509008E
:1017A000032901061301010767800000938EFEFFE5
:1017B0006314D409E3080576370404003374830006
:1017C00013341400131444006310DE0BB367B60027
:1017D000B3E71701B3E7E700E38E07729397D800EA
:1017E000E3DE077263040506B78700002326F102D3
:1017F00023240102232201022320010213060102F5
:101800009307C10203A7070083A6C7FF9387C7FFFB
:101810001317370093D6D6013367D70023A2E7000A
:10182000E312F6FE8327010293040000939737002A
:101830002320F1026F0080026316DE011304000012
:101840006FF0DFF813040000631005022320E102AB
:101850002322C1022324B10223261103B7870000EB
:101860009387F7FF6FF01FDC3366B600B36816018D
:1018700033E7E800E31A07F62320D1022322E1032D
:101880002324F103232661026FF05FFD3387E60016
:10189000B336D7003306CF002320E1023307D6004A
:1018A000B336D7003336E601B366D6003386BF00C1
:1018B0002322E1023307D600B335F6013336D700D1
:1018C00033E6C500B3081301B30816012324E1026F
:1018D00023261103130701029305C1028326070083
:1018E000032647001307470093D616001316F60188
:1018F000B3E6C600232ED7FEE392E5FE378700004D
:101900001307F7FF638EE7000327C1021357170081
:101910002326E10213080000130400006FF09FD09B
:1019200063820904130730006398E902638C0402A0
:101930009307F0FF2326F1022324F1022322F10270
:101940002320F102B7870000130800009387E7FF08
:10195000130450006FF01FCD13072000E39AE9FC39
:10196000E38804FC2326010223240102232201022E
:1019700023200102130800006FF09FFD13072000D1
:10198000639AE9FC638804FC6FF0DFFD6354F03276
:1019900003254100032881008328C10063140E1031
:1019A000832F4101832E81010323C101B3E5DF01B0
:1019B000B3E56500B3E5E5006390050437870000F3
:1019C0001307F7FF6390E7023367050133671701D9
:1019D0003367D700630807001397D80063440700F4
:1019E000130E00012320D1022322A102232401038C
:1019F000232611036FF08FC49385F7FF63940506C8
:101A00003387E640B307F54133B6E600333EF500D1
:101A10003386C7409307000063F6E6003385AF4086
:101A20009337150033E5C701B307D841B336F80043
:101A3000B387A7406306050033880E41933518002D
:101A4000B3886840B3E5D500B385B8402326B1021A
:101A50002324F1022322C1022320E1029307100074
:101A60006F000023378700001307F7FFE39EE74668
:101A700033670501336717013367D700130400008C
:101A8000630A07003704040033F488001334140099
:101A9000131444002320D1022322A1022324010392
:101AA0006FF00FFE378700001307F7FF631EE40295
:101AB000B3670501B3E71701B3E7D70013070000C9
:101AC000638A07003707040033F7E800133717006D
:101AD000131747002320D1022322A102232401034C
:101AE000232611036FF04FC40327C101B705080077
:101AF0003367B700232EE10013074007E34AF73EA0
:101B00009385070013D35540130E00009307000080
:101B10006396670493F5F50113172300639C05048E
:101B20009305300093070000B3856540B30EE600CF
:101B300083AE0E009387170013064600232ED6FFB0
:101B4000E3D6F5FE93074000338367409307100008
:101B5000635C6006930703006F000007139727007C
:101B60003307EF000327070093871700336EEE005B
:101B70006FF01FFA93070104B387E70083A707FDFF
:101B8000930F0002B38FBF40B397F7013306EF0006
:101B900013073000336EFE00930E000033076740DA
:101BA0001306460063C6EE0213060104131727004E
:101BB0003307E6000326C10193074000B38767405F
:101BC000B355B6002328B7FC130640006F00C003CE
:101BD0008327C6FF8323060093922E00B3D7B70056
:101BE000B393F301B3025F00B3E7770023A0F200E1
:101BF000938E1E006FF0DFFA139727003307EF0074
